:020000040800F2
:10000000F8FF0120BDFA04085B48040849480408C9
:100010005D4804086D4804087D480408000000009D
:100020000000000000000000000000008D480408EF
:100030008F48040800000000355804086D58040873
:1000400069F904087D4904088949040891490408AC
:1000500099D7040869F904081149040817490408E4
:100060001D4904082349040829490408097B040898
:10007000197B0408297B0408397B0408497B0408A0
:10008000597B0408697B040869F9040869F90408C4
:10009000D59C0408DD9C0408E59C04082F4904084D
:1000A000A5490408AB490408BD490408C34904082C
:1000B000C9490408CF490408D5490408494A040835
:1000C0004F4A0408554A04085B4A040869F90408C1
:1000D00069F90408254A04082B4A0408314A04082F
:1000E00053490408834904089D480408014A040848
:1000F000074A04081F4A0408194A0408797B0408BF
:1001000069F9040825E10408DD49040869F90408CF
:10011000374A04083D4A0408F5490408FB49040825
:10012000897B0408997B0408A97B0408B97B04082F
:10013000C97B0408000000000000000069F9040801
:10014000EB9C0408F39C0408FB9C040891480408F9
:10015000D97B0408E97B0408F97B0408434A0408B6
:1001600069F9040869F9040869F9040869F90408D7
:1001700069F9040869F904080000000000000000A3
:1001800069F9040869F9040842884378007843EA69
:10019000022340EA032070470B0A017043700B0CE6
:1001A000090E8370C1707047036A0239023B8B42AB
:1001B00083BFC389406B01FB0300002070470246E8
:1001C00000F10B010020C30143EA500312F8010BB8
:1001D00050FA83F38A42D8B2F5D1704737B50D464D
:1001E000044620B9092000232B6003B030BD03680A
:1001F000002BF7D05A79002AF4D081885A8991428D
:10020000F0D10DF107020621186802F0F5FA002876
:10021000E8D19DF8070010F00100E3D12368E3E77F
:1002200038B50368044618785D1C20B140F2B5115A
:1002300057F0FAFD08B1256038BD4FF0FF30FBE7FD
:10024000CA7E8B7E032843EA022301BF487D0A7DD4
:1002500042EA002243EA024318467047C2F30723EA
:100260008A76CB760378032B01BF120C0A75120A2B
:100270004A75704770B5C37904460BB9002070BD4C
:1002800000F13C06826B00680123314602F09FFAC0
:1002900080B9A16BE36A626AE071CB1A9342EDD236
:1002A000A379022BEAD10A4401233146206802F0E7
:1002B0008EFAE3E70120E2E7836B8B4270B50646D6
:1002C0000D4612D0FFF7D6FF044660B92A46012337
:1002D00006F13C01306802F06BFA00281CBF4FF0B9
:1002E000FF350124B563204670BD0024FBE7000004
:1002F000002310B5C3714FF0FF3383630446FFF74B
:10030000DBFF18BB94F83B2294F83A3243EA02230D
:100310004AF6552293421BD194F83C30EB2B03D084
:100320001833DBB2012B15D803220B4904F17200FC
:100330003FF010FD48B10522084904F18E003FF05E
:1003400009FD002814BF0220002010BD0420FCE796
:100350000320FAE70220F8E75F2C0708632C070860
:100360002DE9F043437987B0044601F0FE059BB1C7
:1003700006210DF10702006802F03EFA9DF8070021
:10038000C10709D4002D00F0BC8010F0040000D09B
:100390000A2007B0BDE8F083002363710DF1070266
:1003A0000521206802F028FA9DF80730DA0700F1ED
:1003B000AA800DB15B07EBD400212046FFF798FF20
:1003C0000228034603D0012824D8257975B304F206
:1003D0000225002102AF15F8040C10B12846FFF7E2
:1003E000D3FE47F821000131042905F11005F2D1AF
:1003F000267906B1013E57F826507DB129462046A0
:10040000FFF776FF0346227952B9012B0ED9013648
:10041000032EF0D9042B07D10120BAE70323F2E71A
:10042000042BF9D0012B01D90D20B2E794F8482014
:1004300094F8473043EA0223B3F5007FF4D194F8EF
:10044000533094F8526056EA032604D104F1600058
:10045000FFF79AFE064694F84C90666209F1FF3366
:10046000012B84F80690DFD894F84970BBB2E38181
:10047000002BD9D07B1E3B42D6D194F84E3094F855
:100480004D8048EA032818F00F0FA4F80C80CBD158
:1004900094F8501094F84F0050EA012003D104F171
:1004A0005C00FFF771FE94F84B2094F84A3053EA51
:1004B0000223B9D006FB09F903EB18124A44824221
:1004C000B2D8811AB1FBF7F10029ADD0454881427D
:1004D000AAD84FF6F570814217D903271BE0B8F16F
:1004E000000FA1D0022F4FEA410018BF40184B4423
:1004F00018BF01F0010123630CBF014601EB50015D
:1005000024E0284645E7032043E740F6F577B94263
:1005100094BF0127022702312B442A44032F216272
:10052000A562E3626263DAD194F8672094F86630DA
:1005300053EA02237FF478AFB8F1000F7FF474AF71
:1005400004F16800FFF720FE2063890001F2FF112B
:10055000B6EB512FFFF468AF4FF0FF33C4E905331A
:10056000032F4FF0800323722FD194F86D2094F85D
:100570006C3043EA0223012B27D1691C2046FFF788
:100580009BFE10BB94F83B2294F83A32207243EA67
:1005900002234AF65522934217D104F13C00FFF79B
:1005A000F3FD114B984210D104F50870FFF7ECFDF4
:1005B0000E4B984209D104F50970FFF7E5FDA061E3
:1005C00004F50A70FFF7E0FD6061094A677113885E
:1005D00001339BB2138063810020064B2361E061ED
:1005E000D7E600BFF5FFFF0F5252614172724161C1
:1005F000281900202A19002001292DE9F047054675
:100600000C46174672D9036A8B426FD94379022B85
:100610003FD0032B50D0012B68D101EB5108C16AA8
:1006200001EB5821FFF748FE064638BB05F13C09AF
:1006300008F1010AC8F3080814F001041FBF19F8F3
:10064000083003F00F023B0103F0F00314BF134323
:10065000FBB209F80830E96A0123EB7101EB5A217A
:100660002846FFF729FE064640B9CAF3080A44B1F6
:10067000C7F3071709F80A700123EB713046BDE88C
:10068000F08719F80A30C7F3032723F00F031F433D
:10069000F0E7C16A01EB1421FFF70EFE06460028C1
:1006A000ECD1640005F13C0304F4FF741A191F55E2
:1006B000C7F307275770DFE7C16A01EBD411FFF7D3
:1006C000FBFD06460028D9D1A40005F13C0304F443
:1006D000FE741C442046FFF757FD27F0704700F0DA
:1006E000704139432046FFF757FDC5E70226C5E7AD
:1006F0000129F8B505460C4652D9036A99424FD2F2
:100700004379022B29D0032B38D0012B48D101EBA0
:100710005106C16A01EB5621FFF7CEFD10B14FF033
:10072000FF30F8BD771CE96AC6F308062E4401EBDA
:100730005721284696F83C60FFF7BEFD0028EED111
:10074000C7F308073D44E30795F83C0046EA00205C
:100750004CBF0009C0F30B00E3E7C16A01EB1421B1
:10076000FFF7AAFD0028DAD164003C3504F4FF74D9
:100770002B19285D5B7840EA0320D2E7C16A01EBC0
:10078000D411FFF799FD0028C9D1A40005F13C0060
:1007900004F4FE742044FFF7F7FC20F07040C0E73B
:1007A0000120BEE7B1F5001FF8B506460D4601D39E
:1007B0000220F8BDCA06FBD1826804683161C2B963
:1007C0006379022B01D9236BA3B9A389B3EB551F1E
:1007D000EED9236BB361B3697261002BE8D003EBF0
:1007E00055233C34C5F308052C44B361F461002063
:1007F000DFE71346E7891A467F02BD42114604D25D
:100800002046FFF7D1FCB061E5E73068FFF770FFE5
:10081000431C024606D00128CAD9236A8342C7D99D
:10082000ED1BEAE70120C4E72DE9F04180460568A9
:100830000F4649B96E69CEB12B6AB34298BF012603
:10084000AB69ABB9002409E02846FFF751FF012846
:10085000044658D9421C04D14FF0FF342046BDE86D
:10086000F0812B6A8342F9D83E46E9E70126E7E7A3
:10087000BE4215D12B6AD8F80000741C9C4228BFD8
:1008800002242146FFF734FF01283CD0431CE3D06B
:10089000D8B16B69012B03D92A6A934238BF1E462F
:1008A00034462B6A0134A34202D8012ECAD902244D
:1008B0002146D8F80000FFF71BFF40B1012822D0E5
:1008C0000130C9D0B442ECD1BCE7002CE8D04FF0E5
:1008D000FF3221462846FFF78FFE90B957B92A6AA2
:1008E000AB696C61023A93420FD92B7A43F0010352
:1008F0002B72B3E7224639462846FFF77DFE0028D3
:10090000EDD00128A8D00124A8E7013BAB61ECE7BA
:10091000F8B50D46012D074611462CD90468236A07
:10092000AB4228D92AB14FF0FF322046FFF764FED0
:1009300030B929463868FFF7DBFE064608B90020C3
:10094000F8BD012817D0431C17D0002229462046A5
:10095000FFF752FE0028F3D1226AA369911E8B4251
:1009600005D20133A361237A43F001032372B2421B
:100970003546DED8E3E70220E2E70120E0E7F8B5FC
:1009800005460E46FFF776FC0446F8B93146284680
:10099000FFF70AFC05F13C060746A8634FF4007216
:1009A000214630463FF0C2F9EB899C4204D3E889E6
:1009B000001B18BF0120F8BD01233A1931462868F1
:1009C00001F005FF0028F2D10134EDE70120F2E744
:1009D0002DE9F843076905682037B7F5001F24BFE4
:1009E0000023836183690446894673B1C7F308080D
:1009F000B8F1000F39D141690133836139B9AB894D
:100A0000B3EB571F31D80023A36104200BE0EB891F
:100A1000013B13EA572328D12846FFF769FE012836
:100A2000064602D80220BDE8F883421C01D101200D
:100A3000F9E72B6A834212D8B9F1000FE3D061695C
:100A40002046FFF7F1FE0646A8B10128EAD0431C74
:100A5000EDD001462846FFF792FF0028E7D16661F6
:100A600031462846FFF7A0FBA0613C35454427618D
:100A7000E5610020D7E70720D5E7F8B50F4600214C
:100A800004460668FFF78EFEA8B90546A169304600
:100A9000FFF712FC78B9E3691B78E52B00D01BB98E
:100AA0000135BD4201D1F8BD054601212046FFF7C1
:100AB0008FFF0028EAD0042808BF0720F3E70000D2
:100AC0002DE9F84FFF250668DFF8248182460F469E
:100AD0002C464FF0040B4FF6FF79DAF8181019B9CD
:100AE000BBF1000F76D065E03046FFF7E5FB8346AB
:100AF00000285FD1DAF81C000278002A74D0C37A8B
:100B0000E52A03F03F038AF8063059D02E2A57D041
:100B100023F02001A1F1080CDCF1000141EB0C01F4
:100B2000B9424DD10F2B50D1510647D5DAF81030CC
:100B3000457BCAF82C3002F0BF02437BAB423FD169
:100B4000C17E837E43EA01231BB2002B38D101789A
:100B5000D6F810C021F0400101390D2461434FF057
:100B6000010E13F8084000EB040B045D9BF801B084
:100B700044EA0B24BEF1000F24D0FF2920D82CF822
:100B80001140A646013101330D2BEAD103785B06F3
:100B900007D5BEF1000F04D0FF2911D800232CF88F
:100BA0001130541EE4B200215046FFF711FF834676
:100BB000002892D00023CAF818300DE09442BCD02F
:100BC000FF24F0E74C45DED0FAE744B9FFF7F7FA27
:100BD000A84204D14FF0000B5846BDE8F88F4FF003
:100BE000FF33CAF82C30F7E74FF0040BE2E700BF01
:100BF000402C0708C16A4B1C2DE9F04104460568EA
:100C0000066918D1E5274FF00108A1692846FFF7CA
:100C100053FB60B9E3691F7085F807802369B3420D
:100C20000DD201462046FFF7D3FE0028EDD0042860
:100C300008BF022003E0FFF7B5FD0028E2D0BDE8C1
:100C4000F08100002DE9F04F002185B00446D0F876
:100C500000A0FFF7A7FD8046002840F093804FF0EA
:100C6000FF334FF0FF09E3624E46A1695046FFF79C
:100C700023FB8046002840F08580E5692F78002F0F
:100C800000F08480EA7AE52F02F03F03A37103D0DD
:100C9000120705D50F2B05D04FF0FF33E36258E064
:100CA0000F2B5DD194F82B30580648D479064ED5D9
:100CB000236995F80D90E36207F0BF076B7B4B4506
:100CC00047D1EB7EAE7E46EA032636B2002E40D1F7
:100CD00095F80080DAF810B008F03F0808F1FF330B
:100CE0004FF00D0808FB03F801212A4BF25CAB180A
:100CF0005878AB5C43EA002369B3B8F1FF0F28D8FA
:100D00001846039357F0A4F808F1010202903BF84B
:100D10001800019257F09CF80299814219D1039B67
:100D2000019A1946904601360D2EDED12B785A06CF
:100D300003D511B13BF818305BB9013FFEB2002179
:100D40002046FFF745FE804600288ED01AE0BE42BE
:100D5000B4D0FF26F3E74FF6FF729342E3D0F8E7F3
:100D600026B92846FFF72BFA48450BD094F82B30CC
:100D7000DB0791D40B2204F1200128463EF0EAFF64
:100D8000002889D1404605B0BDE8F08F4FF0040837
:100D9000F8E700BF402C07082DE9F04F90F82BB082
:100DA0001BF0A00489B0054640F0828007683A69CC
:100DB00032F81430002B63D105F1200696E80700C5
:100DC0000DF114091BF0010F89E8070077D04023CB
:100DD00085F82B304FF0010899E80700B4463B69CD
:100DE000ACE803002CF8022BB8F1050F4FEA1242D1
:100DF0008CF8002058D9981E424630F8021F00296E
:100E000040D1072102F00F0C0CF13000392801F11C
:100E1000FF3103AB88BF0CF1370003EB010C120963
:100E20008CF80100EED108AB58184FF07E0C00F89A
:100E300014CC8A4204D0B05C202802F1010C35D1D8
:100E4000324407299BBF08AB5818202010F8140C17
:100E500002F8010BA2EB060098BF01310728F0D978
:100E60002846FFF7EFFE824628BB08F10108B8F1DB
:100E7000640FB1D14FF0070A504609B0BDE8F08FBA
:100E8000013495E74FF0100C01F0010E0EEB420219
:100E9000D30344BF82F4883282F02102BCF1010CFA
:100EA0004FEA5101F0D1A8E74246AAE76246C0E7FF
:100EB0004FF0060AE0E70428DED185F82BB01BF0DE
:100EC000020F1BBF0C340D230124B4FBF3F418BF35
:100ED000013421462846FFF7D0FD82460028CBD1B9
:100EE000013C56D029692846A1EB4411FFF75AFC72
:100EF00082460028C0D13046FFF761F94FF6FF79EE
:100F00008046A9693846FFF7D7F982460028B3D151
:100F1000EB69D7F810E083F80D800F22E1B24FF0B3
:100F20000D0CDA724A1E0CFB02F218739876D87612
:100F30000192844648451FBF019A3EF812000132D3
:100F40000192234A1CF802A00CF1010C03EB0A0BDE
:100F500003F80A004FEA102A002808BF4846BCF1EF
:100F60000D0F8BF801A0E5D1484503D0019A3EF85A
:100F700012200AB941F0400119700123FB710021D0
:100F80002846FFF725FD824600287FF475AF013C17
:100F9000B7D1A9693846FFF78FF9824600287FF458
:100FA0006BAF01462022E8693EF0C0FE03CEEB693C
:100FB00018605960B278318819819A7295F82B308F
:100FC000EA6903F0180313730123FB7154E700BFB0
:100FD000402C0708F8B50446FFF74CF905460028F1
:100FE00042D16379032B37D1277A012F34D104F111
:100FF0003C0601464FF4007230463EF097FE552302
:1010000084F83A32AA2384F83B32522341227221D7
:1010100084F83C3084F83D30612384F83E3084F815
:101020003F2084F8222284F8233284F8201284F8A6
:10103000211204F50970A169FFF7AEF8616904F5A2
:101040000A70FFF7A9F8A26A20680132A2633B4642
:10105000314601F0BCFB257200221146206801F0E8
:10106000CBFB003018BF0120F8BD2DE9F047002769
:10107000D0F800908F75836906460C46002B00F06F
:101080009680C36A013370D1F0690023451E19466A
:101090002E2715F8012F202A01F1010110D0052A71
:1010A00008BFE522092906D10B2B9EBF04EB030CD8
:1010B00001338CF8097004EB030C01338CF8092020
:1010C0000B29E6D1E21800215172A27D002A5CD1E1
:1010D000002B51D004F109010825134611F8012B0A
:1010E000002A4CD092B22E2AA2F1410708BF102547
:1010F000192F03D8077B3D4218BF20320A730133F2
:10110000ECE7B8F1000F05D100F520539BB2B3F521
:10111000006F13D340F2B51140EA084056F064FE68
:10112000FF28C5F1FF0A18D9BAF1010F20D96319B8
:10113000020A9A75D87502231D44002002378046A2
:10114000D9F81030D85B0028DBD1B8F1000F18BFF8
:10115000002525440023AB7596E748B1BAF1000F8E
:1011600008D0631998750123E6E7B8463D46E7E7DE
:101170000025EAE75546E8E73F23A375012323440A
:1011800000229A75037B03B96372F169CB7A2372EB
:1011900001F11C00FEF7F8FF2060CA7D8B7D43EA59
:1011A0000223E3804A7E0B7E43EA0223A380BDE84C
:1011B000F08700002DE9F04F87B0036801930B78AA
:1011C0002F2B0646894601D05C2B0AD14A4613785C
:1011D0002F2B914602F10102F9D05C2BF7D00023AE
:1011E00001E0019BDB69B36099F800301F2B00F22E
:1011F0002C81802386F82B3000213046FFF7D2FA6D
:1012000007B0BDE8F08FFE2D00F248812AF81530B6
:10121000013520E109F101020592DDF8149099F8F9
:1012200000202F2AF6D05C2AF4D01F2B8CBF00247C
:101230000424012D2CD1BAF800302E2B2ED10023FE
:101240002AF8153006F120029D4294BF20212E215C
:1012500001330B2B02F8011BF6D144F0200486F871
:101260002B403046FFF7EEFC96F82B30002800F0BC
:10127000DA800428C4D1990603F0040240F1CF803B
:10128000002A00F0E280802386F82B300020B7E7A8
:10129000022D03D1BAF802302E2BCCD00AEB450335
:1012A0009DBB00230AEB45022AF81530002D00F003
:1012B000F5803AF81310202903F101002DD00BB965
:1012C0002E2902D144F00304E4B232F8021D2E2983
:1012D00001D0013DF9D14FF020314FF0000871628B
:1012E0003162C6F827104FF0080B47463AF8130052
:1012F0005A1C20B3202803D02E2810D1954212D09A
:1013000044F00304E4B21346F0E733F8022D202A38
:1013100001D02E2AC5D1013DC2E70346C9E7D84511
:1013200005D295423ED1BBF10B0F33D102E0BBF1A8
:101330000B0F29D144F00304E4B24FF00B0B96F8E5
:101340002030E52B04BF052386F82030BBF1080FC1
:1013500004BFBF00FFB207F00C030C2B03D007F053
:101360000303032B02D144F00204E4B2A3073FF5C8
:1013700076AFFD0744BF44F01004E4B2780744BFE1
:1013800044F00804E4B26AE7954203D044F0030451
:10139000E4B2D4D3BF00FFB22A464FF00B0B4FF09C
:1013A0000808B0E77F2838D944F00203DBB240F2E6
:1013B000B5110392029356F017FD10F0800FDDE98E
:1013C000023210D000F07F003F49085C30B13F4C42
:1013D00014F8011F002965D08142F9D143F00303BD
:1013E000DBB25F2011E0FF28F0D90BF1FF31884517
:1013F00004D344F00304E4B2D84684E706EB0801C2
:10140000040A81F8204008F1010806EB08011C4697
:1014100081F8200008F1010875E72346D7E7002A84
:1014200008BF0520ECE65A073FF5EAAEB379DB06C4
:1014300036D5019B03F13C013369C3F3080319441A
:10144000019B5879FEF7FCFEB0603368CDF814902C
:10145000D3F810A0002505A8FEF7E2FE421C1DD01F
:10146000B0F5803F24BF030C2AF8153083B228BFA3
:1014700001351F2B7FF6D1AE2F2B3FF4CEAE5C2B68
:101480003FF4CBAE7F2B3FF6BEAE1149184611F8A4
:10149000012F002A3FF4B7AE9042F8D10620AFE604
:1014A0000520ADE6A0F1410189B2192901D847F024
:1014B0000207A0F1610189B219299EBF203847F0C7
:1014C000010780B2A1E700BFC02B0708C22C0708A4
:1014D000B92C070800214171FEF742BF2DE9F04702
:1014E00005468CB091461F460C46002900F0BF808F
:1014F00003F03F063146FEF733FF002840F0AF808F
:101500000DF13008494648F8305D4046FFF752FE7D
:10151000024620B99DF92B30002BB8BF062217F0E8
:101520001C0F49D0002A3ED0042A39D14046FFF78B
:1015300033FC0246A0BB46F00806310746D5DDF86D
:101540001CA0A946514619F8050FFEF779FE07467B
:101550004CF024FE01460AF10E00FEF71DFE079B2B
:101560002022DA72079900224846FEF777FE079B91
:1015700000221A775A779A77DA770123EB712FB323
:1015800039464046D5F83890FFF7C2F9024638B9D7
:1015900049462846FEF790FE013F6F610246A8B11A
:1015A0000023236032E09DF8063013F0110F5AD16A
:1015B0007807C2D50822F3E7002AF1D19DF806305A
:1015C000DA064ED4BF0701D5D8074CD4AB6B079FC2
:1015D0002362676268793107394648BF46F04006A2
:1015E000FEF72EFE0146A06007F11C00FEF7CCFDC1
:1015F0006B89A380B2064FF000030746E0602560C8
:1016000026746374E361636104D4002210460CB055
:10161000BDE8F0870028F8D0EE8960617602BE420E
:101620000FD30022A161002ABAD1C7F30803002B0F
:10163000EBD02846FEF7B8FDB8B100EB5720E061CB
:10164000E4E72068FFF754F801280146A7EB0607F6
:1016500003D9431CE3D10122E4E70222E2E7024678
:101660009EE704229CE707229AE7022298E70922D4
:10167000CCE72DE9F04F994685B000238846C9F89C
:10168000003003A904461546FEF7A8FD0646E0B95A
:10169000667CD6B9237CDA0779D5E3686769DF1BF6
:1016A000AF4228BF2F4687B16269C2F30803002BFF
:1016B00054D1039BDB89013B13EA522A13D142B96F
:1016C000A06801280AD802266674304605B0BDE835
:1016D000F08FA1692068FFF70BF8F2E7431C01D1F6
:1016E0000126F1E7A061DDF80CB0A1695846FEF7CC
:1016F0005BFD0028E7D00AEB00037D0A01932BD0A5
:10170000BBF80E20DBF800000AEB0501914288BF10
:10171000A2EB0A052B46019A414601F049F8002840
:10172000DED10399CB795BB1886B019BC01AA842CB
:1017300006D24FF400723C3108EB40203EF0B2FA82
:101740006D02D9F800302B44C9F8003063697F1B63
:10175000A8441D446561A6E7019BE3616569E169F1
:101760000398C5F30805C5F50075BD4228BF3D4681
:10177000FEF7A2FD0028B3D1039963693C31C3F39E
:1017800008032A46194440463EF08CFAD9E707265A
:101790009BE72DE9F04F9B4685B000238946CBF8A7
:1017A000003003A904461746FEF718FD064610BB95
:1017B000667C06BB237C9A0740F1A7806369FB42E5
:1017C00000D3DF439FB16369C3F30802002A7FD1CE
:1017D000039AD289013A12EA532201921ED173B9B7
:1017E000A06870B901462046FFF71EF848B9237C6F
:1017F00043F040032374304605B0BDE8F08FA16983
:10180000F1E7012802D102266674F4E7431C01D1F6
:101810000126F9E7A368A06103B9A0600398E36912
:10182000826B9A4203D1FEF725FD0028F0D1DDF846
:101830000CA0A1695046FEF7B7FC0028E3D0019B3D
:101840007D0A03EB000835D0019ABAF80E30DAF8B9
:1018500000002A449A4284BF019A9D1A2B464246B0
:10186000494600F0B4FF0028D2D1DDF80CA0DAF828
:101870003810A1EB0801A9420BD201904FF400727D
:1018800009EB41210AF13C003EF00CFA019B8AF879
:1018900007306D02DBF800302B44CBF80030636971
:1018A0007F1BA9441D44E3686561AB422CBFE36024
:1018B000E56087E76269E3689A4207D35046FEF71E
:1018C000D9FC0028A4D1039BC3F83880C4F81C803D
:1018D0006569E1690398C5F30805C5F50075BD4262
:1018E00028BF3D46FEF7E8FC002891D103986369C4
:1018F0003C30C3F308032A46184449463EF0D2F967
:10190000039B4FF00102DA71C4E7072673E7F7B5CE
:1019100001A90446FEF762FC054660BB237C5B061A
:1019200029D54CF03BFC216A07460198FEF7C4FC20
:10193000054600BB666AF37A43F02003F372206821
:10194000A26831460530FEF789FCE16806F11C000B
:10195000FEF722FC394606F11600FEF71DFC019841
:10196000B5740123F574C371FFF734FB237C23F0B6
:10197000400305462374284603B0F0BD13B5044662
:10198000FFF7C5FF28B901A92046FEF727FC00B9DB
:10199000206002B010BD70B50E468CB00021054627
:1019A000FEF7DEFC044668B90CA8314640F8305D0D
:1019B000FFF700FC044690B99DF92B30002B04DAA8
:1019C000029BEB6120460CB070BD9DF80630DB0633
:1019D00009D507996879FEF733FCE861F2E7042836
:1019E00008BF0524EEE70524ECE72DE9F0470E4695
:1019F0000021D2B0317080469146FEF7B1FC074617
:101A0000D0B9D8F81C30CDF8008002934D46DDF8EF
:101A100008A0BAF1000F15D14D4502D1013D2F2389
:101A200073557119334611F8012B03F8012B9A1BDA
:101A30002A449145F7D81E4600233846337052B0E9
:101A4000BDE8F08720216846FEF7ACFE00284BD1A8
:101A500006994046FEF730FC0446002842D107991B
:101A600098F80500FEF7ECFB214602906846FEF769
:101A700099FE002838D100216846FFF721F8044676
:101A800068B9079998F80500FEF7DAFB50450BD0C6
:101A900021466846FEF79CFF04460028EBD0042C44
:101AA00014BF27460227C7E70CA96846FFF7DDFAEF
:101AB0000CAA2244631C927D62B99D4216D32A1B54
:101AC0002346324443B96B1E1B1B2F22E44325449B
:101AD000F2549CE71C46EBE7013B0CA91944897DB5
:101AE000D154EFE70746A7E70746A5E71127A3E785
:101AF000F7B50D4601A90446FEF770FB064600281F
:101B00003FD1667C002E3CD1E368AB4204D2227CFC
:101B100012F0020F08BF1D460022636962610DB911
:101B200028461CE0019AD7897F0203B3013B6A1E55
:101B3000B3FBF7F1B2FBF7F28A4218D37A421340B3
:101B4000A1696361ED1A002940D10020E36865694D
:101B50009D4281BF237CE56043F040032374C5F3BD
:101B6000080575B1E36983420BD0E06109E0A16823
:101B700079B92046FEF758FE0128014604D1022615
:101B80006674304603B0F0BD013001D10126F7E79D
:101B9000A160A161D7E73B446361237C9A07A5EB71
:101BA000070506D52046FEF73FFE014628B9054643
:101BB0000FE02068FEF79CFD01464B1CE6D0012992
:101BC000DDD9019B1B6A8B42D9D9A161BD426369F2
:101BD000E1D863692B446361C5F30803002BB4D0DB
:101BE0000198FEF7E1FA0028C9D000EB5520ADE7D7
:101BF00070B5054616460C4621B30021FEF7B0FB32
:101C000068B9256031462046FFF7D4FAE0B994F967
:101C10002B30002B0BDBA379DB0603D4052000233C
:101C200023600EE06879E169FEF70AFBA0606B892A
:101C3000A38000212046FEF7B5FD0428EED0002841
:101C4000EDD170BD0920FCE70428E7D0E7E713B524
:101C500001A90446FEF7C2FA00B9206002B010BD27
:101C600073B50D4601A90446FEF7B8FA20B901463E
:101C700020461DB9FEF796FD02B070BDFEF720FFAD
:101C800010F0FB06F8D129462046FFF7EEF9314661
:101C90002046FEF79DFE042808BF0020ECE770B543
:101CA0000E468CB0002104461546FEF759FB009401
:101CB000044670B931466846FFF77CFA044640B9DD
:101CC0009DF92B30002B07DB1DB129466846FFF735
:101CD000CCF920460CB070BD0624FAE72DE9F84F88
:101CE000884600210446FEF73BFB074640B9D4F87E
:101CF00020A0A369AAF10202934204D8C8F80030D8
:101D00003846BDE8F88F6379012B17D102260546C6
:101D100031462046FEF7ECFC431C37D0012837D073
:101D200000B90135236A0136B342F1D8C8F8005032
:101D3000237AA56143F001032372E1E7E16A0646D5
:101D4000054604F13C0936B9204601F1010BFEF7C6
:101D5000B3FAF8B959466379022B09EB06000DD1A5
:101D600019F80630427853EA022308BF01350236DB
:101D7000BAF1010AC6F30806E5D1D7E7FEF704FA7F
:101D800030F0704308BF01350436F1E70127CDE795
:101D90000227CBE70746C9E72DE9F0410F4698B087
:101DA00002210646FEF7DCFA0446A0B918AD394612
:101DB00045F8606D2846FFF7FDF9044658B99DF8CF
:101DC0002B309A063ED41B063CD49DF8068018F0B2
:101DD000010F04D00724204618B0BDE8F081079910
:101DE0007079FEF72DFA18F0100F07460BD1284630
:101DF000FEF700FF04460028EDD1D7B93046FFF7C3
:101E0000E9F80446E7E7F3698342E3D00E90214600
:101E10000CA80C96FEF7C6FC04460028DBD1014650
:101E20000CA8FEF74DFE04460028D3D00428D2D1DA
:101E3000DDE7024639462846FEF76AFD04460028DB
:101E4000DCD0C8E70624C6E72DE9F04F0E4691B076
:101E500002210546FEF784FA0446002871D10DF1EF
:101E60004008314648F8305D4046FFF7A3F9044684
:101E7000002874D0042864D19DF83B1011F0200193
:101E80006FD110AF47F8405D3846FEF7CDFC0646EF
:101E900000285AD001285AD0431C5C425C414CF0C7
:101EA0007DF98246002C54D131462846FEF767FD65
:101EB000044600284DD14FF02033EB632B64C5F866
:101EC00043302E2385F83C30102385F847305146A7
:101ED00005F1520005F13C0405F10509FEF75CF936
:101EE000324621464846FEF7B9F905F15C031A4629
:101EF00051F8040B42F8040B9942F9D12E2385F8CE
:101F00005D30069A48464FF0010BFEF7A7F985F8B9
:101F100007B04046FEF740FF0446D0B90B98514643
:101F20001630FEF739F932460B994846FEF796F916
:101F30000B9B1022DA72284685F807B0FFF74AF8A3
:101F40000446204611B0BDE8F08F0724A7E702241D
:101F5000A5E7002231463846FEF7DAFCF1E708240F
:101F6000EFE70624EDE72DE9F0410C46A0B0022191
:101F700006469046FEF7F4F9002879D120AF2146B5
:101F800047F8606D3846FFF715F9002870D19DF8C5
:101F90004B3013F0A00F6ED10F9B6C4603F1200560
:101FA00018685968224603C20833AB421446F7D179
:101FB0003D460FCD14AC0FC40FCD0FC495E80F00F4
:101FC00084E80F00414614A8FFF7F4F848B9169AC0
:101FD0000A9B9A4203D1189A0C9B9A4203D008207C
:101FE00046E0042844D114A8FEF7D6FE00283FD1CD
:101FF0001B990DF10D0301F10D020DF11D0053F8B8
:10200000044B42F8044B8342F9D1188810809B7826
:1020100093709DF80B30DA0658BF43F0200301247B
:10202000CB72F471CB7ADB061BD50A9A169B9A42C7
:1020300017D07079FEF704F901463046FEF7B4F880
:102040000146D0B13046FEF737F988B996F85D30D1
:102050002E2B06D1169A06F15C01701DFEF7FEF8D4
:10206000F4713846FEF7C6FD10B93046FEF7B2FFF0
:1020700020B0BDE8F0810620FAE70220F8E7000072
:10208000F0B595B0074601910221FEF769F90546C2
:10209000002833D102AE4FF0203302930446736020
:1020A000C6F80730019B1B781F2B20D89DF80830FD
:1020B000E52B22D01CB1631EF25C202A30D0002117
:1020C00008A808970A91FEF76DFB0546B0B90121F3
:1020D00008A8FEF7F5FC70BB0F9A1CB3334603CB80
:1020E0001060516019889B78937211811CE001A8DF
:1020F000FEF796F8B0F5803F03D30625284615B0C5
:10210000F0BD55F0A5FE40F2B51155F06DFE00286A
:10211000F3D01D4A12F8013F83B39842FAD1ECE79D
:102120001C46C7E7E52313700123FB713846FEF711
:1021300051FF0546E2E70428FBD1002CDED0012147
:1021400008A8FEF79AFC05460028D7D120220146B0
:102150000F983DF0EBFD0F9B0822DA720F9ABDE756
:10216000092CCAD814AB2344020A03F8482C0134C2
:1021700014AB2344013403F8480C93E7FF28EFD84D
:102180000A2CF5D9B9E700BF4C2C07082DE9F04F10
:1021900006688BB01C4600234371039103790293B8
:1021A000154605210DF11F02304600F025FB9DF874
:1021B0001F30DF0700F18882580700F1878208AAE4
:1021C0000321304600F018FB30B9089A531EB3F5CE
:1021D000004F01D21A4201D00123089345B15D4B53
:1021E000A5F500729A4203D913200BB0BDE8F08F19
:1021F0006A1E2A40F8D1149B5B0A0593002C00F05C
:102200006782002B00F06482029B002B63D00123C5
:102210002146304600F0CCFA08B10120E5E794F8F9
:10222000FF2194F8FE3143EA02234AF655229342F5
:1022300001D00E20D9E7029B04EB031101F5D77101
:102240000B79002BF5D001F10800FDF79DFF8146C9
:1022500001F10C00FDF798FF0990DDF824A0BAF118
:10226000150FE6D96B0A802BBED8039A12F0020E26
:1022700008D002F00701022900F038821146C90790
:1022800040F134820399CA07AED5002B53D13248AE
:102290004FEA1A354FF0010830F8021F09B1A94280
:1022A00031D940F6F571BAFBF8F58D429BBF05EBCD
:1022B0004505013502356D088CBF6D00033505F20B
:1022C000FF154FF020018CBF022701276D0A4FF048
:1022D000010B01912CE209AA0121304600F08CFA91
:1022E00000289AD1039B13F0080F099B0CBF4FF0F5
:1022F0003F094FF000094B459BD3A3EB090309931A
:10230000ABE75B00F8E14FEA4808C5E7022F25D1AB
:10231000049A4FF6F5718A420FD9002B40F0E28102
:102320004FEA4803402BB0D9BEF1000F40F0E081E6
:10233000802B3FF67EAF9846B3E7049A40F6F571DE
:102340008A4212D8002B7FF474AF4FEA4803802BE7
:102350009BD96EE700FEFF00682C0708049A40F640
:10236000F5739A423FF665AF01274FF400720021E2
:1023700020463DF0DBFCD74B84F80EB01A68226093
:102380005A6862601A899B7A2281032F4FF00202F9
:10239000A3724FF00003E3722273CBF3072B4FF0CD
:1023A0000102637418BF0223BAF5803F84F80D80E0
:1023B00084F80FB02274A37480F01D8184F813A0F8
:1023C000CAF3072A84F814A0F82363753F23237601
:1023D0004FF0000AFF2384F819A0A37684F81BA00D
:1023E000494604F11C00FDF7D7FE032F40F0098198
:1023F0004BF0D4FE014604F14300FDF7CDFE294623
:1024000004F12400FDF7C8FE022384F82C300123D8
:1024100084F83030062384F83230802384F840304A
:10242000292384F84230AC4B84F82DA084F82EA0E8
:1024300084F82FA084F831A084F833A004F1470277
:1024400003F1100153F8040B42F8040B8B42F9D14D
:1024500019889B7893704FF0550B6FF055031180DE
:10246000304684F8FF3184F8FEB101234A46214604
:1024700000F0ADF9824600287FF4CFAE032F3FD1A4
:10248000012309F106022146304600F0A0F94FF47D
:102490000072514620463DF049FC52232370637080
:1024A0006123A37084F8E731049B41227221E2701A
:1024B00084F8E41184F8E51184F8E621591E04F546
:1024C000F470FDF769FE022384F8EC316FF05503D8
:1024D00084F8FF3109F107020123214684F8EDA1B8
:1024E00084F8EEA184F8EFA184F8FEB1304600F044
:1024F0006EF9012309EB03022146304600F067F92B
:10250000149B23F4FF7222F00102002120463DF0CB
:102510000DFC032F40F09280F8232370FF2363709B
:10252000A370E37023716371A371E371237263720B
:10253000A3720F23E372059B009AAB4228BF2B4680
:10254000214630469A4600F042F9014600287FF4C1
:1025500064AE4FF4007220463DF0E8FB009BB5EB03
:102560000A0553440093E6D1019B032F08BF43465D
:102570000193019B059A934228BF13462146009A76
:1025800030461D4600F023F900287FF446AE009B3C
:102590002B440093019B5B1B0193EAD1032F56D080
:1025A000099BB3F5803F54D2022F14BF01250425A7
:1025B000029B002B4FD0002201232146304600F021
:1025C000F7F8024600287FF428AE029B04EB0313C1
:1025D00083F8B25101232146304600F0F8F8002874
:1025E0007FF41BAE00221146304600F005F90030A2
:1025F00018BF0120F9E5514604F12000FDF7CCFD9C
:10260000E2E64BF0CBFD014604F12700FDF7C4FDE7
:10261000C5F30723E375802384F82430292384F845
:1026200026302E4BA57504F12B0203F1100153F84F
:10263000040B42F8040B8B42F9D109E7012F28491A
:10264000204618BF6FF00701FDF7A6FD73E70C25C4
:10265000AEE70625ACE7039B1B07C3D44FF400721B
:10266000029920463DF062FB552384F8FE31099A19
:1026700084F8C251AA2384F8FF319DF8083084F809
:10268000BE3184F8C1314A4443F6C163B2FBF3F270
:10269000FE2384F8C331930843F03F03012784F8F5
:1026A000C43184F8C521494604F5E37084F8BF714C
:1026B00084F8C071FDF770FD099904F5E570FDF728
:1026C0006BFD3B46029A86E703208EE50A208CE5E7
:1026D00011208AE5862C0708922C0708A62C0708EB
:1026E000F8FFFF00BEF1000F3FF4A3AD002B59D15E
:1026F0002D484FEA5A45012330F8021F19B1A9426B
:102700007FF6FFAD0021BAFBF3F0284F8500A0F55E
:102710007F40F63805F20725B8424FEA55253FF6C7
:1027200088AD98460B46002101914FF0200B0327FE
:1027300009EB0B0100910199DDF820C068180099A0
:1027400008440CF1FF31032F0144CCF1000C08BF09
:10275000009A01EA0C01A1EB000101BF52188B4461
:102760001146009118BF6D18C9EB08110844824545
:10277000FFF45FAD019AAAEB0B01491B032FA1EBFC
:102780000201B1FBF8F204927FF4C0AD4FF6F5718F
:102790008A423FF6EAAD002B7FF44BAD5FEA580367
:1027A0003FF447AD1946AEE7762C0708FFFFFE0F52
:1027B00010B50C4611461A4638B1234604303CF099
:1027C000D3F8003018BF012010BD0420FCE710B57D
:1027D0000C4611461A4650B1234604303CF006F927
:1027E00010F11E0F05D0003018BF012010BD0420CD
:1027F000FCE70220FAE7000070B50D4614460646D5
:10280000002833D001F00703234AD15C00292FD0E0
:10281000002204303CF038F9062D27D8DFE805F017
:1028200008050A162619190006202AF017FE20604E
:10283000002070BD062805D14FF400732380238843
:10284000B360F5E72AF00AFE2080F8E70123236051
:10285000EEE7062801D0430806D1336A002B0CBFEF
:10286000042300232370E3E70123FBE70420E0E7D0
:10287000062DFBD801A353F825F000BF312800082E
:1028800029280008392800084D2800086D2800086C
:102890005B2800085B280008806D0608086833F094
:1028A00024B9000037B51D46043001AB1446FEF7CD
:1028B00070FF38B1064B1B5C2B604FF0FF34204695
:1028C00003B030BD019BA342F9D01C23F4E700BF45
:1028D000C06D060813B51C46043001ABFEF7C9FEF7
:1028E00030B1044B1B5C23604FF0FF3002B010BDD1
:1028F0000198FBE7C06D06082DE9F8438146506852
:1029000090460F4630F0A8FC254A0138002410F804
:10291000013FD3B92C201DF0CDFB0646054646F8F5
:10292000047BD8F8000030F097FCE3B20246314651
:1029300009F14400FEF7D2FD074640B328461DF0DA
:10294000D3FB184BD85D29F071FF722B13D008D838
:10295000612B19D0622B0CD02B2BD8D144F003045F
:10296000D5E7772B0AD0782B0BD0742B08BF1746EE
:10297000CDE70D4FCBE744F00104C8E744F00A046B
:10298000C5E744F00604C2E744F01204BFE7E306DB
:1029900003D529693046FFF7ABF82846BDE8F88330
:1029A000106E0608C06D0608D46D060830B587B0F5
:1029B000054603AC084611461A46064B009301949F
:1029C00003232AF039FA224629460020FFF794FF14
:1029D00007B030BDA86D06081FB50623CDE901126A
:1029E00001AA03490393FFF787FF05B05DF804FBD5
:1029F000106E060870B5054608460C462AF0A4FC81
:102A00002346024602492846BDE8704000F094BFC4
:102A10009C6D0608022970B5044615461E4613D162
:102A20005368012B0AD0022B0CD01BB91168201D52
:102A3000FFF75EF8A3692B60002070BD81692B68E9
:102A40001944F4E70169FAE701290AD10430FEF7D5
:102A50005EFF0028F0D0084B1B5C33604FF0FF3066
:102A6000EBE7042906D14368002BE5D00430FEF7DC
:102A700085FFEEE71623F0E7C06D06082DE9F74F56
:102A800006299DF8305010D8012905D93F2303703D
:102A900001300023037001E00029FAD1012994BF1D
:102AA0000020012003B0BDE8F08F10EE104A002C8A
:102AB00025DAB4EE400AF1EE10FA20D62D25441C9A
:102AC0000570B1EE400A9FEDC47A0190F0EEC07A35
:102AD000F4EE477A02F0200EF1EE10FA5FFA8EF56E
:102AE00013DD85F04903237085F04E0385F046051C
:102AF0006370E11CA57000230B70081AD2E715B1B2
:102B0000441C0570DFE70446DDE7B4EE400AF1EE51
:102B100010FA08D745F04E0385F041052370657023
:102B2000E11CA370E7E7002B42F02002B8BF0623A8
:102B3000672A02D1002B08BF0123251A0139491B3E
:102B400010EE105A002D4BD1662A3BD15D1C8D42F0
:102B5000A8BF8B1E002766215D1C0091BC463E4627
:102B600023EAE3730099652940F02C815D1C4FF046
:102B700000084FF02E0AB2EE047A454540F38380F8
:102B8000FDEEC07A04F1010917EE901A0029ABBFDF
:102B900017EE901A302101F1300B2170A8BF84F894
:102BA00000B0E04504D11BB104F1020984F801A092
:102BB000F8EEE77A08F1010830EE670A4C4620EE9D
:102BC000070ADAE75D1D8D42A8BF8B1F652A0092B8
:102BD0004FF0000500F0EC802F46AC462E46BFE7D4
:102BE000B5F17E5F80F08F80DFED7C7ADFF8F4C195
:102BF000DFF8F491B4EEE70AF1EE10FA4FF00005B9
:102C0000ACBF4FF031084FF0300820272E46BCEC07
:102C1000017AB4EEC07AF1EE10FAC4BF09EB050AEE
:102C20009AED007A05F10405C4BFF61920EE070AF3
:102C3000182D4FEA6707EAD110EE105AB5F17E5F02
:102C400045D2B4EEE70AF1EE10FA3BDB002E0CBFE2
:102C50002B272D27B7EE000A662A03D0672A48D112
:102C6000042E46DC672A04BF06F1FF355B195D1CA4
:102C70008D42A8BF8B1E84F8008053BB66210134AF
:102C80001D461F460091662A40F0B080AE4240F3D8
:102C9000098197B10A2196FBF1F393FBF1F201FB55
:102CA000136601FB12324EF0450E3032303684F896
:102CB00000E06770A270E670043400232370019B6B
:102CC000E01AEFE6F2EE047A20EE270A01362D270D
:102CD000C2E72E2161701D4602343021013E69D0C9
:102CE0001DB92F464FF0FF3C45E004F8011B013DA4
:102CF000F4E74D1F9D4261DC672A5DD08B1F009277
:102D00000025AC462CE70025DFF8DCC0DFF8D480D6
:102D100020272E46FCEC017AF4EEC07AF1EE10FA90
:102D20009CBF08EB0509D9ED007A05F104059CBFAD
:102D3000F61920EE270A182D4FEA6707EAD1FDEEB3
:102D4000C07A17EE905A092DC2BFDFED257A013601
:102D500020EE270A662A11D18E4212DA9D1901351A
:102D60008D4204DB8B1B023B591C08BF0023F51866
:102D70000135B446002766210091F1E6652A40F04E
:102D80008C804D1F9D4200DC8B1F00252B27AC46FD
:102D90006521F1E71D1D8D4200DB4B1F9E4204DBC8
:102DA0006721009100252B27ABE7711C5B1ADEE73A
:102DB0002B2712E7374695E72B46A0E70025009220
:102DC000AC46CFE6009967297FF4D1AE0BB11D4622
:102DD000CDE601252B46CAE6FFFF7F7FF8FF7F3F48
:102DE000CDCCCC3D1018060828180608F1EE047A60
:102DF000B4EEE70AF1EE10FA26DB651E4FF030095B
:102E0000A84618F801C9BCF12E0F3BD0ACF1300A2E
:102E1000BAF1090F29D9681C0578302D14D190F822
:102E200001C0BCF12E0F31D1009966292ED02D2F73
:102E300080F800C0457027D1013E08BF2B272146EE
:102E4000884225D331210170672A7FF422AF002BFD
:102E50003FF41FAF23461C46013B14F8012C302AD7
:102E6000F9D02E2A08BF1C4613E7BCF1390F05D054
:102E70000CF1010C85F800C02846CDE7A84288F87F
:102E80000190C9D04546BBE70136D8E70134D6E703
:102E900011F8015C01F80159D2E7672A3FF47AAFD3
:102EA00000927FE7F1EE047AB4EEE70AF1EE10FA51
:102EB000A3DAEEE608B5044631B1054B03608A6B30
:102EC000096800232CF0FAFA20461DF0C1F800BF73
:102ED0007C2806082DE9FF471F460192461812B1CB
:102EE000023A222A34D80546B5422C4639D22078F7
:102EF0001EF038FA013580460028F5D123782B2BB7
:102F000029D12C46311B204601AA27F0C0FF2518E5
:102F1000A9460024B1454B4626D3B8F1000F00D096
:102F20006442640044F00104AB4209D01D46B5423E
:102F30002B4642D2187801351EF014FA0028F6D13B
:102F40002049019A20482CF07DFA3946FFF7B2FF5C
:102F50001E4829F085FA2D2B04BF2C464FF001089E
:102F6000D0E74FF00008CDE719F8012BA2F1300AA5
:102F7000BAF1090F09D95F2ACCD042F02002A2F1A0
:102F800061011929C9D8A2F1570A01995145C4D93B
:102F9000204636F07FFC28B9019B03FB04A494EA89
:102FA0004403B7D504A8019B40F8045D4246711B59
:102FB0002DF040FC039B0446B6E7C1D1204604B087
:102FC000BDE8F0875B1806086C2906084618060855
:102FD0002DE9F04F2DED028B83B0914600930E9BAF
:102FE000019346180446B442254680F0288128788B
:102FF0001EF0B8F9013482460028F4D12B782B2B2F
:1030000009D125468346B4420CD30023DFED938AD1
:103010009A46194681E02D2B03D125464FF0010B2E
:10302000F1E783462B7843F02003692B32D1AB1CA8
:103030009E4240F207816B7843F020036E2B40F0F4
:103040000181AB7843F02003662B40F0FB80EB1D41
:103050009E4205F103041AD9EB7843F02003692B53
:1030600015D12B7943F020036E2B10D16B7943F0EF
:103070002003692B0BD1AB7943F02003742B06D1CD
:10308000EB7943F02003792B01D105F108049FED82
:10309000748A14E06E2B58D1AB1C9E4240F2D28051
:1030A0006B7843F02003612B40F0CC80AB7843F089
:1030B00020036E2B40F0C6809FED6A8AEC1CBBF1AA
:1030C000000F01D0B1EE488AA54209D0B442234690
:1030D00080F09580187801341EF044F90028F5D16D
:1030E000614962482CF022F90199FFF7E3FE0220C2
:1030F000274697F800C0ACF1300EBEF1090F07F17A
:10310000010444D802282ED1594FB94201DC08FBF2
:1031100001E1B442ECD302B149420B4413F1250F53
:10312000BEBFDFED547A253368EEA78A13F1090F8D
:103130005AD35B4200EE903AB2EE040AF8EEE00A8F
:103140003DF0C0FD88EE808AB9E700222F46134685
:1031500011461046DFED418A9FED477AF2EE046A90
:103160004FF00A08C5E7F4EEC78AF1EE10FA0BD566
:1031700007EE90EAF8EEE77A0128E8EEA67AF0EE9C
:10318000678A2DD1013BC4E728B90133C1E720B9D3
:10319000BCF12E0F03D10120BBE7022813D04CF065
:1031A000200EBEF1650F0ED1A64253D978782B2898
:1031B00004D1BC1CB44293D00220AAE72D2896D19A
:1031C000BC1C0122F6E7B9F1000F04D04CF0200E30
:1031D000BEF16A0F06D0BCF15F0F9AD03C469AE769
:1031E000002096E7CA4696E707EE903AB2EE040A48
:1031F000F8EEE70A3DF066FD28EE808A5FE77FF48F
:103200006FAFBAF1000F0AD09FED140AF0EE480A32
:1032100003B0BDEC028BBDE8F04F2BF02FB9009B43
:1032200023B1DFED0E0AB0EE480AF1E7B0EE480A2E
:1032300003B0BDEC028BBDE8F04F2CF05BBA4FF051
:10324000000BE2E6BBF1000F3FF44AAF2C469FEDC6
:10325000038A37E73FF444AF5DE700BF000000009A
:103260000000807F0000C07F401806086C29060817
:1032700064666606EA1C0802EC78AD6008461146F2
:1032800042F0E0B970B5054608460E463CF084FDB4
:10329000044620B102466B682868314698472046AC
:1032A00070BD00002DE9F74F01919DF83010914657
:1032B0000D9A11F0DF0F0646A2EB09023DD030292E
:1032C0000CA9244F0EBF4FF010080F464FF0010815
:1032D00013F0800435D0022492FBF4F4151B002C6B
:1032E00036DDA246D045C346A8BFD34673683068D2
:1032F0005A463946AAEB0B0A9847BAF1000FF1DC9F
:10330000B9F1000F05D07368019930684A469847B3
:103310004C44002D0DDD2C44A845C146A8BFA9464C
:10332000736830684A463946A5EB09059847002D71
:10333000F2DC204603B0BDE8F08F074F4FF01008D5
:10334000C6E713F0010501D11446C8E71546D7E7D3
:103350000024D5E70C090608FB0806082DE9F04310
:1033600089B007460020119D9DF84880139E8DF876
:103370000F0002B3814219DA2D228DF80F20494245
:10338000109A08ACA2F10A0C0DF1100EB1FBF3F08B
:1033900003FB1012092A8CBF6244303204F8012D5D
:1033A000744501460DD00028F0D10AE0A80726D5C3
:1033B0002B228DF80F200029E2D108AC302304F82D
:1033C000013D15F040099DF80F301CD023B30122B8
:1033D000CDE900822B460DF10F013846FFF762FF61
:1033E000013E814608AACDE900862B46121B2146E4
:1033F0003846FFF757FF484409B0BDE8F0836A0735
:10340000D9D52022D5E7002BECD004AA9442E9D9E3
:1034100004F8013C013CE5E79946E3E72DE9F04F6C
:1034200091B082461C46C8079DF86C301A9D0593E2
:103430000F469146DDE91C860BD4B90703D13A68E3
:10344000804B9A4205D038462AF008F8400040F0F8
:10345000010715F0810306D1059A302A03D1B04542
:10346000B8BFB0461E4638462DF0F9F800280DF1D9
:10347000200B18DBAA0712D52B238DF820300DF175
:103480002103E1B2EC061DD5B9F1020F0DD11A46A8
:10349000302002F8020B481C5870134612E06B07EC
:1034A00001D52023E9E75B46EBE7B9F1080F3ED1F0
:1034B000A8054FF030021A7045BF01F10E025A7094
:1034C00001330233002215F0200F1A70A3EB0B0317
:1034D000049314BF2C231346012E0CA8C8BF45F03B
:1034E0004005099015F040044FF01000CDE90A02A4
:1034F0008DF81F20CDE9021323D0CDE900923B4681
:103500000BAA0AA909A82CF07BFF03782D2B814672
:1035100040F086800B9C8DF81F30013C012E00F19D
:1035200001090B9400F3898000273C4636E0B9F18D
:10353000100FC7D11A46302002F8020B01F1170014
:10354000AAE708ABCDE900930BAA3B460AA909A854
:103550002CF056FF012E81461FDD0B9CB442B8BFF4
:103560003446A04516DD15F00107A8EB040401D090
:103570002746002425F001054CB1202300930023A9
:1035800001941A4630495046FFF78CFE044630231A
:10359000059303E000273C46ECE7274669061DD566
:1035A0009DF81F305BB100230122CDE900320DF1FF
:1035B0001F015046FFF776FE08F1FF380444049BD4
:1035C00063B100230122CDE900325946049A5046E6
:1035D000FFF768FE049B0444A8EB0308059B0093D7
:1035E000012ED8BF464601962B460B9A49465046B7
:1035F000FFF758FE04444FB12023009300230197A6
:103600001A4611495046FFF74DFE044409980CAB89
:10361000984201D01CF068FD204611B0BDE8F08F43
:10362000012E81DD0B9C9DF81F30B442B8BF34469B
:1036300003B10134049B1C4493E7B442B8BF344641
:10364000F7E700BFC02E060893C706082DE9F04330
:1036500016468BB0B20780469946129F3CD416F0AE
:10366000040F0CBF0023202300930A46139B202144
:1036700002A8FFF703FAF30504460DD5431C1F2BE0
:103680000AD80AAA1444252204F8202C0AAA1A44AB
:10369000002102F8201C1C4616F040051ED09DF8A3
:1036A00008302F2B4FF000031AD8012202A9CDE9D0
:1036B00000324046FFF7F6FD013F0546013C0DF1A3
:1036C0000901CDE90097334622464046FFF7EAFD5F
:1036D00028440BB0BDE8F0832B23C5E702A9F0E72F
:1036E00002A91D46EDE700002DE9F04F824689B0A2
:1036F000144600250E46334613F8012B8AB9B14211
:1037000013D30B78002B00F00E81013120234FF0F2
:1037100000090A780E46481C8AB990464FF0FF32DD
:103720004FE0252AEBD01E46E5E7771ADAF8043099
:10373000DAF800003A4698473D443146E1E72D2A41
:1037400003D149F001090146E3E72B2A02D149F0F0
:103750000209F8E7202A02D149F00409F3E7212AF7
:1037600002D149F00809EEE7302A22D149F0400998
:103770001346E8E70A2000FB0828A8F130080E46A7
:1037800011F8012BA2F130000928F3D92E2AC5D156
:1037900072782A2A10D008460022064610F8011B2B
:1037A000A1F13007092F0CD80A2606FB0212303A85
:1037B000F3E74FF00008E2E72268023622EAE272FD
:1037C000043431786C2908BF01363778002F00F0B7
:1037D000AA80642F00F0818028D8502F2DD00ED8D9
:1037E000A7F14501022940F28780DAF80430DAF8BF
:1037F00000000122314698470135A3464AE0622F76
:103800003BD04DD8582FF0D17A1C27F00F070F3F2F
:1038100002F00602FFB2CDE9023804F1040BCDF844
:1038200004900097C2F11003002260E0712F42D093
:103830000DD8672F60D9702FD7D1CDE90238612319
:10384000009304F1040BCDF804901023ECE7752FDE
:10385000DAD0782FD8D0732FC7D1511C04F1040BC4
:10386000246805D1204604933CF096FA049B024656
:10387000CDE9003821464B4608E0226804F1040BEC
:10388000CDE900384B4642B1294904225046FFF7A2
:1038900009FD0544711C5C462CE705222549F5E726
:1038A00008A9226801F8042D04F1040BCDE90038C1
:1038B00001224B46EAE707A92068CDE904321DF052
:1038C00028FB059A049B0146501CCDE9003804F101
:1038D000040B08BF079A4B46D8E7CDE902386123AD
:1038E000009304F1040BCDF804900A23012221680F
:1038F0005046FFF733FDCCE7073424F00704D4E942
:103900000001CDE9043257F045FD059A049BCDE94D
:10391000008200EE100A4A463946504604F1080B70
:10392000FFF794FEB5E7284609B0BDE8F08F00BF69
:10393000F0080608F50806080EB403B503AA52F805
:10394000041B0192FFF7D0FE02B05DF804EB03B058
:0439500070470000BC
:020000040802F0
:10000000024B1A6902601861002070472C1B002007
:10001000024B1A6912681A61704700BF2C1B00203E
:10002000C460056146618761C0F81C80C0F82090FB
:10003000C0F824A0C0F828B0C0F82CD080ED0C8BFC
:1000400080ED0E9B80ED10ABC0F808E0FFF7D8BF45
:10005000104A08B513690BB924F0C8F8196858603C
:1000600011611846C468056946698769D0F81C8023
:10007000D0F82090D0F824A0D0F828B0D0F82CD018
:1000800090ED0C8B90ED0E9B90ED10ABD0F808E04E
:10009000012070472C1B002010B50021044600F001
:1000A00075FA18B914B120460CF0C6F910BD00213C
:1000B00000F06CBA10B50121044600F067FA18B9D7
:1000C00014B120460CF0B8F910BDFFF7E5BF10B52C
:1000D00001220C4600F0A6FB18B914B120460CF022
:1000E000ABF910BD00F09EBB00F02ABB2DE9F04338
:1000F0002A4C00254FF00309D4F8F8710021013192
:1001000043189A0803F00303BA5C5B0042FA03F356
:1001100003F00303022BF2D0D4F8043209018A0859
:1001200003EB001081B300EB820103681A0728D1AA
:10013000D4F804229A4224D89A1AD4F808624FEAD2
:10014000921C120902F003079E424FEA470718D992
:10015000D4F8F8E11EF80C8048FA07F303F0030323
:10016000012B0ED109FA07F747EA080705F584784D
:100170003F2D0EF80C709ABF24F818200135C4F8F2
:100180000C3204308842D0D12DB1013D05F5847385
:1001900034F81300B0E7BDE8F08300BF2C1B00204B
:1001A00021F00F0370B5174A174D1C1AE400A2FB8B
:1001B0000424640A0219A3EB8416C5F80022002166
:1001C0002246C5F80832C5F8FC41C5F8F801C5F863
:1001D00004621FF0ABFDA2000732D2080021D5F85F
:1001E00000021FF0A3FD00234FF480314FF0FF32D7
:1001F000C5F89012C5F89822C5F89C32C5F894321B
:1002000070BD00BFF32C23FA2C1B0020034AB2F868
:1002100090320133A2F89032704700BF2C1B0020AF
:10022000034AB2F89032013BA2F89032704700BF07
:100230002C1B0020034BB3F89002003018BF0120A4
:10024000704700BF2C1B0020F8B51C4DB5F890324C
:1002500000220133A5F89032C5F89422C5F80C228B
:100260002C1D05F5EC76032754F8043F1A0719D125
:10027000D5F80402834215D3181AD5F808124FEAAC
:10028000901C000900F003028B424FEA420209D29F
:10029000D5F8F81111F80CE04EFA02F303F003035D
:1002A000012B02D0A642DFD1F8BD07FA02F242EAE2
:1002B0000E0201F80C20FFF719FFF3E72C1B0020BA
:1002C00031B3F8B5041F174E04EB8105032754F82A
:1002D000043F1A0719D1D6F80402984215D8181A03
:1002E000D6F808124FEA901C000900F00302994268
:1002F0004FEA420209D9D6F8F81111F80CE04EFA8B
:1003000002F303F00303012B03D0A542DFD1F8BDB4
:10031000704707FA02F242EA0E0201F80C20FFF7DA
:10032000E5FEF2E72C1B00202DE9F04F514ED6F8E8
:10033000FC11D6F80C3283B0890000256BB3C6F8E7
:100340000C52F9B10024A208D6F8F80104F0030316
:10035000825C5B0042FA03F303F00303032B05D036
:1003600001348C42EFD3D6F80C32E7E72046FFF792
:10037000BDFED6F8FC1101348900A142E3D8D6F8BD
:100380000C32DBE7B6F890320022013BA6F890323F
:10039000C6F89C2203B0BDE8F08F0029F2D09E463B
:1003A0001D464FF003084FF0020A06E0032B56D01B
:1003B000012B20D001358D42E4D2AF08D6F8F821C8
:1003C00005F00304D05D640040FA04F303F0030376
:1003D000022B02EB070CE9D1BEF1000FEAD008FABC
:1003E00004F420EA04008CF80000D6F8FC114FF069
:1003F000010E8900DEE74FEAD50BD6F8002212F88D
:100400000B1005F0070941FA09FE1EF0010F5A44CE
:10041000E5D02801D6F804C25CF80030604493B1FE
:100420006A46B1210BF022FA009A3AB10CF046FA72
:10043000DDE900010CF018FA0CF056FAD6F80022AB
:1004400012F80B105A44012303FA09F321EA0301BD
:100450001170D6F8F83103EB070CD85DBFE70AFA44
:1004600004F420EA0400D055D6F8FC114FF0000E39
:1004700089009FE72C1B0020054BB3F89022002138
:100480000132A3F89022C3F80C12FFF74DBF00BF52
:100490002C1B00203C4B2DE9F047D3F80412D3F875
:1004A0000822D3F8FC61D3F8F8710023C0E90133C6
:1004B000C0E90333C0E90533521A02601D46B60095
:1004C0009E469C461C461A4699461946984617F879
:1004D000093049000B4103F00303012B49D040D3FD
:1004E000022B02D1013545600134013296420ED013
:1004F0004FEA920902F0030117F809304FEA410A66
:1005000043FA0AF313F0030301D0012BDFD1012CCE
:1005100011D0022C02D14169013141618169A142AE
:1005200038BF846196420FD0012B26D04FEA920942
:1005300002F00301CBE70169013101618169A14248
:1005400038BF84619642EFD1C44503D99642C0F8C2
:100550000CC017D12D014FEA0E13C0E90153BDE8BD
:10056000F0870EF1010EC0F808E00CF1010C1C46FA
:10057000BBE7013545601C46B7E7E045E6D34FF0E1
:10058000000CD3E7E046FAE72C1B00200F302DE9E2
:10059000F04706095CD0694DB5F89032002B57D171
:1005A000B5F89232002B01F001040CBF4FF0010EA0
:1005B0004FF0000E51D1D5F89C12D5F8FC718F4246
:1005C00039D9D5F8F8C1481E604400231AE0013338
:1005D0009E4254D912F00C0F1ED101339E4240F2BC
:1005E000A48012F0300F1CD101339E4240F2A08053
:1005F00012F0C00F1AD101339E4240F29C800131AB
:10060000B94218D210F8012F12F0030FDFD012F008
:100610000C0F4FF00003E0D012F0300F4FF000034A
:10062000E2D012F0C00F4FF00003E4D00131B94224
:100630004FF00003E6D3BEF1000F09D12AF024FCED
:10064000D5F89C12D5F8FC718F424FF0010EB8D846
:100650004FF000084046BDE8F087D5F89422D5F861
:1006600098329A42A7D32AF00FFCD5F89C12D5F8FD
:10067000FC718F4288BF4FF0010EA2D8E8E78900D5
:10068000CA1A012B02F1010701F1010E08BF4FEA5E
:100690009E034FEA970008BFC5F89C3207F003039A
:1006A0004FEA43081CF80090012303FA08F30232D2
:1006B00043EA090391420CF8003012D34FF00208CC
:1006C0009008D5F8F8C102F003031CF800905B0015
:1006D00008FA03F3013243EA090391420CF80030AF
:1006E000EED2D5F804A2D5F894324FEA0719AEEB52
:1006F00007020AEB09081E44120140460021C5F812
:1007000094621FF013FB6CB10023D5F800124AF875
:100710000930FA080123885C07F0070703FA07F796
:1007200007438F544046BDE8F08789000131A7E7B1
:1007300089000231A4E789000331A1E72C1B0020C6
:10074000F0B41C4EB6F890328BBB80B3D6F80432AE
:10075000D6F80052C01AC10904096B5C04F00707FF
:100760000122BA4023EA02036B54D6F89C22830983
:100770009342D6F8F80138BFC6F89C32C15CA50890
:1007800004F0030303275B0007FA03F321EA0303E2
:1007900043550134D6F8F801A50804F00303415D80
:1007A0005A0041FA02F202F00302022AEBD0F0BC36
:1007B000704700BF2C1B002010F00F031BD11849FD
:1007C000D1F80422824216D810B4D1F808428442EB
:1007D00022D9801AD1F8F84181090209615C02F03E
:1007E00003004000014101F003010129184604D033
:1007F0005DF8044B704700207047013013189908CA
:1008000003F00303615C5B0041FA03F303F00303AD
:10081000022BF2D00001EBE718465DF8044B70475D
:100820002C1B00208C46002800F087802DE9F84F13
:10083000874CB4F89052002952D0002D51D1D4F8F1
:100840000412D4F8FC31A0EB01094FEA1917791C06
:100850004FEA830E0CF10F068E454FEA161640F252
:10086000F380D4F8F8A14FF001084FEA910B01F0A2
:1008700003031AF80BB05B004BFA03F303F0030316
:10088000022B32D023B9013508EB0503B3422ED336
:1008900046454ED02FD34544B5428246C0F08380B2
:1008A00007EB08023744974210D902219008D4F888
:1008B000F85102F0030315F800C05B0001FA03F3DE
:1008C000013243EA0C0397422B54EFD1A6EB080206
:1008D00012010AEB0810002155461FF027FA01E02B
:1008E0007DB300252846BDE8F88F08F101080131E5
:1008F0008E45BAD1CCE73E44354647444FF0030914
:100900004FEA950ED4F8F81105F0030311F80EC064
:100910005B0009FA03F301352CEA0303AF4201F847
:100920000E30EDD1D4F89C32B6089E4238BFC4F8E0
:100930009C6205462846BDE8F88F01466046FFF7F1
:1009400025BED4F80412D4F80062401AC109050982
:10095000735C05F007070122BA4023EA02037354CF
:10096000D4F89C32D4F8F8618009984238BFC4F8B2
:100970009C02315C05F00303A80803275B0007FA1B
:1009800003F321EA030333540135D4F8F861A808CE
:1009900005F00303315C5A0041FA02F202F003024F
:1009A000022AEBD09DE74FEAD919D4F8003213F8A8
:1009B000091007F007073941002A92D001F0010120
:1009C0006046FFF7E3FD054600288AD04FEA08128B
:1009D00051461FF067F9B4F89032002B82D1D4F859
:1009E0000402D4F80072AAEB0000C10906097B5C7E
:1009F00006F0070C012202FA0CF223EA02037B54F0
:100A0000D4F89C32D4F8F8718009984238BFC4F801
:100A10009C02395C06F00303B0084FF0030C5B0046
:100A20000CFA03F321EA03033B540136D4F8F871BE
:100A3000B00806F00303395C5A0041FA02F202F0F2
:100A40000302022AEBD04DE74FF0010820E700BF78
:100A50002C1B00202DE9F04F404BD3F80802D3F8AF
:100A60000422D3F8FC11D3F8F83185B00025821A9E
:100A700003924FEA810EA8462F460295AA46AB463E
:100A80002E46A9462C46AC462A4613F80C105200B6
:100A9000114101F0030101294DD046D3022902D1B1
:100AA0000BF1010B0136013474450CD04FEA940C64
:100AB00004F0030213F80C105000014111F003017F
:100AC00001D00129E1D1012E0FD0022E08BF08F17B
:100AD0000108B54238BF354674450DD001292ED0E6
:100AE0004FEA940C04F00302CFE7B54238BF354615
:100AF000744507F10107F1D14FEA0A130093029BF5
:100B0000039A17491748994538BF99464FEA0B137E
:100B1000E2F712FFCDE9005943463A46124911481F
:100B2000E2F70AFF05B0BDE8F08F0AF1010A09F10A
:100B300001090E46B7E70BF1010B0E46B3E7029A27
:100B40004A4528BF4FF00009CAD2CDF808904FEAB5
:100B5000940C4FF0000904F0030296E72C1B0020D0
:100B6000A4B70508E8080608C8B705082DE9F84F36
:100B7000524F5349D7F804225248E2F7DDFED7F826
:100B8000FC51AD0000F08680DFF870A1DFF87091B5
:100B9000DFF83081002418E0D7F8F83113F80B3073
:100BA00043FA06F606F00306022E6FD0032E6BD032
:100BB000012E44D02E2244494046E2F7BDFED7F82C
:100BC000FC510134AD00A54264D904F00306A0062F
:100BD0004FEA46064FEA940BDED1AC4228D2D7F852
:100BE000F80110F80B303341990721D1234604E076
:100BF000415C41FA02F292074AD1013303F0030249
:100C0000AB424FEA93014FEA4202F1D12A1B7F2AFD
:100C10000ED992092D494046E2F78EFED7F8FC31F5
:100C200025F03F04B4EB830F34D24FEA940B002637
:100C30000AEA041249464046E2F77EFEACE7D7F8DE
:100C40000412234B22018A589A4229D0214B9A42FE
:100C50002AD0214B9A4229D0204B9A4222D0204BB5
:100C60009A421FD01F4B9A4222D01F4B9A421FD04C
:100C70001E4B9A421ED01E4B9A421DD01D4B9A42CB
:100C800014BF68224D2296E76D2294E73D2292E739
:100C90001D46BBE718490B48BDE8F84FE2F7F2BA2A
:100CA000542288E7532286E74C2284E7442282E7D5
:100CB000412280E746227EE742227CE72C1B00206F
:100CC0005CB70508E80806089CB7050878B705086A
:100CD000AC3E06082C300608982206080C3C060894
:100CE0005C3906084C1E0608101E06086C2A060809
:100CF000FC2A0608D8310608A0B70508F0FF0F0047
:100D000094B70508054B5B695A68824204D8801A7B
:100D1000043053F8200070471B68F5E72C1B0020B7
:100D2000014441F20553884204D398B2002808BF19
:100D30000120704710F8012B03EB43135340F2E7F7
:100D4000034B044A5A610022C3F8DC21704700BFFC
:100D50002C1B002080AB06082DE9F84F82468946FF
:100D6000FFF7DEFF134B5C6983460CB920461CE09D
:100D7000E66804F1100707EB86063D46B54201D34D
:100D80002468F2E7A84658F8040B03885B450ED1A7
:100D900083784B450BD14A46514603301EF0DAFFAB
:100DA00028B96068ED1B00EBA500BDE8F88F45464B
:100DB000E4E700BF2C1B00202DE9F04780460E46DB
:100DC000FFF7CAFF0246002840F08180FF2E03D9BA
:100DD000404941480AF0C0FD404CD4F8DC01351DC3
:100DE000A0B1D4F8E431D4F8E0112B448B420DD9F2
:100DF0002944FFF777F90746F0B90246D4F8E41121
:100E0000D4F8DC01FFF76EF9C4F8DC71D4F8DC31FA
:100E1000F3B9802D2F4638BF80273846FFF747F9B2
:100E2000C4F8DC0178B92846FFF741F9C4F8DC01C1
:100E300040B928460BF000FBD4F8E0312B44C4F84D
:100E4000E031E3E72F460023C4F8E071C4F8E43151
:100E5000D4F8E491D4F8DCA131464D444046C4F8BE
:100E6000E451FFF75DFF0AEB09070AF80900324673
:100E7000000ABE703E4478704146F81C4FF00008EE
:100E80001EF010FF86F803806369D3E90253AB427A
:100E900013D36D000A2D38BF0A25281D8000FFF7E7
:100EA00006F90028C5D0626902605368D268C0F8AC
:100EB0000C801344C0E9013560616369D9685A68E0
:100EC000481C0431D860013A43F8217002441046AE
:100ED000BDE8F087EBD00508C82706082C1B0020CA
:100EE00010B504461EF058FF01462046BDE81040EC
:100EF000FFF762BF08B5FFF705FF008808BD08B51A
:100F0000FFF700FF807808BD08B5FFF7FBFE033050
:100F100008BD08B5FFF7F6FE83780B60033008BD07
:100F20002DE9F8431D46002303600B6013602B601E
:100F3000174BDFF860905C690746884616460CB18F
:100F40004C4505D12B68326813442B60BDE8F8830B
:100F50003B6801333B60E268D8F800301344C8F8BE
:100F60000030E26804F1100303EB8202934207D3DE
:100F70002046FFF721FC2B68246818442860DEE730
:100F800053F8041B88783168043101443160EDE77F
:100F90002C1B002080AB06082DE9F8430E4B0F4FA9
:100FA0005C69DFF83C80DFF83C900CB1BC4201D1B9
:100FB000BDE8F883E36804F1100505EB8306B5424C
:100FC00001D32468F1E755F8042B41460332484623
:100FD000E2F7B2FCF3E700BF2C1B002080AB060851
:100FE000E4D00508E808060830B5013100232024C4
:100FF0000A780AB9027030BD120600F1010520D549
:101000000BB1047028460B78124A03F07F0373B9C2
:10101000013A12F8013F13F0800F054600F101007C
:101020000CD003F07F032B7001230131E0E712F9AC
:10103000015B002DFBDA013BDBB2E8E700F8013C85
:10104000E7E7012B04BF047028460B7803700130DA
:101050000223EAE7DEB8050838B5446803680C44A3
:101060009C42054610D9037BDB0703D500210748C6
:101070000AF072FC103424F007040834214680681A
:10108000FFF725F82C60A86038BD00BFC827060808
:1010900070B504460E4611461546FFF7DDFFD4E94C
:1010A00001302A46314618441EF028FE62682A4460
:1010B000626070BD70B5466804468E42354628BFF2
:1010C0000D460121FFF7C8FFA368681C5919721B60
:1010D00018441EF013FE6368A0680133636028445F
:1010E00070BD38B504460025002914BF084601200C
:1010F00020606560FEF7D0FF237BA06065F30003EE
:10110000237338BD38B505460C460131FFF7E9FFBA
:101110006C6038BD0023C0E90132037B016043F0FD
:10112000010303737047000038B514460546FFF706
:10113000D8FF024B2560636038BD00BF91100208E4
:10114000037BDB0710B5044602D48068FEF7CCFFB2
:101150000023A36010BD38B505461020FEF79CFFA4
:1011600029460446FFF7BDFF204638BD10B50446AA
:1011700050B1037BDB0702D48068FEF7B5FF204641
:10118000BDE81040FEF7B0BF10BD000038B5037BCE
:10119000DB0704460D4603D5002107480AF0DCFBB7
:1011A000016880682944FEF792FF2368A0601D440F
:1011B0002560184438BD00BFC827060838B5044666
:1011C0000D46FFF749FFD4E901301D44656018441E
:1011D00038BDD0E900239A4210B5044602D101215E
:1011E000FFF7D4FFD4E901320021D154A06810BD2B
:1011F00010B50C460121FFF7E1FF047010BD7F29F7
:10120000F8B50C46CEB204D80121FFF7D7FF06701F
:10121000F8BD06F03F06B1F5006FC1F3871546F043
:10122000800607D20221FFF7C9FF65F03F05057070
:101230004670EDE705F03F05B1F5803FC1F3073794
:1012400045F0800508D20321FFF7B8FF67F01F03C0
:10125000037045708670DBE70421FFF7AFFFA40C35
:1012600007F03F0364F00F0463F07F0304704370E2
:101270008570C670CCE738B5054608460C461EF0AA
:101280008BFD214602462846BDE83840FFF700BFE7
:1012900010B51446FFF70EFF047010BD10B51446CC
:1012A000FFF708FF047010BD43688B4234BF002372
:1012B0005B1A4360704738B5154642688A42044657
:1012C0000B4603D929448A4201D8436038BD80685F
:1012D000D21A521B014418441EF010FD6268521BC2
:1012E0006260F3E703781A060AD503F07F03402211
:1012F000134207D110F8012F02F0C001802905D058
:101300001846704723EA02035208F1E702F03F0251
:1013100042EA8313EEE7421C10460132037803F0E1
:10132000C003802BF8D070470023814201D81846B3
:10133000704711F8012D02F0C002802A18BF013356
:10134000F3E701440346002099421A4600D870474B
:10135000127802F0C002802A03F1010318BF0130A5
:10136000F2E700007F289DBF024B185CC0F34000ED
:10137000002070471D0906087F289DBF024B185C9E
:10138000C0F3C000002070471D0906087F289DBFDC
:10139000024B185CC0F38000002070471D0906084E
:1013A0007F289DBF024B185CC0F38010002070475F
:1013B0001D0906087F2809D8064B1B5C13F00C0F8B
:1013C00006D1A0F15F035842584170470020704792
:1013D000012070471D0906087F289DBF024B185C3D
:1013E000C0F30010002070471D0906087F289DBF2C
:1013F000024B185CC0F34010002070471D0906081E
:1014000008B50246FFF7E8FF00B12032104608BDDC
:1014100008B50246FFF7EAFF00B1203A104608BDC2
:101420003038092884BF20F020000738704710B5F5
:1014300001440246E5240020914203D8B0FA80F02E
:10144000400917E012F8013B30B103F0C003802BD4
:1014500011D10138C0B2EFE7BF2B09D9F72B09D85A
:10146000DB0803F0060344FA03F303F00300E3E7A9
:101470001B06E1D510BD0020FCE7023981420B4676
:1014800003D31A880239002AF8D00233181A401000
:10149000704770B51C09944215D2121B01EB440130
:1014A000154603F00F030E46012D31F8024B18BF0D
:1014B0003468DC40A4B2013D20F8024BF3D104B9FA
:1014C000013A104670BD0022FBE7F0B5059E0024EE
:1014D000921B2546A6420ED17600841900230E44A5
:1014E0009A4213D104EB420315B124F8125002338F
:1014F000181A4010F0BD31F8147033F814C0674466
:101500003D4420F814502D0C0134E3E736F8131055
:101510000D4424F813502D0C0133E1E7F0B4049E80
:101520000025921B2C46AE420AD176008519002375
:101530000E449A420FD105EB4201F0BCFFF79DBF6C
:1015400031F815703C4433F81570E41B20F8154051
:1015500024140135E7E736F813100C4425F813403E
:1015600024140133E5E72DE9F043079CDDF828E07A
:10157000DDE90876551E023984464FF6FF78A4EB64
:1015800002096C1C0AD100EB42011FB1012320F8B3
:1015900012300231BDE8F043FFF76FBF31F8024F60
:1015A0004444264409EB0504AC4296BF1C884FF620
:1015B000FF744444744486EA040E17FA8EF72CF83C
:1015C000027B98BF02334FEA144E360C3F0C013DAC
:1015D000D7E738B502290446806838BF02210D4696
:1015E00018B12368B1EB930F07D96900FEF76FFDBF
:1015F0002368A06065F39F03236038BD38B50546B6
:101600000C20FEF749FD2A78037862F300036FF39C
:1016100041030446037028682368C0F39D0060F30B
:101620009F0323606B6863604000FEF735FDA06098
:101630002A68A968C2F39D0252001EF033FB2046BF
:1016400038BD10B501394B1C01D1002010BD30F858
:10165000113032F811401B1B002B04DB01F1FF316C
:10166000F1D00120F2E74FF0FF30EFE710B504466C
:1016700038B18068FEF738FD2046BDE81040FEF71F
:1016800033BD10BD38B505460C460221FFF7A1FF5A
:101690002B78002CB5BF43F001036FF300032B70D0
:1016A0002B704FF00003B8BF64426B6004B938BDC3
:1016B000D5E90132581C686022F81340240CF5E784
:1016C0000023C0E900338360704728B103789B078B
:1016D00002D48068FEF708BD704738B505460C4651
:1016E0004968FFF776FF22782B78A86862F3000339
:1016F0002B7063686B606268A1685200BDE8384077
:101700001EF0D0BA034609B959607047FFF7BABF57
:1017100008B5FFF7D5FFBDE80840FFF7F3BF30B4C9
:10172000057805F0FE0545F002050570056862F3D1
:101730009F0500220560C0E9012130BC1946FFF772
:10174000E1BFF8B504469DF8185004211F4616461F
:10175000FFF73FFF23787DB1002E77F100020BDA0F
:1017600043F001037642237067EB47070021616075
:1017700056EA070304D1F8BD6FF300032370F5E7C1
:10178000D4E901104D1C656020F81160310C41EA6C
:101790000741380C0E460746EAE72DE9F04110EE06
:1017A000106A0378F20F62F300030370C6F30F436D
:1017B00013F4FF43074603D100237B60BDE8F081AB
:1017C000B3F5FF4FF8D0C6F3C754A4F17F05002D41
:1017D000F2DB04D10121BDE8F041FFF753BF162D24
:1017E000C6F31606D8BFC5F1170546F40006DCBFE0
:1017F000EE400025A4F16F084FF01003C8BF093573
:1018000098FBF3F8CCBF963C2C464146C4BF05F08C
:101810000F0594FBF3F4FFF7DCFEC7F8048024B156
:1018200062000021B8681EF081FA45B1BB6806FA73
:1018300005F2C5F1100523F81420EE4001346400D0
:101840004FEA48084445B9D0BB681E53360C0234F1
:10185000F8E72DE9F84304468F18C2F35B020D4602
:101860009846511C089EFFF7B4FE2278B8F1000F8D
:101870000CD042F0010200232270636028461FFA58
:1018800086FCB84205D3401BBDE8F88368F300022C
:10189000F1E70278A2F13003092B00F1010E05D91E
:1018A000A2F14103192B15D8A2F13703B342EAD2B2
:1018B000D4E9010180468946B8F1000F11D101EB4E
:1018C000400213B121F810300232521A52106260F5
:1018D0007046D6E7A2F16103192BD4D8A2F15703C1
:1018E000E4E7B9F8002002FB0C3329F8023B08F1C9
:1018F000FF381B0CE0E7F8B5044615461E46C1B19B
:10190000531E1E444FF0FF37E9000F3109092046EE
:10191000FFF75FFE237800216FF3000323706160FF
:101920004DB9D4E9011000EB4101FFF7A6FD60605D
:10193000F8BD0127E8E700230F2908DC32788A4048
:101940001343013D9BB201F108013E44F4D16268AA
:10195000501C6060A068103920F81230E0E70A4699
:10196000416838B5044609B9506890B113782578B4
:1019700003F0010305F00100181A0AD153689942D7
:1019800008D30AD89268A068FFF75BFEEB0748BF50
:10199000404238BD4FF0FF30F8E70120F6E78842BB
:1019A00010B5044601D0FFF798FE23786FF30003CB
:1019B000237010BD884210B5044601D0FFF78DFE9C
:1019C0002378C3F30002C2F1010262F30003237023
:1019D00010BD88421FB5044601D0FFF77EFE626845
:1019E00062B901212046FFF7F4FDA26801231380AC
:1019F0006360237843F00103237010E02378D90754
:101A00000FD56FF30003A16823700123ADF80E30EA
:101A1000009308460DF10E03FFF780FD606004B0EF
:101A200010BD511C2046FFF7D4FDD4E9012101234C
:101A3000ADF80E30009308460DF10E03FFF745FD9B
:101A40006060D6E72DE9F0470E464968054617461F
:101A500001B12AB931462846BDE8F047FFF73DBE3F
:101A600002F10F0424092144FFF7B3FDD6E9011068
:101A700017F00F026FF0004E04EB010707EB0E08A2
:101A80006FF0010C0CFB01FCAB684FEA48088E4478
:101A90000CEB4E0E08BF1022C444864403EB0C0925
:101AA0000020C2F11002F1B9D04023F80C006FF011
:101AB000010303FB049304F100420233013A184688
:101AC00052001EF033F908F102080346434417B1EF
:101AD00033F8022D92B16F6032782B7862F30003F5
:101AE0002B70BDE8F0873EF811A04AEA000020FA0A
:101AF00002FA29F811A000040139D4E7013FE6E712
:101B0000F0B50E46496885B00546144601B12AB9BC
:101B100031462846FFF7E1FD05B0F0BDFFF759FD5E
:101B2000D6E901212346A868FFF7B3FC6860317845
:101B30002B7861F300032B70DB070246ECD5002302
:101B40007768ADF80E3021099F4201D08B4212D147
:101B50008F42E1D9B36804F00F0433F81110012368
:101B600003FA04F4013C214218BFADF80E30BDF871
:101B70000E304BB9D0E7B06830F8130078B10123CC
:101B80008F42ADF80E30E5D8A96801234AB1009321
:101B900008460DF10E03FFF798FC6860BCE70133BF
:101BA000D2E70B806B60B7E773B553680C464968A2
:101BB00099420646154606D308D89268A068FFF7F2
:101BC00040FD002802DA23462C461D4623782A7859
:101BD00061685340DB0713D401313046FFF7F9FC4D
:101BE0006B680093AB68B068D4E90121FFF76DFC26
:101BF00070602278337862F30003337002B070BDF6
:101C00003046FFF7E6FC6B680093AB68B068D4E938
:101C10000121FFF783FCEBE7F7B553680C464968F1
:101C200099420646154606D328D89268A068FFF761
:101C300008FD002822DA234601272C461D4623787A
:101C40002A7861685340DB071AD501313046FFF727
:101C5000C0FC6B680093AB68B068D4E90121FFF762
:101C600034FC70602278337802F001020FB1C2F1C7
:101C7000010262F30003337003B0F0BD0027DEE71A
:101C80003046FFF7A6FC6B680093AB68B068D4E9F8
:101C90000121FFF743FCE4E72DE9F04F16464A68BF
:101CA00073689A4224BF33460E460D4628BF1D4630
:101CB00033787168DA0785B0044621D42B7813F0A5
:101CC00001071DD1FFF785FCD5E9011CA068B668A6
:101CD0003B4699420BD100EB4101FFF7CEFB237845
:101CE00060606FF30003237005B0BDE8F08F36F835
:101CF00013203CF813502A4020F813200133E8E762
:101D000001312046FFF765FC32782978D6F804C007
:101D1000A068D5F8088082EA0103DB4303F00103E1
:101D20005F420093B368BFB202F00102A3F102095F
:101D30006B68029701F001015742BFB2C1F1000E7A
:101D4000A3EB0C0301971FFA8EFE0CF1FF378246BE
:101D500003937B1C16D1009B00EB4C011BB10123AC
:101D600020F81C300231FFF788FB606033782A7856
:101D7000C3F30003C2F300021340227863F30002AE
:101D80002270B1E739F802BF019B83EA0B0B039B7A
:101D90005A4403EB070BBB4598BFB8F800B0029B51
:101DA00094BF8EEA0B0BF346594402EA010B8BEA0F
:101DB000030B009B13FA8BF32AF8023B4FEA134301
:101DC00098BF08F10208090C120C0093013FC0E70C
:101DD0002DE9F84F15464A686B689A4224BF2B4696
:101DE0000D460E4628BF1E462B786968DA07044662
:101DF0002ED4327812F001082AD1FFF7EAFBD6E997
:101E0000013CA9686D68A768ED1A4246934210D15B
:101E10005B00194400223B44954213D103EB450378
:101E2000DB1B5B10636023786FF300032370BDE856
:101E3000F88F31F812003CF81260304327F8120096
:101E40000132E3E731F8120023F812000132E3E730
:101E500001312046FFF7BDFBD6E901382F783678EF
:101E60006968A068AD6807F0010706F00106C7F1D0
:101E7000000EC6F1000C1FFA8EFE1FFA8CFC4A1EE3
:101E8000023D82464FF00109A3EB010B531C08D120
:101E900000EB4101FFF7F1FA2378606043F00103A2
:101EA000C4E735F8023F8EEA03031F440BEB02033D
:101EB000934296BFB8F8003063468CEA03031E4491
:101EC00047EA06036FEA030319FA83F398BF08F1A0
:101ED00002082AF8023B360C3F0C4FEA1349013A3C
:101EE000D4E7F0B514464A6863689A4228BF23468F
:101EF0000E4624BF0C461E462778337861685F4043
:101F000017F0010785B005463AD1FFF762FB237849
:101F100013F0010328D1D6E90117A2686468A86804
:101F2000641A994210D149000A4400230144A34293
:101F300014D101EB4301FFF7A0FA2B7868606FF32F
:101F400000032B7005B0F0BD32F8136037F813C0F2
:101F500086EA0C0620F813600133E2E732F81360DA
:101F600021F813600133E2E7CDE902770197736846
:101F70000093B368A868D4E90121FFF7F4FADCE71D
:101F80000131FFF726FB3378A868DB4303F0010338
:101F900003932378DB4303F00103029301230193AE
:101FA00073680093B368D4E90121FFF7DCFA2B785A
:101FB000686043F00103C4E72DE9F04F4B6885B03A
:101FC00004460E4615460BB1536823B900236360DF
:101FD00005B0BDE8F08F81422FD1FFF70FFBA5427E
:101FE0000646074600D105466B68716820461944CD
:101FF000FFF7EFFA2268A068C2F39D0252000021A9
:102000001DF094FEB368D6F804C002936FF001038C
:10201000D4F808A003FB0CF3D5E90128023B0AEB36
:102020004C010020039392B3039BDDF808B0CDF878
:1020300004C003EB010E002318E0824204D1FFF735
:10204000DDFA05460746CFE70027CDE73EF8029FB9
:1020500099443BF8023B1846B8F8003003FB009364
:102060000198AEF8003001381B0C0190019800284F
:10207000ECD1084601F1020E0BB10B807046A0EBCB
:102080000A004010013A08F102087146CBE760608F
:10209000337829784B4013F0010F237838460CBF72
:1020A00062F3000343F00103237005B0BDE8F04F75
:1020B000FFF7DCBA4B6870B50646144613B11378C7
:1020C000DA0702D50023736070BD636823B901216C
:1020D000BDE87040FFF7D6BA0846FFF78FFA05460D
:1020E0002046FFF78BFA012104463046FFF7CAFA73
:1020F000636883B1A3681B88DB0704D52A46314691
:102100003046FFF759FFD4E9012101230846FFF7C4
:10211000C0F9606038B92846FFF7A8FA2046BDE844
:102120007040FFF7A3BA2A4629462846FFF744FF26
:10213000DEE72DE9F04F0C4651688FB09146013132
:1021400005460293FFF745FAD9F80420A868013242
:10215000520000211DF0EAFD00236B60D9F8041045
:1021600020460131FFF735FA49462046FFF7B5FA18
:10217000029B6768D4F808B0D3E901360193AB68D5
:102180000393019BBB422CD82DD332463946584687
:10219000FFF757FA002823D1039A606001231380C8
:1021A0006B60029A99F8003012785340DB0714D51F
:1021B0002B7843F001032B70636873B14FF0FF314C
:1021C0000BA8FFF7A5FA0BAA29462846FFF7ECFC57
:1021D000029A21462046FFF7E7FC0FB0BDE8F08FDA
:1021E00001DA0023DCE7019B03F1004001384FEAEC
:1021F000400A36F81020002312F4004F03F10101C9
:1022000052D07A009BB24FF0000E791C02F1020806
:102210000592C3F110022BF817E0D8446160DC4648
:1022200077460492C44543D336F8100000FA03F20F
:102230000492019A012A09D906EB0A00C3F110079A
:1022400030F8020CF840049F074304970198059A60
:10225000091A6960039801F10041013900EB41015D
:1022600005910AF102010991B11E5A440891D4F86E
:1022700004A00199514527D30AF1004A0AF1FF3A17
:102280000BEB4A0A0020C3F11006D3457BD96FF04F
:1022900000416B682BB15A18039830F81220002ABD
:1022A0007BD06FF000417DE0520092B20B46A3E775
:1022B000BCF800E00EFA03F21743049A2CF8027BF4
:1022C0002EFA02F7BFB2ADE7118832F8026C46EA87
:1022D00001460499B6FBF1F60999511A069108993D
:1022E0000791069F00218E46BA420CD81088091A21
:1022F000002942D1059921F8026905910AF1FF31BF
:10230000023A6160B3E70798B7F8008030F802CF6F
:1023100007900CFA03F040EA1E4E1FFA8EF070434D
:10232000404503D2A8EB000C8C450ED80144A1EB2C
:102330000808C8F1000139801FFA88F1003118BF80
:10234000012101EB18410237CEE7ACEB01013980E6
:102350000021F8E738F802CF0CFA03FC4CEA1E4ED5
:10236000B7F800C010FA8EF0604427F8020B000C9A
:10237000BA42EFD8091A013EBAE70020DDF8208002
:10238000069F8646F4E7BAF8002042FA03F10143BB
:10239000B2402AF8021990B277E7013B6B6078E708
:1023A000013B63606368002B3FF4FBAE5A183BF8B7
:1023B0001220002AF4D0F4E6F0B51F464B6885B031
:1023C00006460C4615464BB11378DA0706D47B68EF
:1023D000012B07D1BB681B88012B03D1002373603D
:1023E00005B0F0BD01213046FFF74CF96B68002BBA
:1023F000F6D02046FFF702F904462846FFF7FEF81C
:10240000054601A8FFF75CF96B68B3B1AB681B88A0
:10241000DB070AD5224631463046FFF7CDFD3B4665
:102420003246314601A8FFF784FED5E90121012398
:102430000846FFF72EF8686048B901A8FFF745F98C
:102440002046FFF713F92846FFF710F9C8E72246A0
:1024500021462046FFF7B0FD3B462246214601A813
:10246000FFF767FED0E710B5D0E90121002301EBAB
:102470004202914205D30278D20748BF5B42184618
:1024800010BD32F8024D44EA0343F2E730B5D0E91B
:102490000124002304EB4202944206D30278D207BF
:1024A00048BF5B420B60012030BDB3F5004F04D242
:1024B00032F8025D45EA0343EEE70020F4E72DE938
:1024C000F043884661B19D18D0E901140026A4F1BB
:1024D000020C4FF0010937461A4419B9BDE8F083E0
:1024E0001D46F1E73CF8024F103744EA0646072F35
:1024F00001DC0139F1E790F800E0B4B21EF0010F01
:102500001FBFE44359FA84F4A4B24FEA1429E4B299
:10251000B8F1000F09D005F1FF3E05F8014C7345F5
:10252000DCD0083F360A7546E1E705F1010E2C7054
:102530009645F5E7D0E901329FED0C0A9FED0C7A44
:1025400002EB43039A4205D30378DB0748BFB1EEA1
:10255000400A704733F8021D07EE901AF8EEE77A4A
:10256000E0EE077AB0EE670AECE700BF000000007B
:10257000000080472DE9F84F44689DF828A00B9D86
:102580008046894616469B469CB982B1561E2B460C
:1025900016F8012F18463AB930230370002300F8CB
:1025A000013F401BBDE8F88F03F8012BF0E72846F8
:1025B000F2E764002046FDF76FFD22460746D8F893
:1025C00008101DF06FFBABF13A0B28462A4607EBCB
:1025D000040CACF1020300219F421C4632D9303179
:1025E000392988BF5944541C11703B469C451946F3
:1025F00032D8BAF1000F08D00123211A032902BFF3
:10260000941C82F801A02046D3B13846FDF76CFD3A
:102610003EB130461DF0C0FB23463044B0421C465C
:1026200023D898F80030DB0742BF2D2323700134F4
:10263000631E2A469A421DD300232370601BB1E714
:102640002246C6E7248844EA0141B1FBF9F423F8A5
:10265000024909FB1411BFE7098802330029C5D0DC
:10266000BAF1000FECD00023C7E710F8012D03F8F2
:10267000012BD3E71178187802F8010B03F8011940
:10268000D8E7D0E9023293423DBF5A1C82601878E5
:102690004FF0FF307047036810B5044613B140682F
:1026A000FDF722FD2046BDE81040FDF71DBD0000EE
:1026B000F8B5054610200C461F461646FDF7ECFC03
:1026C000054B8460C0E900743444C4606B60034B04
:1026D0002860AB60F8BD00BF832602089726020879
:1026E0000369272B1DD0222B1BD0752B03D023F081
:1026F0001002622A10D14269272A12D0222A10D051
:10270000722B09D1622A0ED18069272809D0A0F145
:102710002203584258417047622B04D14369722BFF
:10272000F1E7012070470020704702690A2A10B5BE
:10273000044622D1C3690133C36101232362636963
:102740002361A3696361D4E9010398476369A061C8
:102750000D2B07D10A239842636103D1D4E9010309
:102760009847A061A369013306D163695A1C03D05D
:102770000A2B1CBF0A23A36110BD036A092A04BFE8
:10278000073323F007030133D8E770B504460E463C
:1027900000252069431C01D1284670BD0A2808D1B4
:1027A00016B1A36A002BF7D02046FFF7BEFF012524
:1027B000EFE7FEF7D7FD18B12046FFF7B6FFE8E7D1
:1027C0002369232B08D12046FFF7AFFF23695A1C4A
:1027D000DFD00A2BF7D1DCE75C2BDDD163690A2B54
:1027E000DAD12046FFF7A1FFE6E700002DE9F74F19
:1027F000044600218164FFF7C8FFE369A363636AAD
:10280000256AE563002B04DA062284F840200133B0
:1028100004E007D0052284F84020013B636203B046
:10282000BDE8F08F90B3A36A83BBD4E90C200423E6
:1028300084F840306FF00043D118013D30F811109A
:102840008D42ECD017D9E16A8A4207D3083149009A
:10285000FDF73DFCE36A60630833E362D4E90C32C0
:10286000591C216322F81350636AD0E7013A2263AE
:10287000626A013A6262226BD11830F811108D42FF
:10288000F4D3CCD0022384F84030C8E72169481C37
:1028900001D10023F7E72046FFF722FF81460028F9
:1028A00000F03D81002384F840302369752B5DD012
:1028B000622B50D16369722B0CBF022501254FF0AA
:1028C0000B030CBF4F46002794F84020002A55D137
:1028D00084F840303DB12046FFF727FF022D02D19A
:1028E0002046FFF722FF23692046222B0CBF4FF022
:1028F00022084FF02708FFF718FF2369434540D10E
:10290000636998453DD12046FFF70FFF2046FFF74A
:102910000CFF03264FF0000A04F14405D4F810B070
:10292000BBF1FF3F00F0F580012E03D1BBF10A0F90
:1029300000F0EF80B24526D3514604F14400FEF783
:10294000B3FC01212046FFF720FF2046FFF7C8FE19
:102950000028AAD163E7722B0CD16369622B4F4622
:102960000BBF022501250B230A23ADE701250A230E
:102970000027A9E700250A232F46A5E79A42A9D0F8
:102980004DE70126C6E7D84509D1414628460AF158
:10299000010AFEF734FC2046FFF7C7FEBEE7BBF195
:1029A0005C0F40F0B0802046FFF7BFFED4F810A0C7
:1029B0002FB15C212846FEF722FCD3467EE0BAF117
:1029C000620F50D028D8BAF14E0F00F0828010D894
:1029D000BAF1220F1ED0BAF1270F1BD0BAF10A0F9D
:1029E0003ED0AAF1300BBBF1070FE2D84FF0030A3B
:1029F00079E0BAF15C0F0DD0BAF1610F7BD0BAF17A
:102A0000550FEED194F840200B2A38D15C2128468E
:102A1000FEF7F5FBD3461BE0BAF1740F26D00BD8B6
:102A2000BAF16E0F25D0BAF1720F0FD0BAF1660F5E
:102A3000D7D14FF00C0B0BE0BAF1760F1CD0E1D3DD
:102A4000BAF1780FCDD14FF0020A1FE04FF00D0B15
:102A500094F840300A2B51D159462846FEF7CFFB57
:102A60004FF0000A97E74FF0080BF1E74FF0090B22
:102A7000EEE74FF00A0BEBE74FF00B0BE8E7BAF18C
:102A8000750F14BF4FF0080A4FF0040A4FF0000B07
:102A900011E02046FFF749FE226901921046FEF739
:102AA0007FFC002800F04B81019A1046FEF7B8FC2D
:102AB0004FEA0B1B83441AF1FF3AEAD2BBF1FF3F06
:102AC000CED0A24B9B45C3D94FF0010384F84030D0
:102AD000C6E79F4809F0B6FE2046FFF726FE2269AA
:102AE000303A02EBCB0B6269303A072AE6D8BAF1EA
:102AF000010AF1D1E2E74FF0070BA9E7BBF1FF0FA5
:102B0000E2D80B2BE0D15FFA8BF12846FEF770FB81
:102B1000A6E7B2453CBF032284F840200CE70846F4
:102B2000FEF72AFC054620691DB95F2801D07F28E1
:102B30003ED9072384F8403004F14405C1B2284649
:102B4000FEF756FB2046FFF7F0FD2069421C1BD123
:102B50002846FEF73EFB7F4F0646002557F8251016
:102B600030461DF023F900281CD10D35EDB2102D93
:102B700084F840507FF453AE774BD3F8E831002B04
:102B800014BF0D230F237EE6FEF7F6FB40B9206944
:102B90005F2805D07F2803D8FEF7F8FB0028D7D0A0
:102BA000217CCCE7FFF63BAE0135242DD6D136E6AD
:102BB000FEF7ECFB68B321692E2935D1092384F88F
:102BC000403004F144063046FEF719FB2046FFF77B
:102BD000ACFD09272069431C3FF421AE002D35D1FF
:102BE00020F02003452B31D16521304684F8407018
:102BF000FEF705FB2046FFF798FD21692B2901D040
:102C00002D29E7D13046FEF7FAFA2046FFF78DFD71
:102C1000E0E723692E2B04D16069FEF7B7FB00289B
:102C2000C9D100254D4F31E00823302984F84030C8
:102C3000C7D1656945F02005A5F16203162B9DBF3C
:102C4000474DDD4005F001050025BAE7FEF794FB8E
:102C500028B121692E290DD184F84070D2E720696E
:102C6000FEF794FB0028F4D123692E2BF1D05F2BC3
:102C7000CBD0D4E521F020034A2BC3D1ECE7652E5D
:102C800001D0632E00D10137013501373E7816B1EE
:102C90002369B342F3D12046FFF747FD0EB9012364
:102CA000F1E5212E07D123693D2BF8D12046FFF70E
:102CB0003CFD3823E7E52E2E0FD123692E2B02D1C0
:102CC00063692E2B01D05B23DDE52046FFF72DFD48
:102CD0002046FFF72AFD0C23D5E56FF0010303FB27
:102CE00005772B4607EB45025678632E01D0652EFB
:102CF0000BD10135216917F81520914213D12046D7
:102D0000FFF713FD2B46652EECD1164AD35C84F8F1
:102D1000403003F0FB02532A01D0552B05D1A36AA2
:102D20000133A3627BE5632EEEE703F0FD02542A34
:102D300002D0582B7FF473ADA36A013BF1E74FF04B
:102D4000010384F84030834682E600BFFFFF100095
:102D5000E2090608940A06082C1B00209D090608B3
:102D600001204000680A06087FB5064601AD5420E0
:102D700085E80E00FDF790F90446034695E8070044
:102D800043F8046B83E8070001236FF00102C4E9F4
:102D9000073200250A22C4E90B23C4E9095514208F
:102DA000FDF77AF92021606304F14400FEF799F9F8
:102DB000636B20461D80C4E905552561FFF7B5FC0E
:102DC0002046FFF7B2FC2046FFF7AFFC2046FFF796
:102DD0000DFDE36B012B18BF0523204618BF84F8B7
:102DE000403004B070BD30B585B001AC054620461A
:102DF000FFF75EFC94E80E002846FFF7B5FF05B02C
:102E000030BD30B585B001AC0146054620461BF00B
:102E10008FFE2846FEF764F894E80E00FFF7A4FF43
:102E200005B030BD10B5044670B1C368406898471E
:102E300004F14400FEF784F9606BFDF755F9204674
:102E4000BDE81040FDF750B910BDD0E90432013B98
:102E5000036152F823007047C1F17F5101F57F11E2
:102E6000036901F57F513F311944436953F821004B
:102E70007047F8B5446A06460D46B4B1D4E900037C
:102E80000B44834222D90831002201442046FDF739
:102E900029F90246B8B9616820460831FDF722F9E0
:102EA00063682360336A63603462802D2F4638BFC5
:102EB000802707F10800FDF7EFF800230760436063
:102EC0000446706202E023682B4423606068054476
:102ED000656008342044F8BD38B50D46D0E90313C9
:102EE0008B42044608D3103189004069FDF7EFF8A2
:102EF000E36860611033E360D4E90432591C216156
:102F000042F8235038BDF8B50D461F46D0E90013EE
:102F10008B420446164608D31031C9008068FDF77D
:102F2000D6F82168A06010312160D4E901104B1C53
:102F3000636050F8312065F3170200EBC10340F8DD
:102F40003120DE705F60F8BD10B48469CAB200231E
:102F5000A16B5DF8044BFFF7D6BF0000F7B586699B
:102F60000F4696F84010072905461FD1D6E91210E2
:102F7000FDF722FF902F04460ED1C100002241F040
:102F8000020105F1280009F0B1FF28B14468E30708
:102F900020D544F0010002E0200140F0020001468B
:102FA000284603B0BDE8F040FFF796BF082907D1D7
:102FB00033460022D6E91210DFF78CFF0446E6E71D
:102FC000092912D1009600230122D6E91210DFF759
:102FD000FFFF04460C212846B66BFFF74AFF4FF46B
:102FE0009D730660C0E90134D9E7A1F10A03012B02
:102FF0001CD8D6E912100A290BD8FDF7DDFE96F889
:10300000403048B10A2B14BF0A21062141EA0010C2
:10301000C5E7FDF7A1FEF2E7064C0748D6E9122105
:103020000A2B18BF20460FF0B3FBD2E7090141F08D
:103030000E00B4E75C3906080C3C0608DE2807D011
:1030400010F0010306D043080CBF01200020704798
:103050000120704718467047FE2807D010F0010382
:1030600006D0430814BF012000207047012070479C
:103070001846704710F0010204D040F001000860CB
:1030800001207047A8B110F003030FD102793A2A4A
:103090000ED183680B6013F001000AD19A0708D1A2
:1030A0001868044BC31A584258417047104670477D
:1030B00018467047C02E06082DE9F04F2D2A85B01E
:1030C0000446884616461D460AD10021FFF7C4FE75
:1030D00030B1810740F070810379922B40F06C8110
:1030E000A6F11E03012B59D82A46A9460BE01E2E35
:1030F00047D1FFF7B1FFB8B90846FFF79FFF002897
:1031000018BF4F46B94609F1FF376AB1013A114677
:103110002046FFF7A1FE2369A3EB090C6369014672
:1031200043F82C00002AE2D10021B94231D16D1AB6
:10313000012D00F04181A6F12303022B01D92A2E93
:1031400078D1691E2046FFF787FE01A9FFF792FF9D
:1031500000285AD0232E3AD0242E3BD0252E14BF3F
:103160004FF022094FF01809AF1E002F35DA002D5D
:1031700040F06C81019EF30740F16D8146F0010142
:103180001FE0FFF75BFF0028CED10846FFF764FF82
:10319000B5E72046FFF759FE0131C6E7202ECAD118
:1031A00000212046FFF758FE0246FFF747FF60B9AF
:1031B0001046FFF751FF0028BDD0DE212046FFF763
:1031C00044FE2046FFF788FEF6E0FE21F6E74FF0CA
:1031D0001609C9E74FF01709C6E739462046FFF739
:1031E0003BFE02A9FFF746FF78B1B9F1220F07D0E5
:1031F000DDE90112484609F03BF9013F0190B4E7CF
:1032000002980DF02CFA0028F2DAA91C8900204659
:10321000FFF72FFE46EA05260146C0F8008046600B
:10322000002DCED02046FFF710FE013D01EB8503B7
:103230009860F5E7A6F12603022B38D8691E2046D0
:10324000FFF70AFE01A9FFF715FF0028DDD0A5F161
:103250000209B9F1000F8ADD09F1FF312046FFF7BD
:10326000FBFD02A9FFF706FF0028CED04946204605
:10327000FFF7F2FDC0F3071000F0FD03412BC4D0AF
:103280002338C7B202980DF0EAF91A2F0AD800289D
:10329000BBDBDDE90112384609F0EAF8A9F10209C1
:1032A0000190D6E71E2FF4D90028F2D1ADE7292EE0
:1032B00018D100212046FFF7CFFD01A9FFF7DAFE64
:1032C0000028A2D001212046FFF7C6FDC0F3071059
:1032D00032281ABF3E38C0B20220019908F094FB90
:1032E000019044E7052E71D100212046FFF7B4FD7F
:1032F0000746002889D010F0030A03D10379563B12
:10330000012B82D901212046FFF7A6FD00F00F0313
:10331000022B7FF47AAFBAF1000F7FF476AF3B79DE
:103320002C2B7FF472AFBB6803F00F02022A7FF4EC
:103330006CAF1B09482B7FF468AFFB68002B3FF490
:1033400064AF9A077FF461AF1A79302A7FF45DAFDA
:10335000D3F808B04FEA101902A95846FFF78AFEC1
:1033600068B9424942480BF0E1FFA1693A6809682F
:10337000054653460CF0A2F82846FCF769FE4FEAD2
:10338000C901012241F0020104F1280009F0AEFD5B
:10339000029B43604846FDF7B7FD03785F2B20464C
:1033A0000DD1FFF752FD2046FFF74FFD0023082205
:1033B00019462046FFF780FE05B0BDE8F08FFFF705
:1033C00044FD59462046FFF787FD1EE72C2E7FF46B
:1033D0001CAF01212046FFF73FFD00210246204699
:1033E000FFF73AFD02F00F03022B7FF40EAF002827
:1033F0003FF40BAF87077FF408AF0379322B7FF4DC
:1034000004AF1109C90087681A48002241F002017F
:1034100009F06CFD00283FF4F8AE02AA39094068B3
:1034200008F024FA029B002B3FF4EFAED90707D433
:103430009A077FF4EAAE19680F4A91427FF4E5AE2D
:10344000039A002A7FF4E1AE019390E62046FFF74D
:10345000FCFC013D8BE60C212046FFF70AFD4FF4F2
:103460009D7301460560C0E90136AAE69D0B06087A
:103470007C280608240B0608C02E0608036830B511
:1034800013B91360184630BD9C0702D010600120AC
:10349000F9E75C68E5B28D42F8D108331360200A81
:1034A000F1E700002DE9F04F93B000244023029093
:1034B0004FF400700F460192CDE90534FCF7ECFDA6
:1034C000202307908020CDE90834FCF7E5FD214654
:1034D000CDE90A070FA8CDE90D4409F0C9FC019B0D
:1034E000002B53D0022B0CBF3F2222460023B96B86
:1034F00005A8FFF708FD4FF00008069C002C00F01F
:103500006981013C079BAE4D069403EBC40253F85E
:103510003430D6785268C3F3170AAA4B13F806B0B2
:10352000A94B9B5D632E88BF43F4807305EB430575
:103530000BF03003102B0BF00F0929D0202B5AD0A1
:10354000B8F1000F40F015810BF001030393039BCA
:10355000134035F8134024F47F6121F00F01B1F5D9
:10356000805F40F0218197F84010C4F30B04A14222
:1035700002F1010440F0FC801BB9314605A8FFF7B9
:10358000EDFC3846FFF732F92246E0E73D22ADE791
:1035900012B1B8F1000FAED005EB4205914502D84B
:1035A0004FF00108A9E7A84635F8023B23F47F61F4
:1035B00021F00F01B1F5805F0DD197F84010C3F3F2
:1035C0000B03994215D105A83146FFF7C7FC3846D1
:1035D000FFF70CF98FE7531C4B4504D23246514696
:1035E00005A8FFF790FCB8F8001005A8FFF7ACFCA1
:1035F00081E70132D2E7B8F1000F11D002F10043A8
:10360000013B35F8133023F47F6323F00F03B3F548
:10361000405F1BD1002105A80392FFF75DFC039AD0
:1036200005EB4204914525D8019B002B46D100248F
:1036300005EB490922464D4560D1012A40F08180C1
:103640001BF0400F7DD00025294674E0012AA7D940
:1036500097F84030052B40F0EC805C495C480BF05B
:1036600065FE00230446BA6B39680BF027FF20463D
:10367000FCF7EEFCA04634F8023B23F47F6121F016
:103680000F01B1F5805F17D197F84010DBB2994276
:103690000ED1072905D1314605A80392FFF75EFC3C
:1036A000039A03923846FFF7A1F8039A0132B9E76B
:1036B000002A3FF475AFCBE7531C8FE7052EB6D138
:1036C000002105A8FFF7C8FB0028B0D1012105A8FB
:1036D000FFF7C2FB830700F0B38000F00F00022861
:1036E000A5D005A8FFF7B1FB05A8FFF7AEFB0023A7
:1036F0000822514605A8FFF7DFFCFCE639F8023D39
:1037000023F47F6121F00F01B1F5805F05D1DBB2B9
:10371000072B90D1013401328DE7214605A8FFF730
:103720009BFB00B10132013485E7FFF78EFB0135C9
:10373000002818BF0146A54205A8F6D1FFF7CCFB2B
:10374000D9E61BF0800F04D0002105A8FFF7C4FBC9
:10375000013423463246CCE7012A3FF421AF12F070
:1037600001010DD0B9F1030F7FF472AF012107E021
:103770002246B9F1020FEFD1012A3FF411AF002127
:103780001BF0010F02F1FF3308D0688820F47F603E
:1037900020F00F00B0F5805F08BF5308012BD9D18E
:1037A00000293FF4A8AED5E7531C514605A8324680
:1037B000FFF7A9FB214605A8FFF7C6FB9DE600BF62
:1037C0005C0C0608AB0B0608E40F0608600B060845
:1037D000702506080FA809F063FB0E9850B14168E8
:1037E00022460831FCF77EFC0E9B5A681A600D9A3F
:1037F0005A600D9397F84030002B7FF429AF099B56
:10380000002B3FF425AF0A9B07981B680C93FCF72D
:103810006BFC0A98FCF768FC3846FFF703FB0CAB1F
:1038200093E80300029B83E80300184613B0BDE849
:10383000F08F022B01D1064910E7064906480EE732
:1038400000283FF4F4AE03793A2B7FF4F0AE48E75A
:10385000720B0608990B06087C28060810B540680C
:1038600000B910BD4468FCF73FFC2046F8E70000B3
:103870002DE9F041054630200E4690461F46FCF7E4
:1038800024FC072D04460570C660A0F8148001D002
:10389000012D0FD1B3681B09E38207F02FFB04232E
:1038A0002061678323852020FCF7F6FBE062204639
:1038B000BDE8F081014B5B5DEEE700BF94100608A8
:1038C00010B50446C06AFCF70FFC2046BDE8104066
:1038D000FCF70ABC30B5448D0022944202D8002384
:1038E000184630BDC36A03EBC2035D688D42F7D052
:1038F0000132F2E770B504460D461646FFF7EAFFBF
:10390000C0B9218D638D8B4208D30631C900E06AAE
:10391000FCF7DDFB238DE06206332385638DE26ACD
:10392000591C02EBC300618502F833600023437029
:103930004380456070BD43680BB9FFF7CBBF1846A5
:10394000F9E7F8B544680F462CB9F8BD032BFCD154
:1039500004230370F9E723465D68002DF5D07E68E7
:1039600018463146FFF7B6FF2B460028F4D00378FF
:10397000033B022BE9D805233B701D46002231464C
:103980002046FFF7B7FF0378002BDFD1057064688E
:10399000F4E7436A5B8B012B1EBF03695B1803616D
:1039A0007047C36A10B50446DB6F806A9847A38BE3
:1039B000626A0133D18C9BB29942A38338BFD3840E
:1039C00010BD838B10B5013B8383C36A0446D3F8D3
:1039D0008430806A984720460121BDE81040FFF7F7
:1039E000D8BF2DE9F04180461F4659B111F00305BB
:1039F00010D14E68F3B293420CD1360A01F108049B
:103A0000B54201DBBDE8F08154F8041B4046B847DD
:103A10000135F5E740463B46BDE8F04118472DE942
:103A2000F04F044685B00D4691469A461BB10B8B6C
:103A300043F008030B83636AA5F820901A8B42F0C9
:103A400030021A831B78002B49D1E36AA06AD3F8AD
:103A5000B4604A4653462946B44605B0BDE8F04F27
:103A60006047DB6A03EBC60B13F83630043B012BCF
:103A700020D8002319E0EB6A039A039903EBC202F2
:103A800013F83130052B0ED1DBF80410536899423E
:103A900009D1E36ABBF802205B69A06A1F460023D4
:103AA000B84708F10108039B01330393039A6B8D18
:103AB0009342E0DC0136636A5A8DB242D1DCD4E92C
:103AC0000A03B8F1000FC0D0CDF800A0D3F8B84079
:103AD00042464B462946A04705B0BDE8F08F002678
:103AE000B046E8E72DE9F0410446884611461A46FB
:103AF00000238579878AC68A837143610F4BFFF75C
:103B000070FFA368C3B9E18A51B1A28A42B9E36ADE
:103B1000A06AD3F8A0309847E36AA06A5B6C984724
:103B2000A38AE28A41462046FFF779FF003518BF95
:103B30000125A571A782E682BDE8F081B152020895
:103B4000024B89689D22FFF74CBF00BF8D5F0208C2
:103B5000024B89686B22FFF744BF00BFFD42020899
:103B6000C36A10B50446D3F88830806A00219847AC
:103B7000E36AA06A5B6B0E219847E36AA06AD3F8F8
:103B8000CC300121984720460321BDE81040FFF7C3
:103B900000BF38B5C36A04469B6C806A0022984710
:103BA000E36AA06AD3F8C05000231A461946A84712
:103BB0002046BDE83840FFF7D3BFC36A89685B6D14
:103BC000806A002209091847C36A89681B6C806AE9
:103BD000184710B50446084611462268FFF748FE0C
:103BE000636A436000238360236A13B9206210BDB7
:103BF00013469A68002AFBD19860F8E770B54379BC
:103C0000012B05460C4606D1436A0A465B8B02210E
:103C1000FFF7DFFF2061A268216928464C23BDE839
:103C20007040FFF75FBF70B513464279012A064620
:103C30000C4604D10A460721FFF7CBFFA061A56916
:103C4000E268304646232946FFF74CFFE88A70BDFC
:103C50002DE9F04F87B0054600AF0C4611B90121A0
:103C6000116013E011F0030619D10B79682B06D10E
:103C7000CB681B0913608C68002CF0D0012604F07F
:103C80000F03022B0DD12109002EE9D0EB6AA86A9F
:103C90001B6B002298471C37BD46BDE8F08F0026FD
:103CA000EDE716B9A3681B09136063684FEA132890
:103CB00004F1080308F1FF3AFB609B464FF000094E
:103CC000C14526DB0AF10E0323F00703ADEB030D1C
:103CD000C7F808D0E9464FF0000BC34522DB514638
:103CE000B868FDF769F8EB6A01461B6BA86A002209
:103CF0009847002ECFD00C3401264645CBDA54F835
:103D0000041BEB6AA86A5B6D00220909984701361B
:103D1000F3E75BF8040B0009FDF7F1F809F101097D
:103D20008244CDE7BBF1000F05D04FF02E0389F898
:103D3000003009F10109FB6853F8040BFB6007F13F
:103D400014010009FDF7E5F87B697B601A4601461E
:103D500048461BF0A7FF7B680BF1010B9944BCE7B9
:103D6000036823B919B18B0704BF0B680360704760
:103D700038B5836804460D465BB9114605480BF01B
:103D8000D5FA2946A06004F10C00BDE83840FFF7E1
:103D9000E7BF38BD7C2806082DE9F04F04460D46E4
:103DA00062712B786162072B4FF000018DB01646CF
:103DB000016105D0824AFFF7DBFF0DB0BDE8F08F4F
:103DC000012A06D0436B00F108021B68006B3146E4
:103DD00098476379D5F80C80032B10D10BAA4621A4
:103DE00008F10C00FFF74AFB636B0B9A9B680146D6
:103DF000206B9847A368A883002B40F0B080D8F8C8
:103E00001010002944D001F00F05022D3CD10B0900
:103E10005E2B0ED004D83E2B0AD06A4A2046CAE751
:103E2000752B37D040F204529342F6D1032500E0BF
:103E30000125D8F8143009930AAA192109A8FFF717
:103E40001DFB4FF000090690069B994524D163792C
:103E5000012B15D9636B206B5B6829469847637902
:103E6000042B0DD10023606A03950293818B226B92
:103E7000CDE900310521D2E90232006907F055F899
:103E8000A368002B6BD198E74F4A2046FFF770FFDD
:103E90000225CEE70025CCE70A9B53F829100B79C1
:103EA000082B4FEA890B02D109F10109CCE7052B58
:103EB00001D0464AB2E7CB68002BFAD18B681A7959
:103EC0002C2AF6D19F6807F00F02022AF1D1DB6895
:103ED0000593002BEDD09A07EBD11B79302BE8D15D
:103EE000059B0BAA03F10800A421FFF7C7FA3F09BD
:103EF00040F203439F4282461BD1012805D10B9A11
:103F0000136803F00F03022B04D0314A0A9B53F8C5
:103F10000B1083E72169012E01F10103236119D000
:103F20001268636B206BDB681209984790B9294AC5
:103F3000ECE7B7F54F7F16D1012803D10B9B196829
:103F4000CF0701D4244AE1E7012E03D04910206BAA
:103F500003F062FAA368002BA6D0DDF81480D8F82D
:103F60000030E36029E7B7F5617F1DD1012803D94F
:103F70000B9B1B68D80701D4184AC7E7012EE9D06C
:103F80005B1001270B9A52F82720D10701D4144A5D
:103F9000BCE719465210206B0793013703F043FA30
:103FA000BA45079BEED1D5E7012ED3D0636B02460D
:103FB000D3F810B0206B0B9B3946D847CAE700BF37
:103FC0008B120608A1120608A5120608AD120608F3
:103FD000BB120608C7120608CB120608D71206083D
:103FE000E9120608014AFFF7C3BE00BFF412060833
:103FF0000B79092B70B50CBF058B458B4FF6FF7302
:104000009D42044602D1064AFFF7B2FEA18BE28B25
:10401000E36AA06A9B6F8A1A2946BDE87040184778
:10402000F110060838B50546A9B101F00F03022BBF
:104030000DD10C09204608F09EFD002806DA224624
:10404000064907480BF0FEF9A860002038BD054A74
:10405000FFF78EFEF9E70846F8E700BF45130608AC
:10406000A82906084A1306082DE9F8430546406AC0
:104070001746028B12F0020C0E4606D0324A314629
:104080002846BDE8F843FFF773BE01F00F0102298F
:1040900017D1AC79310984B1C38B0133C383644632
:1040A0004FF0010800294DD00022FFF723FC0378D0
:1040B0008146002B31D0254AE1E7838B013383838E
:1040C000EEE73179B942344608D1B168AB790909D4
:1040D000002BF2D0C38B0133C383E1E7994214D1A3
:1040E000AC79002CCAD10123AB71B16851B301F096
:1040F0000F03022B18BF0C4642F0040218BFA16840
:10410000028309094FF00308CCE7B16842F00202CC
:10411000090902834FF00508C4E70323037080F800
:1041200001806B6A5B8B032B0CD1482F0AD14CB1F9
:10413000E1682846FFF776FF99F8013043EA00105E
:1041400089F80100BDE8F883990B0608811206087A
:104150004F234E22FFF788BF49234822FFF784BF31
:1041600010B44279446A012A0B4604D120465DF816
:10417000044BFFF7BFBBC16A806A224614315DF869
:10418000044B02F031BC10B44479426A012C0B4656
:1041900004D110465DF8044B02F018BCC16A5DF80A
:1041A000044B806A1C3102F01FBC436A10B55A8B65
:1041B0000446FFF738FD01462046BDE81040FFF7F2
:1041C000E2BF00002DE9F3418D6805F00F030E2BCF
:1041D00004460E4606D0002D30D0AB072ED12B79E9
:1041E000652B1ED10095002501AA65216846FFF7C1
:1041F00045F9019B002103EB800040F2BE5298423A
:1042000015D1F26840F20E439A4235D1636A1F78A5
:10421000B7B1394A31462046FFF7AAFD02B0BDE8E2
:10422000F081622B0AD1AB680093ED68DCE753F8AC
:10423000047B97420CBF01310331E0E70021E0E746
:10424000E36AA06A9B6B9847E36AA06ADB6B05216F
:104250009847E36AA06AD3F8A0303A46012198470C
:1042600001AA29462046FFF7F3FCE36AA06A1B6B0C
:10427000022239469847D1E7E36AA06A9B6B9847C8
:1042800006F10C006A466A21FFF7F8F80026074697
:10429000BE42D4E90A0311D1D3F8A030002231463E
:1042A0009847294601AA2046FFF7D2FC0025AE42D6
:1042B000D4E90A030BD11B6E9847AFE7009ADB6B7A
:1042C00052F826209168090998470136E0E7009ADC
:1042D0001B6B52F82580D8F808703F093946012237
:1042E0009847D8F80C1029B939462046FFF74BFFFC
:1042F0000135DCE70909F8E763120608C36A37B538
:1043000004460D469B6B806A00219847E36AA06AC9
:104310005B6B0E21984701AA29462046FFF798FCBF
:1043200001992046FFF72FFF03B030BD10B4447948
:10433000426A012C0B4604D110465DF8044B02F092
:1043400045BBC16A5DF8044B806A243102F04CBB66
:1043500037B504460D46B1B1CA0705D5C36A9B6B94
:104360004910A06A98470EE08B0731D001F00F0585
:10437000062D4FEA111308D00A2D0CD0022D1FD1A3
:104380001946FFF7EDFE03B030BDC26A806AD26BFA
:1043900019469047F7E74279042A03D0C36A0621F9
:1043A0001B6CDEE701A91846FCF7B3FDE36A01992F
:1043B000A46A1D6C0EF08EFC01462046A847E2E779
:1043C000042BE0D0C26A806A526BD9B29047DAE718
:1043D000C36A09681B69806A98472A79024B294693
:1043E00053F822302046BDE7401106082DE9F14F71
:1043F0000D46A9070446164612D005F00F03022BFE
:1044000017D129090AB1022A05D1204601B0BDE819
:10441000F04FFFF7B8BE01B0BDE8F04FFFF7A0BE08
:104420006968CBB22D2B7BD00BD8062B0DD02C2B53
:1044300012D0554A2946204601B0BDE8F04FFFF79B
:1044400097BC2E2B7DD09D2BF3D1002EF1D105F101
:1044500008030A0A002187E0022A02D0A968FFF7B0
:1044600077FFEF68002FE4D017F00309E1D17B68F4
:10447000DAB28E2AB8460DD1022E4FEA132805D0A3
:1044800007F1080A08F1FF3BD94511DB08F10108E3
:1044900057F8288098F80430312B24D1022E0FD100
:1044A000E36AA06A9B6E9847E36A1B6D012115E0E1
:1044B0005AF8041B2046FFF74BFF09F10109E3E717
:1044C000D8F808102046FFF743FF012EE36AECD12D
:1044D000DB6DA06A9847E36A1B6D0021A06A01B0FA
:1044E000BDE8F04F1847322BA3D1012ED4E90A03BF
:1044F0000CD19B6D9847E36AD8F808105B6D0022D9
:10450000A06A090901B0BDE8F04F1847022E01D199
:104510005B6E9847E36AD8F808105B6D0122EFE7FD
:10452000A868002885D0002A83D1C16839B311F06A
:10453000030324D14A68D6B2952E17D11A46816852
:1045400012E0002A7FF475AFA96829B90B4601B0C3
:10455000BDE8F04F00F01AB88B0703D10B79922B0E
:104560000846E2D000231A462046F0E7962E03D1F3
:1045700001F10803120AE2E7AC2E3FF45AAF00F152
:104580000803022266E700BF9B1006082DE9F84FDA
:104590000F1E05469246994614BF4FF001084FF092
:1045A00000081DD017F003041AD13B79222B17D134
:1045B000C36A806AD3F8B0302146984700260AF1D2
:1045C000FF3B56450FD1631C29D1EB6AA86AD3F88B
:1045D000AC3006EB080198474FB30022394623E080
:1045E0004FF0FF34EAE759F8261081B18A070ED15F
:1045F0000B79222B0BD101340BD1EB6AA86AD3F8CB
:10460000B03006EB0804ABEB0602214698470136B2
:10461000D7E728460F4ABDE8F84FFFF7A9BB37B1E7
:10462000002CDAD1B96822462846FFF7DFFE0027C2
:10463000BE4201D1BDE8F88F59F8271007EB0803F7
:10464000A3424FF0000208BF89682846FFF7CEFE5C
:104650000137EDE7A61006082DE9F74F04460D4691
:1046600016461F462846FEF7E9FC20B1D6B9E36A94
:104670003946DB6E4DE02846FEF7EEFC10B1002E09
:10468000F5D10FE0002D55D0AB0753D16B684FEA41
:10469000132ADBB21E2B1AD1EEB1083505EB8A0ABC
:1046A00055450CD103B0BDE8F08F5B46019A59F82F
:1046B000041B2046FFF7D0FF08F101081AE03B4633
:1046C000324655F8041B2046FFF7C6FFE8E71F2BCC
:1046D00024D1002EE1D0D4F810B00BF101032361F6
:1046E0000AF1FF33009386F0010305F108094FF04A
:1046F00000080193009B4345D7DC0AF101013B46CA
:1047000055F8211032462046FFF7A6FFE36ADB6A20
:104710005946A06A03B0BDE8F04F1847202B03D1DB
:1047200086F00106AD689DE72D2B03D1AB68002B09
:10473000A5D19BE729462046FFF70AFEE36AA06A57
:104740001B6F3A46314603B0BDE8F04F18472DE9DC
:10475000F04706691F46B31C0361C36A04460D4651
:10476000DB6A806A314691469847E36AA06AD3F8CB
:104770008C3006F1010841469847A968002220467E
:10478000FFF734FE2D69002D2DD149462046FFF755
:10479000DFFD636A1978E36A06291DD1D3F8CC30AE
:1047A000A06A2946984720460121FFF7F2F8E36AFC
:1047B000A06A1B6E9847E36AA06ADB6E3146984791
:1047C000E36AA06ADB6A41469847E36AA06AD3F8C5
:1047D0009030BDE8F0471847BA00D3F8A830A06A77
:1047E00005329847E7E72B79AD2B07D1A968334607
:1047F00000222046FFF730FFED68C4E7E968204655
:10480000FFF7A6FDE36AA06AD3F888300121984734
:104810007B1C4A4629462046FFF799FFCBE700005C
:104820002DE9F04104460E466271C36A46620025D6
:10483000114605611B68806A32469847062120466A
:10484000FFF7A7F86779012F08BF7562F5686DB1AA
:10485000AA070BD12B793F2B08D1A968FFF778FD68
:10486000E36AA06AD3F8C43098472CE033784BB998
:1048700029462046FFF76CFDE36A5B6BA06A0E21B8
:104880009847EDE7072B24D1012F12D10023A37104
:1048900046225F4BE9682046FFF7A3F8738B032B92
:1048A00007D129692046FFF7BDFB338B43EA80100F
:1048B000308320466969FFF74BFDE36AA06A9B6875
:1048C00098470028D8D0E36AA06A5B68BDE8F04149
:1048D0001847022B1BD1E36A29681B69A06A984715
:1048E0006379012B07D10023A3714C22494BA9689E
:1048F0002046FFF776F8E9682046FFF729FD338B5D
:10490000DB07ADD5E36AA06A1B6E9847B4E7033BAB
:10491000032B4FD8012FD5F80C8005D1032239463F
:10492000606AFEF7E7FFB783E36A29681B69A06A3C
:1049300098473378032B24D1E36AD3F8A0300122BF
:104940000021A06A98473378062B28D1E36AA06A31
:104950005B6C984701212046FFF702FCE36AA06ADE
:104960005B6C9847E36AA06A5B6C98470023AA686F
:1049700041462046FFF7EBFE3378062B3FF47CAF31
:104980006EE7042B04D1E36A0222D3F8A030D7E704
:10499000052BD8D1E36A0322D3F8A030D0E7204614
:1049A0000121FFF7DDFBE36AA06AD3F8883001211B
:1049B0009847DBE7012F04D103220A213046FEF796
:1049C00099FF17212046FFF7CBFB16212046FFF762
:1049D000DAFBA968E36AA06ADB6B090998471A2128
:1049E0002046FFF7D0FB29692046FFF7B1FC0A21DA
:1049F0003046FEF76FFF0378032BE36A3FF43DAFC9
:104A00005D694288A06A00230A21A84728E700BF01
:104A1000594102085141020838B5436A1B78072BF7
:104A200004460A4606D0022B04D0154ABDE8384099
:104A3000FFF79EB9956885B9E36AA06A5B6B0E21A2
:104A40009847E36AA06AD3F8CC3000219847204603
:104A50000121BDE83840FEF79CBFAB070BD12B7995
:104A6000AF2B08D12046A968FFF772FC2046BDE8AD
:104A70003840FFF775B829462046FFF769FCE0E7A4
:104A80005113060801F00F03022B70B504460E46C1
:104A9000154602D00B4AFFF76BF929462046FFF76F
:104AA00057FCE36AA06A9B6D9847656A2B78033BC5
:104AB000032B9CBF6B68636231092046FFF763FBE1
:104AC000656270BD9B100608D1E90212FFF7DABFDC
:104AD00070B54379CD68012B0446164606D1436A6A
:104AE0000A465B8B3146FFF774F8686100231A466B
:104AF00069692046FEF793FFE9682046FFF728FC26
:104B0000062E05D1E36AA06AD3F8883000219847C1
:104B1000E36AA06AD3F8BC500023AC461A460121D0
:104B2000BDE87040604700002DE9F04F87B0CDE947
:104B30000221044605AAA42103A81F46FEF79EFCF5
:104B40004FF0000B0190D946DA465E46D846019BED
:104B50009B451AD16EB1BAF1000F74D1E36AA06A15
:104B60005B6C9847B9F1000F73D1E36AA06A5B6C84
:104B70009847029AD4E90A03002A70D0D3F8C040BB
:104B8000334642463946A04710E0059A52F82B506A
:104B9000002D49D0A80747D12A79A62A0FD1F107BD
:104BA00007D5304A29462046FFF7E2F807B0BDE8AE
:104BB000F08F46F00106AA460BF1010BC7E7A72AC2
:104BC00007D1B20701D5284AECE746F00206A9460C
:104BD000F2E7A82A28D1EA686AB193070BD11179C4
:104BE000AA2906D19268A9682046FFF74BFF013732
:104BF000E2E7AC2912D0A96801F00F02022A01D025
:104C00001A4ACFE7E26AA06AD26B09099047E968BD
:104C10002046FFF79DFB08F10108CDE70622294653
:104C20002046FFF755FFE2E70EB1114ABAE7B8F1A7
:104C3000000F01D00F4AB5E729462046FFF788FB51
:104C400001374646B8E7DAF808102046FFF780FB40
:104C500088E7D9F808102046FFF77AFB89E7D3F8F0
:104C6000BC408DE701130608081306081013060858
:104C70001D1306082613060870B50D464179012953
:104C80000446134603D12A46FEF7A3FF6861E36A90
:104C9000A06ADB6C98476E6900231A4631462046AD
:104CA000FEF7BDFEE36AF18ADB6BA06A9847E9680C
:104CB00029B18B0703D10B79A32B08BF0021204614
:104CC00002230022FFF730FFF08A70BD436A10B55F
:104CD0005A8B0446FFF7D0FF01462046BDE810403E
:104CE000FFF751BA00231A468968FFF71DBF38B590
:104CF0000C460546C968FFF72BFBA1682846BDE8AE
:104D00003840FFF725BB0B79342B70B504460D46B0
:104D100010D18968FFF71CFBED68AD6885B9E36ABF
:104D2000A06A5B6B0E219847E36A0422D3F8A03097
:104D300002211AE0C36A806A5B6B0E219847ECE798
:104D4000AB071FD12B799A2B13D1E36AA06A5B6B57
:104D50000E219847A9680029E6D02046FFF7F8FA07
:104D6000E36AD3F8A03004220321A06ABDE87040B2
:104D700018479B2B06D1A9682046FFF7E9FAEB6894
:104D80009968E8E729462046FFF7E2FACCE710B534
:104D900004468968FFF7DCFAE36AA06A1B6D00210C
:104DA000BDE81040184700002DE9F7438D68044620
:104DB000164645B9F2B1C36AD3F8A030022229469B
:104DC000A06A984716E0AB0740F085802B79372B17
:104DD00013D132B1C36A806AD3F8A0300222012114
:104DE000984720462946FFF7B3FAE36AA06AD3F84A
:104DF000A430984703B0BDE8F0839F2B6BD1EB68DC
:104E00001A79A12A57D1A22101AA03F10800FEF7BD
:104E100035FBA968804619B38F0721D10B79372B51
:104E20001ED136B1E36A411CD3F8A030A06A022239
:104E30009847A9682046FFF78BFAE36AA06AD3F87F
:104E4000A43098474FF00109002747450ED1B9F12A
:104E5000000FCFD1E36A0322D3F8A030791CAFE76B
:104E60002046FFF775FA4FF00009EDE7019B53F874
:104E7000271099B18E0711D10E79A6F1370046425D
:104E800046412046FFF764FAB9F1000F0FD03EB952
:104E9000164A29462046FEF76BFFABE70026F0E7EF
:104EA000E36AA06AD3F8A43098470137CDE7002E13
:104EB000FBD00F4AEDE7AB684BB19A0707D11B79DE
:104EC000372B04D104222946FFF702FE92E7052280
:104ED00029462046F8E729462046FFF739FAE36AD3
:104EE0000322D3F8A03001216AE700BFB7100608FB
:104EF000C81006080122FFF757BF2DE9F041074609
:104F000015460C4611B1FFF723FA01243DB16E6836
:104F10004FF00008360A0835B04509DB3444FB6A17
:104F2000B86AD3F8A03021460022BDE8F041184706
:104F300055F8041B3846FFF70BFA08F10108EBE7B8
:104F40000A460021FFF7D9BF2DE9F8430C468968CE
:104F50000546FFF7FDF9E668002E4BD07768696AD1
:104F6000FBB209788E2BA36819BF04F10C06012748
:104F70003F0A0836072903F00F024BD1022A3ED11F
:104F80001A099A2A48D132681179302944D1926895
:104F9000002A41D10A212846FFF7E2F86A6AD36A5B
:104FA000528D32B93168414A2846BDE8F843FEF7D0
:104FB000DFBE5978C9071FD559682846FFF7D0F8D2
:104FC000022FEB6A1DD97268A86A1179322918D1AB
:104FD000B4682179302914D191689B6C01220909A8
:104FE0009847A168002301222846FFF79DFD03246E
:104FF000A74232D8BDE8F883013A0833D1E700244C
:10500000F6E7D3F8BC40A86A00231A460221A0475D
:105010000124EDE7022AF2D140F2ED22B2EB131F98
:10502000EDD133681A79302AE9D19B68002BE6D09C
:1050300013F00304E3D11B792F2BD9D1EB6AA86AB3
:10504000D3F8BC80224623462146C0473368224617
:1050500099682846FFF7A8FEDAE704F10108B84589
:105060004FEA840356F824101AD20A79322A17D14B
:105070003344D3F8049099F80430302B10D1896868
:10508000EB6AA86A9B6C0022090998470023012259
:10509000D9F808102846FFF747FD08F10104A7E7F3
:1050A0002846FFF755F9A046F7E700BFDE100608CF
:1050B00070B50D46C9680446FFF74AF9A968E36A66
:1050C000A06AD3F89830C1F3071132291ABF3E39CC
:1050D000C9B20221BDE870401847F8B54E680C46C9
:1050E00089680746FFF734F9360A0C340025023583
:1050F000AE4204F1080400DCF8BD54F8041C384644
:10510000FFF726F954F8081CFB6AB86AD3F89C30FC
:1051100009092339C9B29847E9E72DE9F0414D68FB
:105120000C4689688046FFF713F9A5F10D07FFB219
:105130002D0A0C340126AE4201DBBDE8F08154F8A3
:10514000041B4046FFF704F9D8F82C30D8F82800A3
:10515000D3F89C30394698470136ECE72DE9F04109
:105160004D68044688462D0A8968FFF7F1F8032D3B
:1051700083BF27697B1C236100270126731CAB4278
:1051800022DB032D57DD2569A06A6B1C2361E36ACE
:105190002946DB6E9847E36AA06ADB6A394698477E
:1051A000E36AA06ADB6801219847E36AA06A5B6E44
:1051B0009847E36AA06A1B6E9847E36AA06ADB6AB5
:1051C0002946BDE8F041184708EB86032046D96818
:1051D0000236FFF7BDF8AE4207DAE36AA06A9B6DBC
:1051E0009847E36AA06A9B6E984758F82610E36ACE
:1051F000A06AD3F89C3001F00F020E2A10D1C1F33F
:10520000071124291ABF3339C9B206219847AE4283
:10521000B4DAE36AA06A5B6F3A4600219847ADE7CB
:105220000A79852A01D13221F0E78A680AB9072173
:10523000ECE73321EAE7BDE8F08110B50446896860
:10524000FFF786F8E36AA06AD3F898300321BDE837
:10525000104018472DE9F0474D68D0F810805FFAEC
:1052600085F9A9F11E03D3F1000949EB030908F1FF
:105270000103044603612D0A01F108060027AF422D
:1052800006DBE36AA06ADB6A4146BDE8F0471847DF
:1052900056F8041B20460137FFF75AF8AF42EEDA02
:1052A000E36AA06A5B6F424649469847E7E7000019
:1052B00001F00F03022B70B5044610D00B79492B77
:1052C00001D04F2B02D10123A37170BD4A2BFCD01A
:1052D000502BFAD0482B0CBF0D69CD685DB9A3796E
:1052E000002BF2D1E38A002BEFD020461B4ABDE809
:1052F0007040FEF73DBD837943B3838A8E680133E6
:105300009BB2012B83820ED1C18AD0E90A03D1B1AD
:10531000D3F8A03000229847E36AA06AD3F8A030FF
:1053200002220021984729462046FFF711F8E36A38
:10533000A06ADB6B31099847E36AA06AD3F8A4300E
:10534000BDE8704018475B6C9847E5E7C38A0133B6
:105350002946C382BDE87040FEF7FABF2211060855
:105360002DE9F0410569CF68AB1C0361884604460E
:1053700000222B46B968FFF76FF9D8F808102046CD
:10538000FEF7E6FFE36AA06ADB6E6E1C31469847C3
:10539000E36AA06ADB6A29469847E36AA06ADB6889
:1053A0004FF0FF319847F9682046FEF7D1FFE36AD6
:1053B000A06ADB6A3146BDE8F04118472DE9F047A5
:1053C0000446904699460F4621B91946BDE8F04774
:1053D000FEF7BEBF0669731C036115683DB315F087
:1053E000030A24D12B797B2B21D1A968FEF7B0FFCA
:1053F000524631462046FEF7D4FA5246E968204626
:10540000FEF7F4FF08F104024B46791E2046FFF731
:10541000D5FFE36AA06AD3F880303146984720462A
:105420000321FEF7B6FABDE8F047FEF7CABA2946EF
:105430002046FEF78DFF204600223146FEF7B1FAE6
:10544000E36AA06A1B6E9847DCE737B50C46054651
:1054500001AA7A2104F10800FEF710F8E368019A26
:1054600001462846FFF7AAFF03B030BD2DE9F04FF3
:1054700085B006691D460E9B0393731C0293B31CF3
:10548000044603610F46934631460122FEF789FA2E
:1054900039462046FEF75CFFE36AA06AD3F89430F1
:1054A0000022711C9847E36AA06ADB6A314698477C
:1054B000E36AA06AD3F8D0309847D4F8108008F196
:1054C0000103236100265E4518DB2046FEF779FACA
:1054D000E36AA06AD3F8D4309847E36A0299DB6A9A
:1054E000A06A984703992046FEF732FFE36AA06A54
:1054F000DB6A414605B0BDE8F04F18472B46D4F8AB
:1055000010901A68019209F101022261019A9768CC
:1055100004350136002F47D1B3453AD1E36AA06A7A
:105520001B6E98474FF0000A5746019B2046D968EA
:10553000FEF70EFFBAF1000F19D0E26AA06A526BB3
:105540000E219047E26AA06AD26A39469047E26A21
:10555000A06A526B0E21904751462046FEF713FE7B
:1055600020465146FEF7E2FE2046FEF72AFAE36A9D
:10557000A06AD3F89430012241469847E36AA06AB2
:10558000DB6A49469847E36AA06ADB6801219847CD
:1055900099E720461E4A1968FEF7EAFB204605B047
:1055A000BDE8F04FFEF70DBA17F003032BD13979A0
:1055B00076293A462AD1D368BF684FEA131AE26ABD
:1055C000A06A926D904739462046FEF7C1FEE26A16
:1055D000A06AD2F89C2008219047E26AA06A176F5F
:1055E00000214A46B847BAF1000F97D051462046ED
:1055F000FEF7C9FD27697A1C22613946022220463E
:10560000FEF7CFF991E74FF0000AD8E79A46D6E7C0
:105610002D1306082DE9F347056999466B1C1746BB
:105620000E460361022229460446DDE90AA8FEF778
:10563000B8F917BBE36AA06ADB68032198473146D3
:105640002046FEF785FEE36AA06ADB686FF0020180
:105650009847E36AA06A5B6B0E219847E36AA06AE9
:10566000DB6A2946984720464146FEF771FE2046F0
:1056700002B0BDE8F047FEF7A4B9CDF800A04B4654
:105680003A4631462046FFF7F1FEE2E77FB5CD68A6
:105690002B79782B06460C4609D1AB680193002381
:1056A000009389681A46FFF7B5FF04B070BD742BEC
:1056B00003AA4FF0770116D105F10800FDF7DEFED1
:1056C0002B6902463BB9EB680093039BA168304607
:1056D000FFF7CCFEE9E79B680193EB680093A168B4
:1056E000039B3046DFE704F10C00FDF7C7FE002303
:1056F00000930246039BE9E72DE9F04F8B6803F026
:105700000F03022B8BB004460D4640F00981CB6895
:10571000002B00F00581980740F002811A792C2AAD
:1057200040F0FE809A6802F00F01022940F0F880F4
:1057300012097C2A40F0F480DB681A79302A40F0A4
:10574000EF809B68089309AAA42108A8FDF796FE9C
:10575000431E022B00F2E480099901280A680DD04B
:105760000228D1F8049000F02C818E68F10740F1F6
:10577000D780730800F0D48052B102E0914603262E
:105780000246930704D11179A639022940F2C88054
:10579000B9F1000F08D019F0030F05D199F80410E2
:1057A000A639022940F2BC80AB6801932B690293B1
:1057B000238B6F6903932569638B0493E38BA18B20
:1057C00005936B1C0693E183291DBDF818302161F8
:1057D0006FEA0901638319F0010801F0010305F183
:1057E000020A258305F1030B069305D1494620469D
:1057F0000792FEF7ADFD079A11462046FEF7A8FD79
:10580000E26AA06AD26E59469047E26AA06AD26AFA
:1058100051469047E26AA06A926D90470022019932
:105820002046FEF7E3FD02992046FEF791FDE26A6D
:10583000A06AD26A691C904731462046FEF788FD6F
:10584000E26AA06AD2F89C200E219047E26AA06A20
:10585000D26A59469047E26AB8F1000F56D1D36D2B
:10586000A06A9847E36AA06A5B6E9847E36AA06AF9
:10587000D3F89C30002EACBF002101219847E36A89
:10588000A06A1B6F524601219847BDF80C30238354
:10589000BDF810306383BDF81430E383002F3DD092
:1058A000E36AA06A1B6E9847B8F1000F03D1E36A60
:1058B000A06A1B6E984739462046FEF749FD2669C7
:1058C000A06A731C2361E36A3146DB6E9847E36A82
:1058D0000699DB68A06A01319847E36AA06ADB6A2F
:1058E00029469847E36AA06A1B6E9847B8F1000FF3
:1058F00003D1E36AA06A1B6E984727B1E36AA06AE6
:10590000DB6A314698470BB0BDE8F08FA06A926D14
:10591000904749462046FEF71BFDA7E73E46DCE7D9
:105920002669A38BB4F81E90E3836FEA46436FEABF
:105930005343B4F818B02383F31C2361771CB4F8E5
:105940001AA0E96867832046FEF702FDE36AA06AB1
:10595000D3F8883001219847E36AA06ADB6A3946A8
:105960009847E36AA06AD3F88C3006F102084146F2
:1059700098470022A9682046FEF738FD204629698D
:10598000FEF7E6FCE36AA06A9B68984720B9E36AE1
:10599000A06ADB6E39469847E36AA06ADB6A414633
:1059A0009847E36AA06AD3F890309847A4F818B0F3
:1059B000A4F81AA0A4F81E9069692046FEF7C8FC56
:1059C0009CE70326D8E62DE9F14F0669B0F818B038
:1059D000B0F81AA0B0F81E900683B31C036106F15C
:1059E0000108838BA0F81A800446C38388680D469B
:1059F000FDF724FBF8B927697B1C2361A868FDF734
:105A00002BFB20B9E36AA06ADB6E41469847E36A44
:105A1000A06ADB6A39469847E9682046FEF798FC99
:105A2000E36AA06ADB6A414698473B460122A968BF
:105A30002046FEF711FE2969A4F818B02046A4F804
:105A40001AA0A4F81E90FEF783FCE36AA06ADB6A42
:105A5000314601B0BDE8F04F18472DE9F34706691C
:105A6000731C0361044688680D46FDF7E7FA024699
:105A700010BB27697B1C2361A9683B462046FEF7C3
:105A8000EBFD2046E968FEF763FCA868FDF7E4FA41
:105A900000BB2B690BB96B694BB1E36AA06A9B68C9
:105AA000984720B9E36AA06ADB6E31469847E36AFB
:105AB000A06ADB6A3946984701AA712105F11000F6
:105AC000FDF7DCFC0027824657450BD1696920466B
:105AD000FEF73EFCE36AA06ADB6A3146984702B0F3
:105AE000BDE8F087019B53F82780D8F80800FDF740
:105AF000A5FA024620BBD4F8109009F101032361F6
:105B0000D8F808104B462046FEF7A6FD2046D8F8E8
:105B10000C10FEF71DFCD8F80800FDF79DFA0028D0
:105B2000D8D1E36AA06A9B68984720B9E36AA06A63
:105B3000DB6E31469847E36AA06ADB6A49469847BC
:105B40000137C1E72DE9F74F044692469B46894647
:105B500029B9194603B0BDE8F04FFEF7F9BB056956
:105B60002B1D036113686F1C05F10208EE1C002B4E
:105B700000F0F28013F0030240F0EE8019797B29E7
:105B800040F0EA80996801920093FEF7E1FBE16A38
:105B9000A06A896D8847A8212046FDF7FAFFDDE954
:105BA00000322046D968FEF721FC02222946204611
:105BB000FDF7F7FEE36AA06ADB68032198470AF164
:105BC00004025B4609F1FF312046FFF7BBFFE36AA1
:105BD000A06ADB686FF002019847E36AA06A5B6B1A
:105BE0000E219847E36AA06A5B6E9847E36AA06A51
:105BF000DB6E39469847E36AA06ADB6A2946984714
:105C0000E36AA06A9B6D9847E36AA06A9B690122D8
:105C100021219847E36AA06AD3F89C30082198476D
:105C2000E36AA06A1B6F424600219847E36AA06AB4
:105C30009B6D9847E36AA06A9B6E9847E36AA06AE7
:105C40005B6E9847E36AA06A9B6C0022A921984783
:105C5000E36AA06A9B6E9847E36AA06A9B6E9847C6
:105C6000E36AA06A9B6D9847E36AA06A5B6D0022B5
:105C70000A219847E36AA06A5B6E9847E36AA06AC4
:105C80005B6B0E219847E36AA06AD3F8C0500023EB
:105C90001A460321A8472046FDF762FFE36AA06A7F
:105CA0001B6F324600219847E36AA06A1B6E984733
:105CB000E36AA06A5B6B0E219847E36AA06ADB6E19
:105CC00031469847E36AA06ADB6802219847E36A95
:105CD000A06ADB6A41469847E36AA06A9B6E9847D0
:105CE000E36AA06A9B6E9847E36AA06ADB6A39465A
:105CF0009847E36AA06A9B6C0022A9219847E36A4F
:105D0000A06A5B6B0E219847E36AA06A9B6D984777
:105D1000E36AA06A9B6D9847E36AA06AD3F8C05013
:105D200000231A460321A8472046FDF719FFE36A1E
:105D3000A06A1B6E9847E36AA06ADB684FF0FF31E8
:105D40009847E36AA06ADB6A31469847204603B069
:105D5000BDE8F04FFDF735BE19462046FEF7F8FACC
:105D6000E36AA06A9B6D98472046A821FDF711FFC2
:105D7000E36AA06A1B6E984717E72DE9F04F8D681C
:105D80002B79032B87B004460AD12946FEF70DFA7A
:105D9000AA69138B43F00103138307B0BDE8F08FAA
:105DA000162B40F0B5800669EB684FEA1318331DD7
:105DB0000361E968FEF7CCFAE36AA06A9B6C0022F3
:105DC000AA219847E36AA06AD3F8C07000231A4654
:105DD0001946B84741462046FEF7D5F92769238B77
:105DE0000093BA1C638B2261A28B0193E38BE28345
:105DF000E26A02937B1C6383194606F1010BA06AD9
:105E00002783D26A03939047012259462046FDF723
:105E1000C8FD41462046FEF7A3F92046AC21FDF718
:105E2000B8FEA96820460022FEF7E0FAE26AA06AFE
:105E3000D2F8948006F1020949460022C047E26A7E
:105E4000A06AD26A59469047E26AA06AD2F8D02086
:105E50009047E26AA06A926D9047E26AA06AD2F81F
:105E6000188040F20F310122C047E26AA06AD2F8DE
:105E70009C2008219047E26AA06AD2F8708006F15F
:105E8000030A52460021C047E26AA06A126E904798
:105E9000E26AA06AD2F8948031460122C047E26AE1
:105EA000A06AD26A51469047E26AA06AD26801218C
:105EB00090472046FDF785FDE26AA06AD2F8D4201B
:105EC0009047E26AA06AD26A49469047296920460B
:105ED000FEF73EFA039BE26AA06AD26E194690472B
:105EE000BDF800302383BDF804306383BDF808306B
:105EF000E383E36AA06ADB6A314698476969204612
:105F0000FEF726FAE36AA06ADB6A3946984744E757
:105F100005AA7A2105F10800FDF7B0FAEB68059AA9
:105F200001462046FFF70EFE37E770B58D68044640
:105F30003DB9C36AD3F8C8302946A06ABDE87040AD
:105F40001847AB070ED12B795E2B0BD1A968FEF752
:105F5000FFF9E9682046FEF7FBF9E36A0221D3F86E
:105F6000C830EAE729462046FEF7F2F9E36A012144
:105F7000D3F8C830E1E710B504468968FEF7E8F9C0
:105F8000E36AA06A1B6EBDE8104018472DE9F04790
:105F900005460C4604F00F03022B05D121092846C3
:105FA000BDE8F047FEF7C2B9002C68D0A20766D161
:105FB00023792C2B39D1A1682846FEF7C9F9E66868
:105FC000002E5CD016F0030859D17768FAB28E2AF9
:105FD000334609D13F0A06F1080907F1FF3AC245E5
:105FE00010DC013756F827301A79312A12D1996816
:105FF0002846FEF7ADF9EB6AA86A1B6D0221BDE8E1
:10600000F047184759F8041B2846FEF7A1F908F194
:106010000108E4E7322A32D19968EB6AA86A5B6D1D
:1060200002220909BDE8F04718472D2B27D1A468A3
:106030002CB3E668EEB1B3071BD17768FAB2952AA4
:1060400001D1A468A6E7962A11D1A1682846FFF7D6
:106050009DFF3F0A08360024BC4201DBBDE8F08703
:1060600056F8041B2846FFF791FF0134F4E7AC2AE9
:1060700005D0A1682846FFF789FFE4688AE7214632
:106080002846024ABDE8F047FDF772BEAD1006088B
:106090002DE9F041CD6804460E4635BB0379BBB10E
:1060A000436A1D78A5B9CE21FEF75AF8B16820469B
:1060B000FEF74EF9E36AA06AD3F8BC602A462B4685
:1060C0000121B047E36AA06A1B6EBDE8F0411847A2
:1060D000B168880700F0BB8001F00F03022B40F08D
:1060E000BD802046FEF734F9ECE7AA0740F0B880FF
:1060F0006B68DAB25B2A14D1ED68002D40F0B080F5
:10610000406A0378072B40F0A980896801F00F03EB
:10611000022B40F0A38003220909BDE8F041FDF7FE
:10612000E9BB562A13D101228968FEF75FF9E968B5
:106130002046FEF70DF9A968E36AA06AD3F89C30FF
:1061400009093D39C9B298470222B1687AE0572A55
:1061500040F086801B0A5F1E013355F82310FEF7BE
:10616000F7F8002F03DDE36AA06A9B6D9847B168DA
:1061700000222046FEF73AF908350026BE426DDAC5
:106180000136BE4203DAE36AA06A9B6D984700229B
:1061900055F8041B2046FEF729F9EFE76A68D3B2E9
:1061A000062B5FD1B768002F5CD0BB075AD17B6844
:1061B000D9B2062956D14FEA1228B8EB132F51D184
:1061C000A8F10203012B4DD8BB6823B1980702D177
:1061D0001B79222B46D0FB6823B1990702D11B798A
:1061E000222B3FD0B8F1020F06D03B6923B19A07AA
:1061F00002D11B79222B35D0A9682046FEF7A8F8DA
:10620000E9682046FEF7A4F8B8F1030F07D120464D
:106210002969FEF79DF8E36AA06A9B6E9847E36AD6
:10622000A06A5B6E98470022B9682046FEF7DEF848
:106230000022F9682046FEF7D9F8B8F1030F0DD116
:10624000396900222046BDE8F041FEF7CFB80029A9
:106250003FF447AF0B793A2B7FF443AFBDE8F081B1
:10626000AB079BD029462046FEF772F800226CE768
:106270002DE9F04F044685B08A4602AA42210AF170
:106280000800FDF7FBF8636A019000255E8BA846C5
:10629000019B9D420AD1DAF80C100B79032B4ED1E9
:1062A00032462046FDF7BFFC064656E0029B53F8F7
:1062B00025B003AA6C210BF10800FDF7DFF8039B62
:1062C00019680A09732A81460CD02046FEF740F867
:1062D00001274F4528D3DBF80C1059B12046FEF7B3
:1062E00037F807E0022807D0294A2046FDF740FD8D
:1062F00008F101080135CBE759680B09412B0DD096
:1063000040F2434293420BD040F22352934209D0D1
:1063100040F246329342E7D10426E9E70126E7E757
:106320000646E5E70326E3E7039BA06A53F8271038
:10633000E36A00225B6D090998470137C9E7442BDE
:1063400017D18F68324639462046FDF76CFCBA6992
:10635000138B43F00103064613830027A5EB0805C2
:10636000BD420BD831462046FDF70DFF05B0BDE814
:10637000F08F32462046FEF77FFC95E7E36AA06A7D
:10638000D3F8BC8000231A460121C0470137E7E754
:106390000A1106084B682DE9F04106460F461D0A12
:1063A00001F108080024AC4201DBBDE8F08158F897
:1063B000041B3046FDF7CCFFB36843B1023406F14D
:1063C0000C0057F82410BDE8F041FDF7C9BC0134BA
:1063D000E9E710B50446FFF7DDFFE36AA06AD3F8EA
:1063E0009C302221BDE81040184770B58D680446E6
:1063F00045B9C36AD3F8A03001222946A06ABDE896
:1064000070401847AA0739D12B79922B36D1EE6804
:1064100036B3B30724D13379952B08D1A968FDF79A
:1064200097FFE36A0122D3F8A0301146E6E7962BE6
:106430000ED1A968FDF78CFF31462046FFF7AAFF71
:106440007168E36A090A0122D3F8A0301144D5E744
:10645000AC2B05D129460322BDE87040FEF738BBBE
:10646000A9682046FDF774FFE9682046FDF770FF34
:10647000E36A0122D3F8A0300221BFE72946204673
:10648000CDE7896830B4054619B90A4630BCFEF735
:1064900034BDCB688BB113F003020ED11C79952C5F
:1064A00001D18968F2E7962C01D11A46F9E7AC2CA4
:1064B00003D1062230BCFEF70BBB0A46284600215A
:1064C000E4E70000436A1B78072B10B50A46044630
:1064D00006D0022B04D0074ABDE81040FDF748BCA7
:1064E00020461146FEF730FD2046BDE81040FDF77E
:1064F00037BB00BFD3100608184B2DE9F041D3F885
:10650000E86104460F463EBB05696B1C036101222E
:106510002B468968FEF7A0F8E36AA06A9B691F21F1
:1065200001229847F96851B12046FDF711FFE36A4F
:10653000A06AD3F8BC70324633460121B847E36AFB
:10654000A06AD3F8C83001219847E36AA06ADB6AE1
:106550002946BDE8F0411847BDE8F0812C1B00201A
:10656000426A1278072A2DE9F041044604D01B4AFA
:10657000BDE8F041FDF7FCBB8D685DB9C36A806A78
:106580005B6B0E219847E36AA06AD3F8C430BDE87C
:10659000F041184715F003021DD12B791B2B1AD19E
:1065A0000669EF68731C0361B9683346FEF754F857
:1065B000A9682046FDF7CCFEE36AA06AD3F8C43090
:1065C0009847E36AA06ADB6A31469847F968204633
:1065D000FDF7BEFED7E72946F9E700BF75120608AA
:1065E0002DE9F74F4379012B04460D4608D10F7969
:1065F000102F08D0436A1B782BB9224AFDF7B8FB4D
:1066000003B0BDE8F08F01AA6D2105F10800FCF789
:1066100035FFDFF87CB080460026B045F0D0019B06
:10662000606A53F8261000220909FDF763F9102F5C
:106630008146027815D112F0FD0F05D05A46294641
:106640002046FDF795FB0AE04FF0020A80F800A013
:106650004168606AFDF76FF908B180F800A0013663
:10666000DBE75AB9012202700146606AFDF769F959
:1066700099F80030012BF2D1034AE0E7052AEED069
:10668000024ADCE72C1206084F1206085C120608C4
:10669000421206082DE9F04F91B00D4614460190C4
:1066A0003422002103A819F041FB4FF0FF33089377
:1066B000019AAD4B126893F8EC310295002102A8C3
:1066C0008DF80C40FDF785FA054600F053FEA74B08
:1066D0000A9C0C9080460D93002714B1049E002E56
:1066E0003DD00A9C14B1049B002B58D0394640463B
:1066F00000F043FEDFF874920A9CDFF874A2DFF822
:1067000074B20026049B002C40F039815BB10B9BD6
:1067100005A8D968FDF724FB0B9B059ADB8A029933
:10672000049808F0CBFE404600F02FFE16B130462C
:1067300003F0EEFC0E9808B104F09BFB0198FDF706
:106740008DF82C69AE682846FDF7BAF83546002E5C
:10675000F8D10498002800F03081F9F779FC638BB8
:10676000042B4FF00102214602A807D1FDF714FBCC
:10677000069BA4689F4238BF1F46AEE7FEF750F85D
:10678000638D9E42F4D2E36A03EBC60113F8363000
:10679000012B02D12046FDF7D4F80136F0E7228B19
:1067A00052071CD5608D411EC900C0B1E26A0A447F
:1067B000567816F0020F2DD08BB192E8030093F8B3
:1067C000009093F801E0B3F802C05E6883E803002C
:1067D00082F8009082F801E0A2F802C056604FF003
:1067E000000363840026B4F82AC0664519DB002341
:1067F0009C454DD1D4F804E0BEF1000F08D0002034
:10680000BEF82AB00346584552DB002B40F0898081
:10681000A46867E713B9012E08BF13460138083989
:10682000C3E72378D4F82C904FEAC60B012B09EB71
:106830000B0A05D1DAF804300A2B09D10136D2E768
:1068400019F8363004D9012B04BF022309F80B30A4
:1068500019F80B30022B06D1638B032B11D0238B3D
:1068600043F01003238319F80B30032B03D09AF85D
:106870000130DB07E2D5638C5A1C6284AAF802302F
:10688000DCE7DAF8040006F076F90128EBDCE6E74D
:10689000E26A02EBC30112F83320042A06D14A78D7
:1068A000D6075FBF628C4A800132628401339FE762
:1068B000DEF82C2002EBC00A12F83020043A012A3C
:1068C00015D8002611E0E26A02EBC60912F836205C
:1068D000052A09D1D9F804201146DAF804208A42A1
:1068E00004BFA9F8023001330136B445EBD10130C1
:1068F00089E7E06A00EBC20110F83200052802D1F6
:106900004878C00702D54888184448800132944529
:10691000EFD1A28B9BB21A44A283628C134463848E
:1069200076E70022F3E7023B012B25D82EB93A4641
:1069300006A904A803F0CEFB0646CDE90C6A0222A4
:10694000214602A8FDF76CFF049B23B903222146D0
:1069500002A8FDF765FF049B6BBB0422214602A839
:10696000FDF75EFF27E000BF2C1B00205C1306082C
:106970000015060884160608CDE90C89DFE7002B10
:106980007FF4C5AE638B042BCDD10E9B1BB938466B
:1069900004F05AFA0E9000230322214602A80C9319
:1069A000CDF83CB0FDF7F8F9049B23B90422214649
:1069B00002A8FDF7F1F9A468A4E632463146204664
:1069C00004F0C8FA11B0BDE8F08F00BF10B504465E
:1069D0000122FCF78FFF2378012B04D90378012BC8
:1069E00004BF0323037010BD70B505460E46104664
:1069F00019461C46FCF76EFF0378012B06D173681D
:106A0000002221462846BDE870401847022B02D1DB
:106A100073680122F5E736684288032B2146284631
:106A2000B4460CBF00230123BDE870406047807965
:106A3000003018BF012070470346026A40790328DE
:106A400094BF1846186B114492BF196280181962DE
:106A5000704710B50C460121FFF7EEFF047010BD22
:106A60000346806A5A79032A88BF5A6A01448BBF59
:106A700012181846186B996284BF80189962704783
:106A800010B50C460121FFF7EBFF047010BD4379F0
:106A9000012B09D083681944C36881609A8C9142A4
:106AA000C8BF998400238371704738B51446FFF737
:106AB000EEFF0121FFF7D4FF047038BD53220121FE
:106AC000FFF7F3BF54220121FFF7EFBF5722012147
:106AD000FFF7EBBF58220221FFF7E7BF59224FF023
:106AE000FF31FFF7E2BF5A220021FFF7DEBF5B2232
:106AF0000021FFF7DABF5D224FF0FF31FFF7D5BF6E
:106B000000290DBF5E225F2203210021FFF7CDBFC8
:106B1000A1F13002D2B20021FFF7C7BF62226FF0AD
:106B20000101FFF7C2BF10B5632204464FF0FF31E9
:106B3000FFF7BBFF0123A37110BD01F16402D2B2C4
:106B40004942FFF7B2BF10B501F167020446D2B265
:106B50004942FFF7AAFFE268138B43F00103138356
:106B600010BD70B51C461546FFF791FF0321FFF7D6
:106B700077FF4470240A0570847070BD012A10B438
:106B80000B46044608D0022A0ED169224FF0FF318D
:106B90005DF8044BFFF789BF11461B322046D2B285
:106BA0005DF8044BFFF7DDBF4FF0FF31F5E70B4613
:106BB00010220121FFF7D5BF11320B46D2B20121BD
:106BC000FFF7CFBF10B4002A4FEA42040B4618BFAC
:106BD0001522C4F1010108BF14225DF8044BFFF730
:106BE000C0BF16320B46D2B24FF0FF31FFF7B9BF2C
:106BF00019320B46D2B20021FFF7B3BFF8B51646E3
:106C00001F46FFF744FF4379032B81BF846AC269A3
:106C1000C4F5FF4452F8273088BF7D344FF003019C
:106C20008CBFE4180024FFF71BFF44702412067089
:106C30008470F8BD0B4642220021FFF7DFBFF8B594
:106C400016461F46FFF723FF4379032B81BF846A53
:106C5000C269C4F1FF2404F57F0484BF52F82730D1
:106C6000FD344FF003018CBFE4180024FFF7F8FE59
:106C70004470240A06708470F8BD10B4002A0CBF5A
:106C80000224002447320B46D2B221465DF8044B61
:106C9000FFF7D5BF0B464B220121FFF7D0BF0B46B4
:106CA0004A220021FFF7CBBF6FF00301FFF7EFBED1
:106CB0000421FFF7ECBE6FF00201FFF7E8BE000011
:106CC000254BD3F8E831022B2DE9F04706468A46DA
:106CD0000DD84569A9420AD9846A03694D1BE41A93
:106CE00040F2FF792CB915BBB36AC6E9043ABDE896
:106CF000F087062D01D90F2C1BD91F2CA04628BFC9
:106D00004FF01F08444510D8032D2F4628BF0327F6
:106D100001213046FFF790FE48EA47130370A4EBC9
:106D20000804ED1BDEE7A046EEE70027F0E7062D9E
:106D3000F9D94D452F464FF0020128BF4F46304646
:106D4000FFF77AFE3B0903F0700364F07F02134300
:106D500003704770A046E2E72C1B002038B50D46B3
:106D60000021FFF794FE4379012B05D0032B9EBF32
:106D7000C369826A43F8252038BD70B50D460446C4
:106D800011462AB92B461322BDE87040FFF7E9BE31
:106D9000022A04D1FFF792FE2046FFF7A4FE2B46FD
:106DA00018226FF001012046EEE710B5044631B914
:106DB00055224FF0FF31BDE81040FFF776BE0229A3
:106DC00004D1FFF77BFE2046FFF791FE56226FF0BD
:106DD00002012046EFE7134621B143224FF0FF3175
:106DE000FFF70CBF4422F9E7134621B145224FF0CB
:106DF000FF31FFF703BF4622F9E72DE9F0410546D1
:106E00000C4621F400471646C2B90B040ED5592191
:106E1000FFF736FE59212846FFF732FE5921284652
:106E2000FFF72EFE59212846FFF72AFE3B4628464B
:106E300042220021BDE8F041FFF7E0BE3B460021C1
:106E40004022FFF7DBFE210A21F07F013143284673
:106E5000C9B2BDE8F041FFF713BE322938B5054687
:106E600013D0332914D101240721A1F12902D2B270
:106E70004FF0FF312846FFF718FE5CB12846D322B9
:106E80000021BDE83840FFF710BE01240621ECE7E1
:106E90000024EAE738BD4379012B70B5044626D0BB
:106EA0000021FFF7D6FD626B236A00259B1A6363FE
:106EB000A563E068438D9D421AD3A38FE38763796E
:106EC000032B25D1A36A206A6062E3621844F9F7B4
:106ED000FCF8E3682063988BDB8B1844A38F18447D
:106EE000B4F8403018448000F9F7EFF8606470BDE2
:106EF000C36A03EBC50213F83530042B06D1917831
:106F00002046FFF7A6FDA36B0133A3630135D0E74D
:106F1000042BECD1038B626C216B0069BDE87040DF
:106F200003F0F6BF01F110033F2B73B506460C4684
:106F300007D8A1F18002D2B20121FFF7B6FD02B05D
:106F400070BD01212222FFF7B0FD0DF105031946A6
:106F5000E2B202F07F00E41103F8010C601C01288A
:106F600003F1FF3516D8013402F0400214D11AB9EA
:106F70007F2205F8012C9D1E491B3046FFF770FD4E
:106F800001AC411E2B46A3420AD15D1B9DF8042093
:106F90004255D4E72B46DBE7002AEDD00022E8E794
:106FA00013F8012B62F07F0201F8012FEBE773B5B4
:106FB0000DF1050406461D46FFF777FD214605F055
:106FC0007F03ED0904F8013DF9D1091B3046FFF7B5
:106FD00047FD01AD411E2346AB4205D19DF804207B
:106FE0001B1BC25402B070BD13F8012B62F07F026C
:106FF00001F8012FF0E770B4C4681E46A58BE38B3F
:10700000B0F840401D44C38F1D44631CA0F84030BD
:1070100063194479042C04BF446C44F8236070BCA9
:10702000FFF7C5BF30B41D4604460B692AB925B920
:107030003222012130BCFFF7DEBF33224FF0FF3197
:107040002046F7E7F8B515460446069F0A69EEB2F2
:1070500063B95FB91346C5F101012022FFF7CBFFE9
:1070600031462046BDE8F840FFF70ABD1346E94324
:1070700021222046F2E710B4044643B90F2A06D86D
:10708000503AD2B201215DF8044BFFF70EBD03F177
:107090002401204613465DF8044BCAB20121FFF7D4
:1070A00086BF10B404464BB90F2A07D8403AD2B273
:1070B0004FF0FF315DF8044BFFF7F7BC03F12601F9
:1070C000204613465DF8044BCAB24FF0FF31FFF77C
:1070D0006EBF03F128011346CAB20021FFF767BF54
:1070E000022A02F12A020B46D2B214BFC1F10101F9
:1070F0000121FFF75CBF032910B40CD004290DD087
:10710000002102248B1844EA83032F22C9435DF82F
:10711000044BFFF74CBF00210C46F3E70121FBE7CE
:107120000B4630220139FFF742BF10B4144641EA42
:107130000223214431225DF8044BFFF738BF70B4BD
:10714000DDE90365D2B203EB460443EA062315B139
:1071500001320234D2B2091B70BCFFF728BF07B559
:10716000CDE900230B4634220021FFF7E8FF03B0EE
:107170005DF804FB07B5CDE900230B4636224FF03E
:10718000FF31FFF7DCFF03B05DF804FBC268938BAF
:10719000D28B1A44838F10B45C1C134442798487C9
:1071A000042A08BF426C5DF8044B08BF42F8231064
:1071B00023220121FFF7FBBEFFF7E8BF0C2902D114
:1071C0000449FFF7E3BF01F14302D2B20121FFF707
:1071D0006CBC00BFFC36060838B504460D460E21CF
:1071E000FFF7ECFF20462946FFF7B8FD02215C229D
:1071F000FFF75BFC20466FF00301BDE83840FFF766
:1072000046BC2DE9F74F15460446002361716E8C8C
:107210008360C0E90323837183620362AB8CB5F89A
:107220002680AF8BB5F81890B5F820B00122F6187B
:1072300008BF16468A464FEA8801013E426101F0C6
:10724000040107F003021143F20002F07802EB8B15
:1072500009F00F09114336094FEA5808BF0846EAFA
:10726000080242EA09023A431A4352EA0B023ED1AB
:107270002046FFF7EEFBBAF1020F16D9D4E90D3222
:10728000590002F001009B09520801F07E01014300
:1072900063631343A26318BF41F080012046FFF7E8
:1072A000D8FBD4E90D321343E8D1236A636302218A
:1072B0002046EE8AFFF7C0FB0670360A46700221B0
:1072C0002046AE8AFFF7B8FB00230670BAF1040F20
:1072D0004FEA16264670A387A4F8403047D1A88B02
:1072E000EA8B1044984242D06E8D00213BE041F081
:1072F000800120460193FFF7ACFB4FEA8911320170
:1073000002F03002019B01F0400111430BF0010239
:107310001143DA0002F008021143BA0002F004023D
:1073200011434FEA480202F002021143B6084FEA45
:1073300058084FEA59097F085B084FEA5B0B8EE754
:10734000EA6A02EBC1025778FF070BD557889F42C4
:1073500008D15268616CD20042F0020241F8232049
:107360000133BFE701318E42EADC0522F2E703B0C8
:10737000BDE8F08F4820F8F7A8BE10B5044681613B
:107380008800F8F789FEE06110BD10B50446C069B9
:10739000F8F7AAFE2046BDE81040F8F7A5BE10B5E4
:1073A000044601618800F8F777FE606110BD10B5F2
:1073B000044611B1C068F8F797FE6069BDE8104057
:1073C000F8F792BE012938B504460D460ADC026979
:1073D000406992004FF0FF3118F0A8FC00232560AF
:1073E000636038BD4068F8F757FE6368E060A360EB
:1073F000F4E7D0E90032022B0ABFC36800239B18D0
:1074000011444160184670470368012BDEBF436991
:10741000426843F82120704742684B1E134449429A
:1074200019404160704738B50C461546FFF7E1FF3B
:1074300010B10444A04200D138BD00F8015B2D0A10
:10744000F8E7704710B50C460221FFF7D2FF10B1E4
:107450000470240A447010BD38B50D46042114464A
:10746000FFF7C7FF28B1057084702D0A240A457004
:10747000C47038BD70B50546032917D8DFE801F0A0
:107480001A1A02020024FE2646F435412846FFF768
:10749000D9FF44B17F2C10D844F4304141F0800131
:1074A0002846FFF7CFFFC5E9066470BD023921F019
:1074B0000104E8E70024F226E6E7A300A201DBB21C
:1074C00043F4506302F4E0421A434FF2AD212846E0
:1074D000FFF7C2FFE7E7C16910B5044629B17F296C
:1074E0000BD841F43041FFF7ADFFA169204641F4CC
:1074F0003D41BDE81040FFF7A5BF8A00D2B2890127
:1075000001F4E04142F450620A434FF20D21FFF7CB
:10751000A3FFEAE7114341EAC301FFF793BF072A3C
:1075200085BF083AD200D20042F04002072984BF4A
:10753000083941F08001114341F48C41FFF782BFCB
:1075400070B5DCB244EA02225C101D0104F48064D0
:10755000C3F303334668234305F4E0452A43194344
:10756000FFF77AFF304670BD38B5436953F82140C4
:107570004368E41A043C0546C4F34A0141F46041FF
:10758000FFF760FF2B68022B0AD124F4FF6020F084
:10759000070028B110F5006F14BF0020012038BD8E
:1075A0000120FCE7F8B5446954F822404268A41A67
:1075B000043C074666101D46ABB9090241F4504130
:1075C000F6B23143FFF73EFF3B68022B09D134F09E
:1075D000FF0506D015F5807F14BF0025012528463C
:1075E000F8BD0125FBE7A312890104F4005203F45E
:1075F000806341F47041C6F30B061943C4F385342C
:1076000042F4004232432143FFF726FFE7E738B553
:10761000436953F821404368E41A043C0546C4F327
:107620004F02C4F30A3142F4784241F47041FFF74B
:1076300013FF2B68022B08D1A00D800528B110F58F
:10764000800F14BF0020012038BD0120FCE7F8B5F1
:1076500004460D461646476813460A464FF2402137
:10766000FFF76EFF330C2A464FF2C0212046FFF78A
:1076700067FF3846F8BD072910B404460AD832F02F
:10768000FF0307D142F4005242EA01215DF8044BA6
:10769000FFF7D8BE130C1B0443B9134620460A4615
:1076A0005DF8044B4FF24021FFF74ABF20465DF8DA
:1076B000044BFFF7CCBF120242F41042C9B211438F
:1076C000FFF7C0BE090241F41841D2B21143FFF7DF
:1076D000B9BE090241F42841D2B21143FFF7B2BE4C
:1076E00038B5436953F8223042689B1A083B0C4670
:1076F00043F001030A464FF240210546FFF720FF01
:10770000210104F0070444F4884444F0780401F0B3
:10771000800121432846BDE83840FFF793BE072982
:1077200030B4054614460CD8072A0AD81F2B08D8AF
:1077300041EA831343F4D04343EAC20130BCFFF76C
:1077400081BE9B0043EA013244F47841284641F06F
:10775000D00130BCFFF780BE436953F82110436865
:10776000CB1A043B013130B4C3F34A0204460DD0B6
:10777000D91C0BDA23F4FF6525F0070515F5006F1A
:1077800004D142F4604130BCFFF75CBEC3F30A335E
:10779000204642F4384243F4704130BCFFF75CBEEF
:1077A000436953F822204368D31A043B013230B4B2
:1077B00005464FEA63040ED0DA1C0CDA23F0FF0210
:1077C00012F5807F07D10902E4B241F45041214310
:1077D00030BCFFF737BE8901981241F4704103F4C1
:1077E000005200F480600843C4F30B0442F40042EA
:1077F000C3F3853122430143284630BCFFF72CBE3A
:1078000038B514460B46072221460546FFF787FF89
:10781000E100284641F48F41BDE83840FFF712BE31
:1078200090F854007047436C1944C3684164012BBD
:1078300004DD836D9A8C9142C8BF9984704770476C
:10784000002280F854204FF0FF31FFF7ECBFFFF724
:10785000F7BF002280F854206FF00301FFF7E3BF69
:107860004FF0FF31FFF7DFBF38B5446CC3692144E7
:107870009942054608D9083121F00304E100006A65
:10788000F8F725FCC5E9074038BD70B504460E463B
:1078900001211546FFF7E8FF606C216A01EBC00388
:1078A00001F8306001215D6020465970BDE87040EC
:1078B000FFF7B9BF70B504460E4601211546FFF724
:1078C000D3FF606C216A01EBC003022201F8306033
:1078D0005D6020465A700121BDE87040FFF7A3BFEC
:1078E000002280F854201146FFF7E4BF002280F800
:1078F00054200A460221FFF7DDBF38B50D1E0446AD
:1079000015DDFFF7B1FF636C226A02EBC3020023AF
:10791000194602EBC300012D417006BF94F8240004
:1079200002F8330002F8331001339D42F1D12946A9
:107930002046BDE83840FFF776BFF8B5D0E90A53D6
:107940000133AB4204460E46174606D90435A9005A
:10795000006BF8F7BCFBA5622063D4E90B104B1C4D
:10796000E36230F8213066F30E0320F8213000EB9B
:107970008102C3F3072367F3C71353704FF6FF73F6
:107980005380E06D32460021FFF7AAFEE06D002231
:107990000321BDE8F840FFF78EBE10B4019C41EA18
:1079A000C301A40104F4F864114321435DF8044BBE
:1079B000FFF748BD41EAC20141F4C05141EA8311D9
:1079C000FFF740BD0B46D0E90B2102F18042013A9E
:1079D00001EB820210B50446D0786FF3C710D07067
:1079E000043A91420BD892F903000028F8DA128881
:1079F000E06DC2F30E020021FFF772FE06E063B9EC
:107A00001A4644F24001E06DFFF784FDE06D00226C
:107A10000321BDE81040FFF74EBE10BD10B504466F
:107A20000121FFF7CFFFE06D01220021FFF74AFEA1
:107A3000002220461146BDE81040FFF726BF000097
:107A40000C2903D1084A0021FFF734BF00220E2978
:107A500080F8542001D15421F6E7B1F10D0218BF8E
:107A600001220121F0E700BFFC36060810B4D0E97E
:107A70001640248BE407134604D506225DF8044B18
:107A8000FFF74DBE5DF8044BFFF71CBE70B5044612
:107A9000D0E91660368BF6070D460AD59200FFF73F
:107AA000EAFD2A462946E06D0623BDE87040FFF74F
:107AB00081BFBDE87040FFF70CBE037C70B5044683
:107AC000154623B9826D938BD28B13441D44E36812
:107AD000B4F84020042B08BF236D204608BF43F8AC
:107AE00025100021FFF7C2FF00221146E06D03239D
:107AF000FFF715FE00222B46E06D1146BDE87040F1
:107B0000FFF70DBEF8B5476C046A07F10053023B5E
:107B100004EBC30404F10803054693E8030084E87A
:107B20000300667856B9B5F842203A44013A314626
:107B30002846FFF79BFF01236370666028464FF0DD
:107B4000FF31BDE8F840FFF76EBE13B5D0E916303F
:107B50001B8BDB0707D5009106234FF4C041FFF7CD
:107B60001CFF02B010BD02B0BDE81040FFF7A3BD7E
:107B70002DE9F041466C002405460F46B61AA04692
:107B80006B6CA34201DCBDE8F081B44211D02B6ADA
:107B900003EBC4035A78012A0BD15A68BA4208D1C0
:107BA000B5F8421083F801803A4621442846FFF791
:107BB000CCFF0134E4E7826D138B70B543F02003F2
:107BC0000446002513830E4680F854502A46294661
:107BD000FFF7CEFFB4F84A200132A4F84A2031461C
:107BE0002046FFF76AFF2A4629462046BDE8704036
:107BF000FFF74BBE70B5002405460E4680F8544092
:107C000022462146FFF7B4FFF2002146E86D42F01C
:107C10000202FFF730FD224621462846BDE87040AB
:107C2000FFF733BEF8B583699E5C602E04461546A7
:107C300006D1076814480A46144907F003FC386067
:107C40000023022D84F854300DD8A36DDA8C52B97C
:107C50001B8BDB0707D40E4B5A5D31462046BDE82F
:107C6000F840FFF712BE002211462046FFF780FFC2
:107C7000B4F84220E36BED431A442A440021204625
:107C8000FFF7F4FE0022E8E7A8290608A414060876
:107C90001016060870B50024054626466B6CA342F4
:107CA00000DC70BD2B6A03EBC4035A78012A07D1AC
:107CB000B5F842105E705A6821442846FFF745FF28
:107CC0000134EBE7F8B504461E4617460D46FFF7AC
:107CD000E1FF3A463146E06DFFF7CDFC2946E06D05
:107CE0000322BDE8F840FFF78BBD38B504460D46CA
:107CF000FFF7D0FF2946E06D0322BDE83840FFF7CB
:107D00007FBD38B50025044680F854500821FFF7A0
:107D1000ECFF2A4629462046BDE83840FFF7B5BDAE
:107D2000F8B504461E4617460D46FFF7B3FF3A4620
:107D30003146E06DFFF79FFC2946E06D0322BDE868
:107D4000F840FFF75DBD10B4002302F1290480F86C
:107D500054300A46E1B25DF8044BFFF7E1BF00235F
:107D600070B504460E4680F85430154662B1037C67
:107D700053B1084604F0FFFE021E05DD20467021C7
:107D8000BDE87040FFF796BD06353246E9B22046A1
:107D90000023FFF7C5FF002220461146BDE87040D2
:107DA000FFF773BDF8B5164604460F46FFF772FF9E
:107DB00031462046FFF758FD0025636C2A46B54240
:107DC0000CD1B4F84220394620461A44FFF75EFE33
:107DD00029462046BDE8F840FFF725BD216A58191D
:107DE00001EBC00C01358CF8012001F83020E6E7EA
:107DF000F8B5044617461E460D46FFF74BFF3A46B8
:107E0000E06D0021FFF737FC3246E06D0121FFF7FE
:107E100032FC2946E06D0322BDE8F840FFF7F0BCD4
:107E2000037C63B1C1F1FF5101F5FF11436C01F512
:107E3000FF511F311944036A13F831007047184687
:107E40007047000070B50E4615463BB9037C2BB158
:107E5000C06D5268FFF70FFC287870BD2C7834B9DC
:107E60006A68C06D3146FFF706FC0020F5E7012C7B
:107E700007D16B68013307223146C06DFFF74FFC15
:107E8000F3E7A31E012B04D86A68520042F00102F6
:107E9000E7E7542C01D10023EDE7014804F0D2FCC0
:107EA000F2150608F8B5002504462E46636CAB4271
:107EB00005DC00252F46636CAB4210DCF8BD236A5D
:107EC00003EBC5035A78012A07D1B4F842105E705B
:107ED0005A6829442046FFF738FE0135E6E7266A4E
:107EE00006EBC5025378022B0ED1002357701946BA
:107EF0002046FFF7A7FFB4F8421006F8350000222D
:107F000029442046FFF721FE0135D4E738B5044661
:107F100000230D4680F85430FFF7C4FF2946E06D7A
:107F2000BDE83840FFF718BC38B504460D467AB1B5
:107F300000221146C06DFFF79EFB00220121E06D7B
:107F4000FFF7B9FB29462046BDE83840FFF7DEBF02
:107F50001146FFF737FDF5E72DE9F04104460E46DF
:107F6000C2B3D0E90B1C01F1804101390CEB810156
:107F70000023084615461F4690F901E0BEF1000FA8
:107F800011DA90F903E0BEF1000F0CDA002F08BF00
:107F900007463BB1B0F80080B3F802E068F30E0E7C
:107FA000A3F802E00346013DA0F10400E4D16FF024
:107FB0000300424301EB020EE06DCBB9F44510D94A
:107FC0001A4644F24001FFF7A5FA00220321E06DB2
:107FD000FFF771FB26F400412046BDE8F041FFF7B2
:107FE00095BF8A5A1946C2F30E02FFF779FBECE7F8
:107FF0005A8847F6FE7161F30E025A80294626F42C
:108000000042FFF76DFB2A460421E06DFFF753FBAA
:108010002A462946E06DFFF72EFB2A460121E06D36
:10802000FFF749FB3E88C6F30E06D3E7F8B50446D2
:108030000E4617460A4619461D46FFF799FD636C22
:10804000216A981B01EBC00211F830103970517889
:1080500001290DD002D3022913D0F8BDB4F8422073
:108060001A44921B29462046BDE8F840FFF7FEBCA3
:108070005268AA42F1D02946E06DBDE8F840FFF70A
:108080004EBA002329462046FFF7DCFE3870E4E7AD
:1080900010B50023044680F8543013460A460121E7
:1080A000FFF7C4FF20464FF0FF31BDE81040FFF757
:1080B000BABB70B5049E04461D46FFF7E9FF324681
:1080C00029462046BDE87040FFF7E2BF7FB5012595
:1080D0000DF10F030DF10E01009500220446FFF78C
:1080E000E8FF9DF80F609DF80E1020460022FFF774
:1080F000CCFB2A4631462046FFF7C7FB04B070BDD3
:10810000F0B585B001250DF10F030DF10E010095BD
:1081100000220446FFF7CDFF9DF80F709DF80E601A
:108120002A4639462046FFF7B0FB3146204600225A
:10813000FFF7ABFB2A4639462046FFF7A6FB002295
:1081400031462046FFF7A1FB05B0F0BD7FB51D46C7
:10815000002304460E4680F854302ABB25BBFFF7A7
:1081600099FD2A460121E06DFFF785FA2A46022192
:10817000E06DFFF780FAB4F84E20B4F84C30316966
:108180000133501CA4F84E001A442046FFF795FC1A
:10819000E06D03221A21FFF733FB0022114620462F
:1081A000FFF773FB04B070BD0123009320460DF16F
:1081B0000E0302220DF10F01FFF77BFF2046FFF7B0
:1081C00069FDD8E72DE9F041DDE9068504461F4643
:1081D000089EFFF75DFF424639462046FFF758FFED
:1081E000324629462046BDE8F041FFF751BF2DE950
:1081F000F04186B002260DF11703012501930DF120
:1082000015010DF116030296009500220446FFF7B2
:10821000D9FF9DF817809DF816709DF8151020461F
:108220000022FFF732FB324641462046FFF72DFB86
:108230002A4639462046FFF728FB06B0BDE8F08104
:1082400030B587B00DF117030025019302230446D2
:10825000009301220DF116030DF115010295FFF7B0
:10826000B1FF20461921FFF740FD2A462946204646
:10827000FFF70BFB07B030BDF7B5C46A05460F46E4
:10828000D4B104F18044036B013C03EB840292F906
:108290000120002A21DA33F82430C3F30E038B4285
:1082A0001BD100220DF10701FFF7F2FE0022012190
:1082B000E86DFFF700FA01240026284685F854608F
:1082C000FFF7F0FD3946E86DFFF79EF81CB1314627
:1082D0002846FFF777FB03B0F0BD0024ECE770B54C
:1082E00000260446012280F854603146C06DFFF735
:1082F000E9F922212046FFF7F8FCD4E90B35013BD0
:1083000005EB8305E3626B8847F6FF72C3F30E0348
:10831000934228D004223146E06DFFF7D3F94FF4A1
:108320002051E06DFFF78EF86368E06D1A68314602
:10833000FFF736FA698847F6FE73C1F30E029A42D8
:108340000BD14FF48E41E06DFFF77CF86368204657
:108350001968BDE87040FFF78FBFC1F30E012046DA
:10836000FFF7D4FDF2E770BD2DE9F04304468168C4
:1083700085B0FFF781FFA36DDA8C198B12B901F07C
:10838000110373B311F0010117D1B4F84020204656
:108390000132FFF76BFBA36DDD8C55B94FF4205113
:1083A000E06DFFF74FF8A268E06D01322946FFF754
:1083B000F7F905212046FFF798FC21212046FFF719
:1083C00094FCA36D1A8BD20706D4DB8C23B9A16869
:1083D00020460131FFF750FF05220021E06DFFF735
:1083E00071F9E06DFFF777F8237C002B5CD1E36D2A
:1083F000E56B5B686363A36D013D9E8B1F8BB3F8D8
:108400001E90B3F82080EA0006F0030302F0780221
:1084100007F00F071A432D09B60845EA070333434F
:1084200043EA090353EA0803E06D75D10121FEF721
:10843000FAFF0421B4F8483003F001025B0842EA75
:108440004102A4F848300BB142F080020121E06DF6
:10845000FEF7E9FFB4F848500021002DEAD1A36DE2
:10846000E06DDA8A0121FEF7DEFFA36DE06DDA8AA6
:108470000121120AFEF7D7FFA36DE06D9A8A012150
:10848000FEF7D1FFA36DE06D9A8A0121120AFEF773
:10849000CAFFE36D5E68D4E91620538DAB425BDC06
:1084A00043689B1BA4F84830E06DFEF7CAFFE36801
:1084B000B4F84A00A4F84C00032B12D1B4F84E30A3
:1084C00001301844237C002B53D1A36D9D8BDB8B93
:1084D0001D4428448000F7F7DFFD274B206540F856
:1084E0002530E368042B14D1257CA16DE36D086968
:1084F000002D4FF00005D3E9023203950D8B029554
:10850000898B0191216D00910CBF0321042102F0A0
:108510000CFD05B0BDE8F08342F080020121FEF7BA
:1085200082FFBA012B0103F0300302F040021A432C
:1085300008F001031A434FEAC90303F008031A4382
:10854000B30003F004031A43AD087F0876084FEA2E
:1085500059094FEA580860E7D26A02EBC50312F8DE
:108560003520042A03D15A880121FEF75CFF01352A
:1085700091E70025AEE700BFFC190608F8B543688F
:108580001A688260826D158BD28C04461AB915F078
:10859000110F00F0E7801E6815F0010506F10207D3
:1085A00016D1B4F8402029462046FFF75FFA2A4644
:1085B00001232946E06DFFF7B2F805212046FFF7B9
:1085C00094FBB4F840102A4601312046FFF7BDFA6B
:1085D000D4E91630DA8C002A68D1198B11F0010524
:1085E00008D14FF42051FEF72DFF3A462946E06DA1
:1085F000FFF7D6F800221146E06DFFF76AF8202158
:108600002046FFF772FB4FF42051E06DFEF71AFF92
:108610003A460021E06DFFF7C3F8A36D198B11F006
:10862000010109D1B4F8402020460132FFF71EFABB
:1086300005212046FFF759FBD4E91630198B11F0BC
:1086400001014FF0010200F086800021FFF73AF8A7
:1086500046F27011E06DFEF7F5FEE06D022200219A
:10866000FFF709F8E06DFEF736FF39462046FFF7C1
:1086700003FEA36D1B8BDB0774D5B4F840202046A6
:1086800001320021FFF7F2F9E06D4FF48E41FEF761
:10869000D9FEE06D4368A36300210122FFF712F8C1
:1086A00020462221BDE8F840FFF71FBB00231A46F1
:1086B00044F24001FEF72EFF00220421E06DFEF798
:1086C000FAFF751C3A460421E06DFFF709F82946C8
:1086D0002046FFF7D1FD04220521E06DFEF7F2FFF1
:1086E00000221146E06DFEF7F4FF20212046FFF73F
:1086F000FCFA05220421E06DFEF7DDFF03364FF49E
:108700002051E06DFEF79EFE32460121E06DFFF73D
:1087100047F800231A4644F24001E06DFEF7FAFEE6
:1087200000220321E06DFEF7C6FF44F22071E06DE8
:10873000FEF788FE31462046FFF79EFD0322042106
:10874000E06DFEF7BFFF4FF43051E06DFEF77AFEAB
:108750002A4601215EE7FEF7B5FF22212046FFF7FA
:10876000C4FA82E7F8BD0000538B2DE9F041DE1E0C
:10877000044673427341E160037400234364A0F82C
:108780004A30A0F84E3080F854300F464369518C7F
:10879000A2658B42154605D28069F7F798FC6B8C71
:1087A000A0616361A16DCB8B8A8B1A442B8B580718
:1087B00048BF01329B074FF0000348BF0132184603
:1087C0009A4209D1227C22B1B1F82AC000229445F4
:1087D00006DC6269602115E0A669F0540133EFE719
:1087E000CE6A06EBC2060132707810F0010F1FBF8F
:1087F000B6F802E0A669000906F80E00E7E7A069EE
:10880000C15401339A42FAD80023E1691846602620
:10881000994234D1042F14BF01210221E06DFEF7EB
:10882000D1FDA26D0023A4F84030D38C1BB9118B6D
:1088300001F0110111B11221A4F840106E8CA98C25
:1088400094F81080E06D3144E163B8F1000F00F05E
:10885000D380EBB9128BD70707D4032E3346AE8BE8
:10886000A8BF0323032E00D9013B12F0110F10D132
:108870002E8BB4F84020B60648BF01320CE0226AC5
:1088800002EBC30C8CF8010002F833600133BFE740
:108890000023B4F840200232A4F84220B4F8422069
:1088A0001144C91AFEF7E6FD032300220621E06DFC
:1088B000FEF735FF002306220721E06DFEF72FFFAC
:1088C000A36DDA8C1AB91B8B03F030032BB1002295
:1088D000B4F84010E06DFEF7EEFE01220021E06DDD
:1088E000AA4EFEF71CFE02220121E06DFEF717FEE4
:1088F00003220621E06DFEF712FE4FF42451E06DD5
:10890000FEF7A0FD6368E06D1A6801210432FEF7EE
:1089100047FFAA8BE06D0221FEF7ADFE0223002285
:108920004FF48541E06DFEF7F5FD6368E06D1A6870
:1089300000210532FEF734FF6368E06D19680431E9
:10894000FEF762FDAB8BE06D5A0042EA4342022122
:10895000FEF791FE03222C21E06DFEF751FF6368C4
:10896000E06D19680531FEF74FFD0025A36D9A8B68
:10897000AA4214DC032A0DD9DA8C5AB91B8BDB0707
:1089800008D4B4F84220E36BE06D1A44033A0621A0
:10899000FEF798FE2046BDE8F041FFF7EFBD2B46FD
:1089A00006220021E06DFEF7BAFEA3695A5D22B1EE
:1089B000012303212046FFF785F9022D11DCA36D69
:1089C000DA8C72B91A8BD2070BD4022D02D19B8B91
:1089D000032B06D10022715DE06DFEF7A0FD01358D
:1089E000C4E7B4F84210E36B194401390022491B73
:1089F0002046FFF7AAF8F2E7168B16F001063DD0E5
:108A00004FF4A0232364626B0421FEF70CFDA26BDC
:108A1000E06D0421FEF707FD1221E06DFEF72AFD4F
:108A200042460621E06DFEF77AFD01221146E06D17
:108A3000FEF741FEB4F84030E06D06224146FEF7F5
:108A40006EFE032342464146E06DFEF768FEA26DCE
:108A5000E06D918BD38B42460B440721FEF75FFEFE
:108A60002046FFF78BFDA36DDA8C1AB91E8B16F02A
:108A7000010657D000236E8D194661E0B4F84030EE
:108A800005339BB2A4F842301944FEF7F3FC32469A
:108A9000E06D03230621FEF742FEA26DE06D918B8F
:108AA000D38B06220B440721FEF739FE3246B4F879
:108AB0004010E06DFEF7FFFD626BE06D3146FEF7A2
:108AC000DAFDB4F84010324620460131FFF73DF898
:108AD000E26BE06D3146FEF7CEFDB4F84010324651
:108AE00020460331FFF731F8B4F84020E06D3146FD
:108AF000FEF7EFFD04222D21E06DFEF781FEAFE7CA
:108B0000B4F84220E36B18F80610E06D1A44013AFD
:108B1000921B0136FEF7D6FD032EABD06B8CB34211
:108B2000EEDCA7E7DFF86480F8E7EA6A02EBC3004F
:108B300012F83320042A02BF4288A069815401330D
:108B40009E42F2D8042F05D1A88BEB8B002218444B
:108B5000904218D1BDE8F081EB6A03EBC1035F7866
:108B6000FF070BD55F88974208D15B68216DDB005A
:108B700043F0020341F822300132E9E701318E422D
:108B8000EADC0523F2E70021F9E700BF101606082A
:108B90007FB504460D46164682B90DF10F01FFF769
:108BA00077FA2A46092120460123FFF7B9F8324611
:108BB00031462046FEF769FE04B070BD012A0FD190
:108BC0000223009300220DF10F030DF10E01FFF7B8
:108BD00070FA01232A460E212046FFF7A1F8EBE7A1
:108BE0000DF10F010022FFF753FA02231A4644F257
:108BF0004001E06DFEF78EFCEBE773B504460E46D0
:108C0000154672B901220DF10701FFF741FA05F18E
:108C10000C0100233246C9B22046FFF781F802B0AA
:108C200070BD0021FFF7FCF88DF8070020B9012284
:108C30000DF107012046E8E70DF10701204600226B
:108C4000FFF726FA9DF80720204601230421FFF7AD
:108C500039F800220121E06DFEF761FCD7E773B51A
:108C60000D4616460DF1070100220446FFF710FAE3
:108C7000721C2A4420460221FFF794F8012345EA9A
:108C8000062228212046FFF71DF802B070BD37B537
:108C900004460D4600220DF10701FFF7F9F92A46B7
:108CA00020460221FFF77EF801232A46272120468D
:108CB000FFF708F803B030BD37B50D4600220DF1BF
:108CC00007010446FFF7E4F955B1012120460422CB
:108CD000FFF768F81E212046FFF707F803B030BD04
:108CE0002A46E06D0121FEF7C6FC20461E21FEF754
:108CF000FCFF2A4629462046FEF7C7FDEEE70000A6
:108D000037B500220DF107010446FFF7C1F99DF8C0
:108D100007302BB105490648256806F093FB28600B
:108D200022212046FEF7E1FF03B030BDB91406084A
:108D3000A829060873B501220E460DF10701044665
:108D4000FFF7A6F99DF8075065B932461121204674
:108D50002B46FEF7B7FF2A4629462046FEF795FD2B
:108D600002B070BD20460121FEF75DFD044B0549B0
:108D70009A5D0548246806F065FB2060F0E700BFB7
:108D8000E0400608D8150608A82906082DE9F34191
:108D90000E460021174604461D46FFF741F802A97A
:108DA000024601F8010D38BB2046FFF771F91DB9E5
:108DB00001212046FEF737FD10212046FEF795FFE2
:108DC0001DB99DF8073084F824302046FFF76AF873
:108DD0004FF42051E06D7EB3FEF734FB3A4601219B
:108DE000E06DFEF7DDFC25B94FF0FF312046FEF7C0
:108DF0001AFD02B0BDE8F08100222046FFF748F9D5
:108E00001DB901212046FEF70EFD9DF807305A1EC0
:108E1000022AD5D9072B98BF0A4A0B4998BF32F8C6
:108E200013200A48D4F8008088BF4FF4387206F047
:108E300009FBC8F80000C3E7FEF704FB3A463146D9
:108E4000CEE700BF3414060897140608A8290608C0
:108E50000023FFF79BBF0123FFF798BF022A7FB5CE
:108E600004460E46154614D8836DDA8C8AB91B8BDE
:108E7000DB070ED41D4B0DF10F015A5DFFF708F90A
:108E8000A1699DF80F204B5D602B13D14A5504B0AA
:108E900070BD0DF10F0120460022FFF7F9F8E16BDC
:108EA000B4F842300B44E943002219442046FEF74F
:108EB0004CFEE5E79342EAD0072B98BF0C492468A3
:108EC00098BF31F813300B4888BF4FF43873072A26
:108ED00096BF07494FF4387231F8122000920649C4
:108EE000324606F0AFFA2060D1E700BF1016060840
:108EF00034140608A8290608CB14060870B50446E1
:108F00000D4616464BB90E21FEF79AFD324629460C
:108F10002046BDE87040FFF7A1BF70BDF8B5446CB6
:108F2000D0F820C0DDF818E004F100540E46013CF2
:108F3000002180F854100CEBC40105464F78012F36
:108F400012D1496899420FD071450DD01CF83430C8
:108F5000337011603A46FEF70BFE28464FF0FF31A2
:108F6000BDE8F840FEF75FBC136801213246284691
:108F7000FFF75CF8F1E77FB504AA002342F8043D4F
:108F80004FF0FF3300930DF10B010446FFF7C6FFCE
:108F90009DF80B50039E294632462046FEF775FC8D
:108FA000324629462046FEF770FC04B070BD000032
:108FB000F0B50D4685B001210446FEF731FF0021D2
:108FC00002468DF80A002046FEF72AFF931E012B69
:108FD00007468DF80B0000F2D280861E012E00F2AB
:108FE000F880A5F109030C2B9CBF0D35EDB21F2DA8
:108FF00001D0212D23D10023009301220DF10A037A
:109000000DF10B012046FFF754F89DF80A30022BB2
:1090100007D07F4B7F495A5D7F48266806F012FAD9
:1090200030601F2D0CBF2E212F212046FEF75DFE44
:10903000002202212046FEF728FC05B0F0BD04AA5C
:109040000126022342F8043D0DF10B0100232046C6
:109050000096FFF763FF32460DF10A012046FFF745
:1090600017F8A5F11903B34217D8192DE06D039B2A
:1090700008D132464FF48141FEF74CFA01229DF8A7
:109080000A10D7E79DF80A20032A08BF44F2C0015E
:10909000324618BF4FF48241EEE7162D05D1039BEF
:1090A00032464FF48641E06DE6E7172D04D1039B6D
:1090B000324644F24001F6E7182D04D1039B3246B4
:1090C0004FF48041EFE71B2D06D1039BE06D324644
:1090D0003146FEF76FFCD1E71C2D08D10399E06DF6
:1090E00041F6092343EA8111FEF7ACF9C6E71D2DCD
:1090F00004D1039B324644F24031D4E7052D31D8E8
:109100009DF80A209DF80B309A4205D04349424809
:10911000266806F097F930609DF80A300022032B8C
:109120001146204614BF06260026FEF721FD012227
:10913000039BE06D4FF48541FEF7ECF93544384B65
:10914000E06D33F81510FEF77DF942F20101E06D94
:10915000FEF778F94FF40051E06DFEF773F9002245
:10916000012167E720460121FEF75DFB284B2D49D1
:109170005A5D2948246806F065F920605DE742BB26
:1091800038BB012600960DF10A0302220DF10B01F6
:109190002046FEF78EFF322D17D0332D17D03E46D6
:1091A00000232A4612212046FEF78CFD56B10022EC
:1091B0000121E06DFEF7B3F90023032211212046BF
:1091C000FEF780FD0022114634E70625E8E7072573
:1091D000E6E74FF0FF312046FEF725FB9DF80A3009
:1091E0000D482468072B9CBF0F4A32F813209DF8C6
:1091F0000B3088BF4FF43872072B96BF0A494FF4E3
:10920000387331F81330094906F01CF9B5E700BF8F
:109210002E3F060844140608A82906085414060818
:10922000F8150608671406083414060875140608AD
:1092300070B5044686B00D4616461BB9FFF70EFE04
:1092400006B070BD00221146FEF792FC20460022B7
:109250000121FEF78DFC324629462046FEF7E2FC4E
:1092600006AA002342F8083D4FF0FF3300930DF1AA
:109270000F012046FFF752FE01230593049B009344
:109280000DF10F01204605AAFFF748FE059B049942
:10929000E06D43F4C04343F0400343EAC101FEF7ED
:1092A000D1F8CDE77FB504460D4616461BB9FEF74B
:1092B000B9FC04B070BD00221146FEF759FC3246DD
:1092C00029462046FEF7AEFC04AA00254FF0FF33E6
:1092D00042F8045D0DF10B0100932046FFF71EFEDE
:1092E000039AE06D29460123FEF719FA2A4629461A
:1092F0002046FEF7CAFADCE703297FB50546164685
:1093000012D101220DF10F01FEF7C2FE1824002335
:109310000DF10F0231462846FEF788FE2146284609
:10932000FEF7E3FC04B070BD052906D101220DF162
:109330000F01FEF7ADFE1724E9E702230093012297
:109340000DF10F030DF10E01FEF7B3FE1924DEE758
:10935000F0B5044685B00F461546C2B90223067C17
:109360002274009301220DF10F030DF10E01FEF79F
:10937000A0FE3A4626742B4623212046FEF7D0FC59
:109380002A4611462046FEF780FA05B0F0BD012AB4
:1093900010D1002680F8546033460DF10F022946A3
:1093A000FEF744FE3A462B4624212046FEF7B8FC41
:1093B0003246E6E70DF10F010022FEF769FE252196
:1093C0002046FEF792FCE0E72DE9F84F0446894677
:1093D0001746FEF75FFC00256FF06048AA46BD42C5
:1093E00010D10027BB46BD422BD169422046FEF773
:1093F0001AFAB4F84220636C49461A44BDE8F84FA3
:10940000FEF744BB666CD4F820B04644761B0BEBE9
:10941000C6025378022B12D182F801A001234946DB
:109420002046FEF70FFDB4F84210636C0BF83600CF
:10943000194401394A46491B2046FEF786FB01358F
:10944000CDE7636CD4F820A003F1005808F1FF3891
:10945000A8EB07081AF83820BAB1B4F842601E44E5
:10946000013EF61B324600212046FEF7FFFA01239B
:109470001AF8382004212046FEF724FC0022314649
:109480002046FEF762FB0AF838B00137ABE7000070
:10949000037C37B504460D4613B1544803F0D2F9A6
:1094A000826D138B43F001031383FEF7FBFC012D48
:1094B0000BD16368196820460231FEF727FD636807
:1094C000196820460131FEF7D7FE0122002120460F
:1094D000FFF77AFF002202212046FEF736FB012229
:1094E0000021E06DFEF7C7F800220521E06DFEF7D0
:1094F000E2F86368E06D1A680021FEF7F1F8B4F84D
:109500004010002201312046FEF71FFBA168E06DEC
:10951000FEF722F96368E06D1968FDF775FFE36AED
:10952000BBB1226B03F18043013B02EB83039A4200
:109530000FD893F9031000291BDA1A88E06DC2F3E3
:109540000E020021FEF7CCF800220321E06DFEF7A9
:10955000B2F801212046FEF7D0F965B92946E06D41
:109560000122FEF7AFF822212046FEF7BEFB03B032
:1095700030BD043BDBE76368196820460231FEF723
:109580007BFE0DF1070120460122FEF781FD00233D
:109590000DF1070220460121FEF748FDE06D012292
:1095A0000221FEF78FF8204602220021FEF76DF916
:1095B000012220460221FFF707FF20463021FEF757
:1095C00094FBE06D4FF42051FDF73CFF6368E06DC4
:1095D0001A6801210132FEF7E3F820460121FEF767
:1095E0008CF92046FEF78EFAC1E700BFE5150608A4
:1095F000F8B5174604460D46520093B10B1D1A44A8
:109600000221FFF7E1FE45EA072301221D21204642
:10961000FEF7EEFB002220461146BDE8F840FEF7BB
:1096200034B984F854308B1C1A440221FFF7CCFE65
:109630003B462A461C21EAE72DE9F743164600255A
:1096400001EB42020F4680F85450114604469946F9
:10965000FEF7E6FB70288DF8060032D1626C236AB3
:1096600003EBC2032946204613F80C6CFEF7D8FB27
:1096700007280DD888B12046FEF744FA636C226AA9
:1096800003F10053013B02F8336003B0BDE8F083FF
:109690005428F0D01E4803F0D5F82A460DF10701F2
:1096A0002046FEF7F5FC2046FEF7CAF832460321B5
:1096B0000123FEF707FB2A4631462046FEF7E5F870
:1096C000E3E747EA0628B9F1000F0DD00332022183
:1096D0002046FFF779FE43462A461D212046FEF725
:1096E00087FB00221146E8E707B91EB10221204698
:1096F000FFF76AFE0DF1060120460022FEF7C8FCC6
:10970000012342461B212046FEF7DCFAE9E700BFB1
:109710008F140608F8B500270E460446154606992C
:1097200080F854700BBB01BB0221FFF74DFE2A46A7
:10973000E06D0121FDF79FFFB4F84E20B4F84C30E6
:1097400031690133501CA4F84E001A442046FEF73C
:10975000B4F9E06D03222B21FEF752F800222046D7
:109760001146BDE8F840FEF790B8AA1C0221204639
:10977000FFF72AFE45F48072DAE770B5042A86B056
:1097800004460E4615462AD102294FF0000518D18D
:109790000DF1160301220DF117010095FEF789FC6A
:1097A0002B4607223146E06DFDF7B9FF2621204602
:1097B000FEF79BFA002211462046FEF766F806B037
:1097C00070BD0DF1150301930123009302950DF176
:1097D000160302220DF11701FEF7F4FCE6E7002361
:1097E000012A80F8543001D9032A04D132460121DC
:1097F0002046FFF7E9FD05F1130100233246C9B207
:109800002046FEF75FFAD5E770B50025044604222E
:109810000E4680F854502946FFF7D6FD2046042115
:10982000FEF701F81F21FEF760FAE06D4FF42051BA
:10983000FDF708FE32462946E06DFDF7B1FF2A46E6
:1098400029462046BDE87040FEF71FB870B50025D8
:1098500004460E4680F854502946FEF7B3F82046D9
:109860004FF0FF31FDF7DFFF636819680231FEF743
:1098700003FD2A4620465421FEF71CF82A462046BE
:109880005421FEF717F82A4620465421FEF712F815
:10989000204605220221FFF797FD03222B46204692
:1098A0001C21FEF7A5FA636820461968FEF72EFB17
:1098B0003146E06DFDF7A8FD20460121FEF782F854
:1098C00020460221FEF719F801222946E06DFDF736
:1098D000F9FEE06D4FF42051FDF7B4FD6368E06DD3
:1098E0001A6829460232FDF75BFF2B462A46E06DD7
:1098F0000121FDF714FF294620460122FDF7C5FF8F
:109900002A4629462046FDF7C0FF2A462046542114
:10991000FDF7D0FF204605220221FFF755FD2B461B
:10992000032220461C21FEF763FA20461021FEF791
:10993000DCF9E06D4FF42051FDF784FD6368E06DC4
:109940001A6829460132FDF72BFF63682046196823
:10995000FEF792FC2A462946E06DFDF78CFEE06D8D
:109960002A460121FDF7A7FE6368196820460131E8
:10997000BDE87040FEF780BC73B504460E46154640
:10998000002A56D1134601210DF10702FEF74EFBC6
:10999000022211462046FEF705FA01230D220A2174
:1099A0002046FEF7BDF902220DF107012046FEF721
:1099B0006FFB01220DF107012046FEF769FB2A46E5
:1099C0000DF107012046FEF763FB01229DF8071009
:1099D0002046FDF75AFF02229DF807102046FDF7AA
:1099E00054FF022211462046FEF7DCF901230C2227
:1099F0000A212046FEF794F9022211462046FFF77D
:109A0000E3FC2B462A461C212046FEF7F1F92A46A4
:109A100029462046FDF739FF2046FEF743FA204647
:109A200001223146FDF789FF2046FFF7A4FA02B074
:109A300070BD002380F85430FEF734FAAB1E5A4252
:109A40005A4131462046FDF778FFF0E737B5044626
:109A50000D4682B103220121FFF7B6FC022201214B
:109A60002046FEF79FF900232A460B212046FEF7E9
:109A700057F903B030BD0DF10701FEF709FB0222D3
:109A800011462046FEF78EF901232A460A21EDE70A
:109A9000836D73B51D8B15F00106044613D00122AA
:109AA0000021FFF791FC002202212046FEF74DF82D
:109AB00000221146E06DFDF7DEFD00220521E06D7C
:109AC000FDF7F9FD1CE0027C002A52D03146FEF77A
:109AD000A7F95428C5F3871528D12046FDF7B0FE15
:109AE000C5B92B4607222946E06DFDF718FEA36D88
:109AF000DA8C002AE1D11B8B03F01103002BDCD19F
:109B0000E26AA1682046FEF727FA012384F8543060
:109B100002B070BD32463146E06DFDF7ACFD012369
:109B20002A4604212046FEF7CDF8E0E732460DF143
:109B300007012046FEF7ACFA9DF80730AB4215D07E
:109B4000072D98BF0D4A0E4898BF32F81520266899
:109B500088BF4FF43872072B96BF08494FF438730B
:109B600031F81330074905F06DFC3060002DBED090
:109B7000D5E70DF10701FEF78BFAB8E734140608B4
:109B8000A8290608C31406082DE9F04389B0044645
:109B90000F460DF11C08002940F021810121FEF73C
:109BA0003FF90DF12009054609F8090D80BB014672
:109BB0002046FEF735F98DF81C00B8B90122414660
:109BC0002046FEF765FA002249462046FEF760FA75
:109BD00004220F2102232046FEF774F800221146CA
:109BE0002046FDF752FE09B0BDE8F0832A46414603
:109BF0002046FEF74DFA9DF81C2020460123042143
:109C0000FEF760F82A460121E06DFDF788FCDAE7EF
:109C1000636C226A03F10053013B02EBC30132F88B
:109C2000332040F202239A426CD1204601254E682F
:109C3000FDF706FE2B460095424649460797FFF77B
:109C40006DF99DF81730062B26D0072B3FD0052B3A
:109C500040F0B580C6B1731E1E2BE06D09D8079B7E
:109C600000963A464FF4F041FDF797FE002202219C
:109C7000B6E732462946FDF7FEFC079BE06D2A4613
:109C80002946FDF797FE07950799C90041F4F04171
:109C9000E06DFDF7D7FBE9E7A6B1731E1E2BE06D63
:109CA00005D80096079B3A464FF40841DCE772005E
:109CB0002946FDF7E0FC079BE06D2A462946FDF7A3
:109CC00079FE07950799C90041F40841E0E7A6B17C
:109CD000731E1E2BE06D05D80096079B3A464FF485
:109CE000D041C1E7B2002946FDF7C5FC079BE06DF6
:109CF0002A462946FDF75EFE07950799C90041F4FB
:109D0000D041C5E70123079342463B4606A92046BA
:109D10000097FFF703F93A4649462046FEF7B8F99F
:109D20009DF818309A1E012A0ED9072B98BFBB4AFE
:109D3000BB4998BF32F81320BA48256888BF4FF452
:109D4000387205F07FFB28609DF81730062B0CD089
:109D5000072B19D0052B32D100221146079BE06D4D
:109D6000FDF728FE4FF4F04192E700221146079BD1
:109D7000E06DFDF71FFE00221146079BE06DFDF729
:109D800019FE4FF4084183E700221146079BE06D5E
:109D9000FDF710FE00221146079BE06DFDF70AFE5D
:109DA00000221146079BE06DFDF704FE00221146DC
:109DB000079BE06DFDF7FEFD4FF4D04168E7072BF0
:109DC00098BF964A984998BF32F81320954825685D
:109DD00088BF4FF4387205F035FB286046E701294B
:109DE00040F06481FEF71CF808AE014606F80B0D42
:109DF00030BB2046FEF714F8022102468DF8180009
:109E00002046FEF70DF88DF81C0002B940B1002184
:109E100020460322FFF7D8FA03212046FDF703FD71
:109E20000223CDE901830023009306A9204633468F
:109E30000122FEF7C7F90F212046FDF756FFD2E6B3
:109E4000636C226A03F10053013B02EBC30132F859
:109E5000332040F202239A4240F08C8020464D6825
:109E6000FDF7EEFC02230022CDE90623009306AAAB
:109E70003B463146FFF752F8069B009742460DF1EC
:109E800017012046FFF74AF89DF817305A1E022A9C
:109E90000ED9072B98BF614A644998BF32F8132046
:109EA0006048266888BF4FF4387205F0CBFA3060FE
:109EB0009DF81530062B27D0072B40D0052B40F0FE
:109EC000E580BDB16B1E1E2BE06D07D8DDE90632C3
:109ED00000954FF4E041FDF760FD84E62A4601213C
:109EE000FDF7C9FB0122069BE06D1146FDF762FDFF
:109EF00001230693079941F4E041069B41EAC3011F
:109F0000E06DFDF79FFA6EE6ADB16B1E1E2BE06DA6
:109F100005D80095DDE906324FF40041DBE76A0021
:109F20000121FDF7A8FB0122069BE06D1146FDF71C
:109F300041FD01230693079941F40041DDE7ADB1EE
:109F40006B1E1E2BE06D05D80095DDE906324FF43F
:109F5000C041C0E7AA000121FDF78DFB0122069B4D
:109F6000E06D1146FDF726FD01230693079941F4A4
:109F7000C041C2E702230793009306AA00230DF114
:109F8000160120460697FEF7C9FF002231462046FB
:109F9000FEF77EF89DF816309A1E012A0ED9072B7F
:109FA00098BF1E4A224998BF32F813201D482568E1
:109FB00088BF4FF4387205F045FA2860069B00937D
:109FC000424600230DF117012046FEF7A7FF9DF83A
:109FD00017305A1E022A0ED9072B98BF0F4A134971
:109FE00098BF32F813200F48256888BF4FF43872A5
:109FF00005F028FA28609DF81530062B1AD0072B9B
:10A0000028D0052B42D100221146069BE06DFDF7BA
:10A01000D1FC079941F4E04172E700BF341406080F
:10A02000E4140608A8290608DB140608EE1406083E
:10A03000F914060800221146069BE06DFDF7BAFCF4
:10A0400000221146069BE06DFDF7B4FC079941F430
:10A05000004155E700221146069BE06DFDF7AAFC82
:10A0600000221146069BE06DFDF7A4FC002211467C
:10A07000069BE06DFDF79EFC00221146069BE06DFD
:10A08000FDF798FC079941F4C04139E7072B98BFC9
:10A090000D4A0E4998BF32F813200D48246888BF36
:10A0A0004FF4387205F0CEF920609CE50025434658
:10A0B00006A900950122FDF7FCFF02232A460F2185
:10A0C0002046FDF7FFFD8EE534140608F31406085C
:10A0D000A8290608F8B5074660200D461646F5F78C
:10A0E000F4FFC0E9007508250446C5614020F5F776
:10A0F000D3FFA56220622020F5F7CEFF2063202049
:10A10000F5F7E3FF3146E065FDF749F92046F8BD74
:10A1100010B504460021C06DFDF749F9E06DF5F773
:10A12000E3FF206BF5F7E0FFA069F5F7DDFF206A9C
:10A13000F5F7DAFF2046BDE81040F5F7D5BF00007F
:10A1400038B50446B2B1950714D110792E2811D133
:10A1500092687AB190070DD15068C5B2922D09D19D
:10A16000000A022806D191681960049BD2681A601F
:10A17000012038BD0A460448044905F063F9636AC2
:10A1800018600020F5E700BF7C2806083217060893
:10A19000038C032B70B5C46A03D1856A00239D42EA
:10A1A00005D144F82120FDF72FF9012070BD54F8A6
:10A1B0002360964201D00133F1E70020F6E710B5A5
:10A1C0000446FDF788F92046BDE81040FDF739B98F
:10A1D00038B58BB2032B04460D460384426205D189
:10A1E000826AC06A9200002115F0A0FD042D20466D
:10A1F0000CBF02210121FDF7E5F820460021BDE852
:10A200003840FDF737B9000002F00F03022B10B5FC
:10A21000044608D00A460C490C4805F013F9636A55
:10A220001860002010BD836A12090020834204D107
:10A23000238C042BF5D10649EEE7E16A51F8201092
:10A240009142EFD00130F1E76A1706087C28060832
:10A250007017060800F00F03022B02D10009F6F771
:10A2600053BE0148704700BF93C7060870B5054646
:10A2700010460E46FFF7EEFF0378732B19D1437893
:10A28000BBB103460A22002013F8014F5CB91F2816
:10A2900008D91F2332460A490A4805F0D3F86B6AE9
:10A2A0001860002070BD303C092C02D802FB004031
:10A2B000EAE732460449034805F0C4F8EFE700BF77
:10A2C000931706087C280608A01706082DE9F04118
:10A2D000054610461F460E46FFF7BCFF174B90F889
:10A2E00000C000229E4603EB8204617861451CD1C8
:10A2F00090F80180A178884517D190F80280E17824
:10A30000414512D171B91EF82200B84208D93B4626
:10A3100032460B490B4805F095F86B6A186000202F
:10A32000BDE8F081C1780029EDD00132152ADAD1DB
:10A3300032460549034805F085F8EEE7A9170608F7
:10A34000931706087C2806087C1706082DE9F347B2
:10A3500007468846002A3BD0930739D113792F2B23
:10A3600036D1926802F00F03022B08D10F23FFF7BA
:10A37000ADFF01248440204602B0BDE8F0873AB327
:10A3800012F0030A24D113799F2B21D1D5682B79A0
:10A39000A12B1DD10F239268FFF798FF012606FA23
:10A3A00000F401AAA22105F10800F9F767F8814637
:10A3B000CA45E0DA019A0F2352F82A20414638466E
:10A3C000FFF784FF06FA00F004430AF1010AEFE701
:10A3D00042460449044805F035F87B6A00241860B9
:10A3E000C9E700BF821706087C280608F0B585B0CB
:10A3F00005460E46104603A91F46F8F73BFE48B92E
:10A4000032460B490B4805F01DF86B6A18600020B6
:10A4100005B0F0BD039803F03FF830EA0703F7D02A
:10A420000346009732460449024805F00BF8ECE772
:10A430004E1706087C280608541706082DE9F04F29
:10A440000F4687B0044603A938461E469046F6F7E5
:10A4500060FD0378762B054640F02A81B8F1020FA3
:10A4600040F0D58040F21D539F4231D14EF6B46882
:10A470004FF42C6906E04EF6B168F9E74EF6B16884
:10A480004FF42469326829462046FFF7EFFE7268D0
:10A49000074629462046FFF7E9FEFB02420102F08B
:10A4A000200203F470431343B90143EA0903C0F3E4
:10A4B000430201F040011A4341EA08012046FCF73B
:10A4C000CBFF1CE14EF6B868D2E74EF6BD68CFE789
:10A4D00040F229539F42CED0B7F5A56FCED040F2BF
:10A4E0001E539F42EED040F21F539F42EDD040F2E8
:10A4F00027539F421ED13068FFF7ACFEAF4915F0DD
:10A5000055FCA8B10F23326829462046FFF7DEFE2E
:10A5100007467068FFF79EFEA94915F047FC002822
:10A5200040F0BD803A0342F421624EF6F161C5E786
:10A530000F27EEE740F226539F422ED13068FFF7F7
:10A5400089FE0378722B18D10F23326829462046E2
:10A55000FFF7BCFE2946804672682046FFF786FE5C
:10A560004EF610610746FA01D2B242EA0832C7F34A
:10A57000430742F421623943A0E732682946204666
:10A58000FFF774FE294607460F2372682046FFF73F
:10A590009DFE4FF46E418046E5E740F224539F4212
:10A5A0002ED14EF69058326829462046FFF75EFEBF
:10A5B00005AB0093074604AB726829462046FFF7B7
:10A5C000BFFD002800F09B800723049A29462046FF
:10A5D000FFF77CFE059A064629464FF47F73204616
:10A5E000FFF704FFFA02B90102F4704201F04001E2
:10A5F00042F4206241EA080142EA900231435DE7F9
:10A6000040F22A539F424AD14EF68058CBE7B8F128
:10A61000030F44D1DFF8B891002709F1010A00F1D6
:10A62000010B03220AEB8701584615F0D7FB98BBB4
:10A630002B798BBB326819F8278029462046FFF713
:10A6400015FE7268074629462046FFF70FFEB268DE
:10A65000814629462046FFF709FEFA02430102F42B
:10A66000704203F0200313434FEAC912D2B243EA07
:10A6700050031343BF014FEA0812D2B207F040075C
:10A6800008F0F00142F4206247EA590941F46E41B2
:10A690001A4349EA010111E70137042FC1D14346AA
:10A6A0002A464849484804F0CDFE636A186026E00F
:10A6B000B8F1000F10D140F247439F4205D14FF44B
:10A6C0003F412046FCF7BEFE19E040F22D539F4269
:10A6D000E5D14BF63071F4E7B8F1010F40F0FD80A1
:10A6E000B7F5537F0ED1014632682046FFF78CFD47
:10A6F00001462046FCF738FF002800F0628307B0CF
:10A70000BDE8F08F40F25332974209D101463268DA
:10A710002046FFF779FD01462046FCF778FFEBE77E
:10A7200040F25D32974209D101460F23326820463C
:10A73000FFF7CCFDC10041F48E41C2E7622B49D145
:10A74000039B032B0CD0052B40F09480C3785F2B28
:10A7500040F0908003796E2B02D0772B40F08A80F6
:10A7600095F801C0194A00234FF0FF3703EB43016E
:10A77000501890F801E0E64505D195F802E08078A0
:10A78000864508BF8F5C01330E2BEFD1781C86D035
:10A79000326829462046FFF737FD039B052B02460A
:10A7A00009D12B79A3F177014B424B413946204621
:10A7B000FCF7F8FEA0E70023F8E700BF98160608AC
:10A7C000A2160608B51606087C2806081316060801
:10A7D00022170608692B4DD14378742B4AD1306873
:10A7E000C84EFFF737FD90F800C0002237465100F1
:10A7F0008B18334493F801E0E64529D190F801E045
:10A800009B789E4524D1837813BBAE1C304603460B
:10A81000013093F800C0BCF1000FF8D1681D8342ED
:10A820003FF63DAF0A44013BBA5C12F0010F4FEA1C
:10A83000C2000CBF4FF0080C4FF0000C00F00800F5
:10A840000821B34208D241EA021141F43F4138E7FE
:10A8500001320E2ACBD122E713F80179742F4FEA87
:10A86000510101D10143ECE7652F7FF418AF4CEAA9
:10A870000101E6E740F27E339F4202D14BF2726162
:10A880001FE740F27F339F4202D14BF2626118E72B
:10A8900040F273439F420ED1326829462046FFF7AB
:10A8A00055FD10F47F4F024602D140F4344108E7D1
:10A8B0004EF62D1102E6782F7FF4F1AE326829466C
:10A8C0002046FFF743FD10F47F4F024602D140F4CB
:10A8D0003C41F6E64EF6BD01F0E5B8F1020F40F05E
:10A8E000AB81736803F00F03022B40F09D80B7F536
:10A8F000876F12D1326801460F232046FFF7E6FC2E
:10A900007268074629460F232046FFF7DFFC3946C9
:10A9100002462046FCF703FEF1E640F26D339F420B
:10A920001CD14FF6B0284FF280070F23326829461A
:10A930002046FFF7CBFC7268814629460F2320464C
:10A94000FFF7C4FC47EA000242EA092248EA000194
:10A95000B4E54FF690284FF2A007E6E740F27F43B8
:10A960009F42F6D040F23D439F422BD101463268D0
:10A970000C232046FFF7AAFC07467068FFF76AFC25
:10A9800006460146604815F011FA98B131465F4815
:10A9900015F00CFAA0B12A465D495E4804F052FD5C
:10A9A000636A0022186042EA072242F400424FF232
:10A9B000EF3183E50023584A02EBC302D25CF2E791
:10A9C0000123F8E740F23F339F4215D14FF480470F
:10A9D0003268294607232046FFF778FC72688046D4
:10A9E000294607232046FFF771FC424603463946B5
:10A9F0002046FCF78FFD82E6DFF82091002709F161
:10AA0000010A03220AEB8701284615F0E7F938B955
:10AA1000EB782BB919F827703F0147F48047D7E747
:10AA200001370F2FEDD13AE6B7F5876F1CD14FF400
:10AA300000570723326829462046FFF747FC29467E
:10AA40008046FF2372682046FFF7D0FC47EA0001EA
:10AA500041EA082135E64FF42057EAE74FF4405722
:10AA6000E7E74FF46057E4E740F26F339F42F2D0DC
:10AA700040F235339F42F1D040F2DE439F42F0D0A6
:10AA800040F23A439F4219D14FF240270F233268D8
:10AA900029462046FFF71AFC4FF6FF73804672687E
:10AAA00029462046FFF7A2FC424603463946204687
:10AAB000FCF746FD23E64FF2C027E7E740F23943B3
:10AAC0009F42F8D040F23B439F4229D101460F23D9
:10AAD00032682046FFF7FAFB294607464FF0FF335E
:10AAE00072682046FFF782FC3A4683B205464FF271
:10AAF00040212046FCF724FD2B0C3A464FF2C021A2
:10AB0000D5E700BF13160608FE1706080718060843
:10AB1000A81606087C280608FD170608CD160608A4
:10AB200040F207439F4228D101460F233268204656
:10AB3000FFF7CCFB05AB0093074604AB72682946D0
:10AB40002046FFF7FDFA00283FF4D9AD0F23049A01
:10AB500029462046FFF7BAFB059A06462946FF23F9
:10AB60002046FFF743FC3A0342F4706246F4684122
:10AB700042EA900241F05001A0E440F205439F42B6
:10AB80003FD040F206439F423DD0B7F5816F3CD0A5
:10AB9000972F3CD040F2DA439F423AD040F2DC4358
:10ABA0009F427FF47CAD0523894A294632F8237001
:10ABB000326807232046FFF789FB05AB00938146E7
:10ABC00004AB726829462046FFF7BAFA00283FF422
:10ABD00066AD049A072329462046FFF777FBFA045F
:10ABE000064618D51F23059A29462046FFF7FEFB87
:10ABF00047EA0901800141EAC60100F4F860014317
:10AC00005FE50023D0E70123CEE70223CCE703234F
:10AC1000CAE70423C8E73B04059A06D53E23294624
:10AC20002046FFF7E3FB4008E2E77C232946204665
:10AC3000FFF7DCFB8008DBE7B8F1030F7FF42FADF3
:10AC400040F217439F4221D100270723326829464B
:10AC50002046FFF73BFB07238146726829462046C2
:10AC6000FFF734FB294680461F23B2682046FFF7D2
:10AC7000BDFB47EA090747EA801747EAC80120E514
:10AC80004FF40067E1E74FF48057DEE7B7F5836FD5
:10AC9000F6D040F247339F42F5D040F235339F4221
:10ACA0002BD14FF4C0580723326829462046FFF7BE
:10ACB0000DFB07237268074629462046FFF706FB6F
:10ACC000B26802F00F03022B81460ED107232946FA
:10ACD0002046FFF7FBFA47EAC90747EA080747EAB1
:10ACE0008011EEE44FF4D058DDE7072329462046D3
:10ACF00048F48068FFF77AFBEDE740F2B1439F42EA
:10AD000022D14FF690370F23326829462046FFF7AD
:10AD1000DDFA0F238146726829462046FFF7D6FAEE
:10AD2000B268804629460F232046FFF7CFFA40F449
:10AD3000704242F0F00242EA092247EA0801FFF7B6
:10AD4000BDBB4FF6B037DEE7B7F5A06FF9D040F2E4
:10AD5000DE439F42C6D040F2DB439F427FF49FAC6C
:10AD600001460F2332682046FFF7B0FA0F237268BE
:10AD7000294607462046FFF7A9FA05AB009380460F
:10AD800004ABB26829462046FFF7DAF900283FF401
:10AD9000B6AC0F23049A29462046FFF797FA059A86
:10ADA00006462946FF232046FFF720FB3A0242EAE7
:10ADB000083246F4684142EA900241F04001FFF750
:10ADC0007DBB04490448646A04F0B0FA206096E44C
:10ADD0000A170608C21606087C28060804292DE969
:10ADE000F04106460C46904625D9446A134914485A
:10ADF00004F09CFA206000242046BDE8F0810009A0
:10AE0000F6F782F8074614F0C7FF022810D13B7806
:10AE1000722B0DD17A7805F130039A4208D10135B1
:10AE2000A542E9D058F8250000F00F03022BE6D028
:10AE3000746A0449DBE70025F2E700BF3D16060807
:10AE40007C2806086616060838B505463020F5F752
:10AE500023F920220446002114F068FF29462046E9
:10AE6000FCF79DFAA562A800F5F716F9E062204606
:10AE700038BD10B50446C06AF5F736F92046002102
:10AE8000FCF795FA2046BDE81040F5F72DB90129E9
:10AE900010B5146824D934F01001037815D1302B83
:10AEA0001ED1417841F02001782900F1020303D13D
:10AEB00010211160181A10BDACB96F2901D10821F9
:10AEC000F7E762290DD10221F3E7082C0DD1302BD1
:10AED00009D1437843F020036F2B04D1831CE9E7A9
:10AEE0000CB90A2313600346E4E7022CFBD1302B94
:10AEF000F9D1437843F02003622BEEE708B5102028
:10AF0000F5F7E3F80278012161F30202027008BD4F
:10AF100030B50478022565F302040470048863F3F5
:10AF2000C9040480C0E9011230BD037861F3020353
:10AF300003700388029961F3C903038003680199D0
:10AF400061F39423C0E90032009B8360039BC360DC
:10AF50007047000038B5044608462378656803F05A
:10AF60000703032B114603D3042B0AD9052B12D058
:10AF7000A3682A4604F048FF23881B070AD50A4B1A
:10AF800007E0A3682A4604F06DFF23881A0701D55D
:10AF9000064B036038BD2068E2682946C0F38A206A
:10AFA000BDE8384004F066BFA82D0608E42D060869
:10AFB00038B5154611F480720C4614BFD5E900125D
:10AFC0001146FFF7C7FF620902F008022A44E1B206
:10AFD000BDE8384003F0D6B92DE9F04303685A1CA8
:10AFE00002601B780022C3F3C304C3F3800E03F096
:10AFF0000307154616469446D0F800801B0608F154
:10B0000001091ED4C1E9046501340022C1E9004EE2
:10B01000C1E902C71346144606270568691C01608A
:10B020002D7805F001069640334307FB02FCC5F37B
:10B03000450606FA0CF62D0644EA06042DD5013223
:10B04000EBE7C0F8009098F800304FEA420903F0AF
:10B05000300808FA09F844EA080403F0020808FA7C
:10B0600002F84EEA080EC3F3801808FA02F84CEA18
:10B07000080C03F0040808FA02F847EA0807C3F3CB
:10B08000C00808FA02F846EA080603F0010808FAC0
:10B0900002F845EA08050132AEE723440B44036099
:10B0A0000846BDE8F08302884B0803F4806322F46D
:10B0B000816243EA113322F007021343038043887D
:10B0C0000A0103F4706302F4E0421343C9B2194366
:10B0D00041807047D0E90003184770B505460C461B
:10B0E0008E18B44200D170BDD5E90003984704F82A
:10B0F000010BF6E770B506460C460025D6E90003BD
:10B10000984724B12368187023680133236000F046
:10B110007F0343EAC5150306F0D4284670BDF8B591
:10B120000C4600210746FFF7E5FF20B93846BDE889
:10B13000F840FFF7CFBFC3074FEA500528D5238853
:10B140005A1B02F01F0204EB420193424E8835461F
:10B150000ED2911C6FF001034900C8185A433E32C9
:10B160002144204414F0CAFD6388A4F84030002232
:10B170002388501C40009A1A811C2144204452000C
:10B1800014F0BCFD238804EB430466802846F8BD18
:10B190002846F4F781FF2A46064601463846FFF75F
:10B1A0009CFF29463046F5F707FE05463046F4F782
:10B1B0009BFF2388013303F01F03238004EB430428
:10B1C0006580E3E72DE9F843244F0646884691461B
:10B1D00000243068FFF77EFFC5B2FF2D01D1BDE826
:10B1E000F883C2070FD500213068FFF783FF10F006
:10B1F000010F18BF73684FEA500416BF586808EB78
:10B20000840400EB84046B08052B0FD8DB070BD5F7
:10B2100000213068FFF76EFFAD081CD0736853F84B
:10B2200025300246214610E00120F5E7062B1BBF22
:10B2300003F18043073B3B4657F823300120F0E7FA
:10B2400051F8045B1D4441F8045C12F1FF32F7D25F
:10B2500004EB8004BDE74B46E3E700BFFC1906089A
:10B260002DE9F04F0F4697B000210446FFF742FF4B
:10B2700000F00305AB1C05931C22830800210FA8D6
:10B28000089314F053FDAB1C022B089840F0AA80E1
:10B29000F4F702FF0DF15808064648F82C0D0A9005
:10B2A00041462046FFF726FF41462046FFF722FF92
:10B2B0000FA90AA8FFF790FE394620460B9DFFF71D
:10B2C0002EFF2870000A687039462046FFF727FFD6
:10B2D000A870000AE8700B990A9A0431521A2046A5
:10B2E0000B91FFF7FAFE089B0A9D06EB0309A9459F
:10B2F00049D800212046FFF7FDFE00218246204666
:10B30000FFF7F8FE8146DDE9120318445044484433
:10B310004FF000088000F4F7BFFE4FF0000B0690DE
:10B320000546DDE9123213445B4500F20F81059BAF
:10B33000022B12D0C74B2B60119B9A0600F1128191
:10B340000435119B5B0608D500212046FFF7D2FE8D
:10B35000F4F7BBFE043545F8040C00230793079B64
:10B36000534540F0108105EB83054FF0000ACA45B4
:10B3700000F0CB8039462046FFF772FF45F82A00DF
:10B380000AF1010AF3E72046FFF7A4FE0022287025
:10B39000414628460EF08EF80B9B012803F1FF333F
:10B3A00005F1010A0B9313D139462046FFF7B7FE8A
:10B3B0006870000AA8700B9B023B05F1030A0B930F
:10B3C0000B9A51462046FFF788FE0B9D55448EE7A9
:10B3D0000228F5D12046FFF77DFE03060AF8010B8F
:10B3E000F8D4EDE7F4F758FE089A014606462046E1
:10B3F000FFF773FE032D36D1059B032B6FD1002180
:10B400002046FFF777FE331816A80FA940F82C3D09
:10B41000FFF7E2FD394605462046FFF780FE28701B
:10B42000000A687039462046FFF779FE4FF00008A1
:10B43000A870000AE87041462046FFF75BFE4146CF
:10B4400082462046FFF756FE8146DDE91230184459
:10B4500050444844119B9D064CBF023001305906B0
:10B4600048BF013056E700212046FFF743FE002584
:10B4700080464545C0D000212046FFF73BFE3946B7
:10B4800081462046FFF74BFE4FEA990319F0030966
:10B4900006EB030A05D1F054000A8AF801000135D1
:10B4A000E7E7B9F1030F05D1C00040F00200CAF888
:10B4B0000000F4E7B9F1020F0ED1C00040F002091C
:10B4C0001FFA89F15046FFF7EEFD4FEA19410AF1E4
:10B4D0000400FFF7E8FDE2E781B25046F9E70021FA
:10B4E0002046FFF707FE059B11900025052BCDE9AF
:10B4F000125519D129462046FFF7FCFD2946129026
:10B500002046FFF7F7FD06958046FFF7F7FC059B01
:10B51000022B054675D1119B069A3146FFF7F8FCC0
:10B52000284617B0BDE8F08F00212046FFF7E2FD66
:10B53000002182462046FFF7DDFD8146DDE912034A
:10B540001844504448444FF0000883E739462046E9
:10B55000FFF7E5FDC00040F0020045F8040B0BF1D9
:10B56000010BDEE600212046FFF7C4FD0790F4F74B
:10B5700093FD079A834601462046FFF7AEFD083546
:10B5800045F804BCDDE62046FFF7A4FD5FFA80FB2A
:10B59000BBF1650F33D000212046FFF7ABFD01461C
:10B5A00009900BA8F5F7AEFD099A0D992046FFF713
:10B5B00094FDBBF1730F0BD0BBF1620F0AD126488B
:10B5C0000BA907F009F9079B45F823000133C5E6ED
:10B5D0002248F5E7BBF1690FDDE90C104FF00003DD
:10B5E00003D10A22D7F776FCEDE7ABF1630CDCF16F
:10B5F0000002009342EB0C02D7F7EAFCE3E718489D
:10B60000E1E7069B0C93119B0B94DB0612D5154CBE
:10B61000D4F8C41021B9084605F006FDC4F8C400EA
:10B620003146D4F8C40005F0ADFA324631460BA8D5
:10B63000FFF7C8FD119B0293129B0193069B009399
:10B64000CDF80C80089B059932462846FFF76DFC23
:10B6500066E700BFFC1906085C3906080C3C0608C2
:10B66000FC3606082C1B002030B593B00422694636
:10B670000446FFF732FD9DF800304D2B02D01748ED
:10B6800000F0EEFE9DF80130052BF8D19DF8023058
:10B6900003F00303022BF2D19DF803301F2BEED8E9
:10B6A00000212046FFF726FD2028E8D89DF802302B
:10B6B0009B0804D0043B032B01D90948E0E712A9F9
:10B6C000002321F8443D2046FFF7CAFDA368054644
:10B6D00020689847284613B030BD00BF6718060899
:10B6E000731806081FB5014601A813F021FA01A836
:10B6F000FFF7BAFF05B05DF804FB0000F8B51A4C7F
:10B7000000250127F5F71CFBE564A4F8F651A4F821
:10B71000F47103F0A7FD154B656304F19006C4E9CD
:10B720000B350321124BA36304F13C00C4F8E8512C
:10B7300084F8EC5103F0A4FB3946304603F0A0FB3B
:10B74000AA22BA21304603F024FCC4E90266C4E907
:10B750003055C4F8C851C4F8CC51C4F8D051C4F81D
:10B76000D451C4F8D851F8BD2C1B0020242606085B
:10B77000A03E060808B5084BD3F8C00008B9074832
:10B7800008BD002240F27A51043001F0AFFB0028DE
:10B79000F5D04068F4E700BF2C1B0020704306087A
:10B7A000034BC0000A4640F00201986803F0F1BB69
:10B7B0002C1B0020034BC10041F00201986803F0EC
:10B7C000F6BB00BF2C1B0020034BC0000A4640F014
:10B7D0000201D86803F0DDBB2C1B0020034BC10025
:10B7E00041F00201D86803F0E2BB00BF2C1B00202F
:10B7F000F8B51C46930707460E46154609D113684F
:10B800009A88910617D5530612D5F268124B9A42C0
:10B8100001D12560F8BD58B9104B9E4208D00C20CC
:10B82000F4F73AFC0E4B8560C0E900362060F1E782
:10B83000C4E90057EEE70B4A934202D16B682360DC
:10B84000E8E7094A9342E4D110B101F071FD0646E0
:10B850006B68C4E90036DDE731530308143206088B
:10B860007C1906082C400608F03F060800232DE945
:10B87000F041C2E900330D460746144601F058FD79
:10B880000A2D064602D12060BDE8F081192D05D1B0
:10B89000836A1BB10F4BC4E90037F5E7F3692BB19D
:10B8A000224629463846BDE8F0411847B06B0028CB
:10B8B000EAD0E9001A4641F00201043001F016FB1B
:10B8C0000028E1D02346426831463846BDE8F041C1
:10B8D000FFF78EBF64440608F0B593B0054668468E
:10B8E0000E4617461C46F4F79BFB40B93A463146D4
:10B8F0002846FFF7BBFFF4F78BFB13B0F0BD002C1D
:10B90000FBD1019B0449186809F0C6FE0028F4D158
:10B910000198F4F79DFB00BF0824060870B5456840
:10B920000024AB68A34200D870BDEB6853F8340024
:10B93000E60078B104280DD007F08EFC03785F2B69
:10B9400008D0EB68985907F06FFCEB6833445968EE
:10B95000FFF726FF0134E4E708B519B903F0D6FC78
:10B96000F4F776FB03F0E2FCFAE70EB403B503AAA2
:10B9700052F8041B019203F003FDF4F769FB000089
:10B9800070B5114EC4000546F06844F00204002270
:10B990002146043001F0AAFA40B9D6F8C0303BB1D4
:10B9A00002462146181D01F0A1FA08B1406870BD99
:10B9B00000222146054801F099FA0028F6D12A46CE
:10B9C00003490448FFF7D1FF2C1B0020FC44060864
:10B9D0001B190608D82606080A4B10B50446D3E9F9
:10B9E0000203984207D0E100002241F00201043036
:10B9F00001F07CFA20B92046BDE81040FFF7C0BF37
:10BA0000406810BD2C1B0020032837B505460C46A6
:10BA100007D1084601F0AEFE00B30E24204603B065
:10BA200030BDCA072ED54B10082829D801A252F8DC
:10BA300020F000BF1DBA020865BA020881BA0208E8
:10BA400081BA020859BA020881BA02081DBA02086E
:10BA500061BA02081DBA0208002BDED01E24DDE701
:10BA6000002BDBDAB3F1404F05D14FF0804004F0FA
:10BA700054FE0446D2E75C42640044F00104CDE782
:10BA8000DC43F9E7062821D101F00703022B0CD093
:10BA90008B071BD10B689A691C4B9A4216D14868D8
:10BAA00040B98B680193C8680CE0CC082046F5F7D4
:10BAB00021FA18B1400040F00104AFE701A9204687
:10BAC000F5F727FA0199F5F72BF9F3E7204601F08E
:10BAD0002FFC43694BB9082D0DD1204601F034FCF1
:10BAE0000B4902460B48FFF740FF2146284698477E
:10BAF0000028BED1EFE7084B20465D5D01F024FC35
:10BB00002A46034605490348FFF72FFFC9320308B9
:10BB1000B8190608F4280608E0400608BF19060808
:10BB20002DE9F04104460E461746984601F000FC08
:10BB300005693DB143463A4631462046AC46BDE82C
:10BB4000F0416047204601F0FFFB024902460248EF
:10BB5000FFF70BFFF4180608F428060800231A461E
:10BB60001946FFF7DDBF00002DE9F041194C96B0F2
:10BB70001646E26800928046A268019204A80F4629
:10BB8000C4E90236F4F74CFA2546E0B9D8F800408B
:10BB90003A46414602A8F7F785FCB7FA87F22146F4
:10BBA000520902A8FAF776FD044616B1FFF7D6FF50
:10BBB0000446F4F72DFA009BEB60019BAB60204636
:10BBC00016B0BDE8F081009BE3600598019BA3607F
:10BBD000F4F73EFA2C1B002007B502AB002243F815
:10BBE000041D0121FFF79CFF03B05DF804FB07B5BE
:10BBF000CDE900126B4600220221FFF791FF03B04E
:10BC00005DF804FB30B454680034154618BF0124B5
:10BC10006FF0030303FB042308330A462118286846
:10BC200030BCFFF77DBF000010B5044603F018FCE0
:10BC300038B1002320461A461946BDE81040FFF7E8
:10BC40006FBF204603F022FC28B904490448BDE830
:10BC5000104003F06BBB204610BD00BF381906082A
:10BC6000F42806087FB50623C000CDE902330F4B48
:10BC700040F002000190D3F8C000CDE9041278B181
:10BC8000002240F2EA51043001F030F940B101AB3A
:10BC9000002205214068FFF743FF07B05DF804FB71
:10BCA00001A905200AF094FCF7E700BF2C1B002037
:10BCB00070B5164604460D46FFF7D8FD336893B9B4
:10BCC000A30709D12268084B9A4205D1E2880749A7
:10BCD0002B460748FFF749FE204601F035FB2B466F
:10BCE00002460449F5E770BDA44006082719060876
:10BCF000082406083019060807B56A46FFF7D8FF7A
:10BD0000DDE9000111B903B05DF804FB02F0D4FADB
:10BD1000F9E700002DE9FF411D4606460C4617468F
:10BD200001F006FB324B984208D12B463A46214699
:10BD3000304604F041F904B0BDE8F081D0F8288025
:10BD4000B8F1000F08D0062C21D13046C04728603A
:10BD5000003018BF0120EEE7062C18D101AA1921E6
:10BD60003046FFF783FD019B6BB901AA8A2130465B
:10BD7000FFF79EFF039401AA00210120FFF742FF75
:10BD800028600120D7E701AA41464046F6E7002C8B
:10BD9000EBD1384601F0CCFA164909F07DFC01AA36
:10BDA00068B147213046FFF761FD019B7BB101AAD5
:10BDB00021462046FFF726FF28602046BBE79B214F
:10BDC0003046FFF753FD019B0BB10397D3E70A49B8
:10BDD000384603F062FB30B10849094803F0A6FA7F
:10BDE00028600220A7E73846FFF71EFFF8E700BFEC
:10BDF0006C2D0608F8240608402806086419060871
:10BE0000C827060873B505460C46164601F090FA99
:10BE1000C36943B10422CDE9002621466A4628467B
:10BE20009847009B43B1284601F08EFA234602460C
:10BE300002490348FFF799FD02B070BD30190608AA
:10BE40000824060873B505460C4601F071FA174A36
:10BE5000436A9342064627D063B134B9144A9342E9
:10BE600003D01020F4F718F90446736A21462846D7
:10BE7000984778B96A460F212846FFF7F7FC009BE0
:10BE800053B11CB91020F4F707F90446214668465F
:10BE900004F090F902B070BD284601F055FA05494A
:10BEA00002460548FFF761FD2846F3E739D9020845
:10BEB000A5500308FA180608F428060837B5044602
:10BEC00001F036FA856A1DB12046A84703B030BD9F
:10BED0006A4619212046FFF7C9FC009B2BB16A4630
:10BEE00029462846FFF78EFEF0E7204601F02CFA9F
:10BEF000024902460248FFF738FD00BF0D19060847
:10BF0000F428060830B5054695B000F0FBFE28463B
:10BF100001F00EFA846A2CB12846A0470446204658
:10BF200015B030BD6A4619212846FFF79FFC009BDB
:10BF3000ABB102A8F4F774F8014630B96A46FFF7CE
:10BF400061FE0446F4F764F8E9E7039B08491868C2
:10BF500009F0A2FB0028E2D10398F4F779F828460B
:10BF600001F0F2F9034902460348FFF7FEFC00BF67
:10BF7000402806080D190608F42806082DE9F04F98
:10BF80008BB01368029300284ED102F104090446D5
:10BF9000C1F307235FFA81F800935B0008EB03020B
:10BFA000019359F822A009EB82025768002F3FD075
:10BFB00017F003003CD13968834A914202D13846D8
:10BFC00002F0E4FF009B1D186D004FEA880BBAF1E8
:10BFD000000F2FD108F101000544A800F4F75CF828
:10BFE00006460CB10460012406EB84005A4649461B
:10BFF00013F058FE4444009B09EB0B01DA0006EBFA
:10C00000840013F04FFE019B23449846002F00F05C
:10C010008A8017F0030340F0968039686A4A91429B
:10C0200040F091801D467BE002F108095468AFE7BB
:10C030000020C7E71AF0030F2AD1DAF8002063497D
:10C040008A4202D062498A4222D106AA05A95046F4
:10C0500001F0ECFA059B013343441D44A800F4F7BA
:10C060001BF806460CB1046001245A46494606EB0B
:10C07000840013F017FE059A069908EB040092005D
:10C0800006EB800013F00EFE059B43441C44B2E710
:10C0900008F104000544A800F3F7FEFF06460CB1C2
:10C0A000046001245A46494606EB840013F0FAFD69
:10C0B000504606A9FFF7C6FE444482464FEA84086C
:10C0C0005046FFF71FFF0246002894D0A54207D82C
:10C0D000E90030460392F3F7FAFF039A06466D0033
:10C0E00046F80820013408F10408E9E7FB6853F832
:10C0F00035004FEAC50990B1042810D000F00703BD
:10C10000022B01D007F0C2FF46F82800FA684FEA78
:10C1100088034A44334452685A6008F102080135E2
:10C12000BB689D42E2D3A8EB040221463346520885
:10C130000298FFF7F5FC04463046F3F7D5FF20469A
:10C140000BB0BDE8F08F06AA6A213846FFF7B0FDB4
:10C15000002106AA0846FFF755FD0021FFF772FEF1
:10C160004FEA880982465046FFF7CCFE83460028F6
:10C17000D9D008F101039D4208D86D00042D38BFC5
:10C1800004253046A900F3F7A2FF06460BF007038B
:10C19000022B03D0584607F079FF834606AA0F21E9
:10C1A0003846FFF785FD06AA00210120CDF820B012
:10C1B000FFF728FD06EB090346F809B008F102086D
:10C1C000586009F10809CEE798220608AC3E060837
:10C1D0002C300608F0B5830787B00C4615461BD1F6
:10C1E00003681F4A934202D01E4A934214D102AA06
:10C1F00001A901F01BFA019BA3422BD31CD8029B7F
:10C20000043D03EB84049C4201D107B0F0BD54F817
:10C21000042D45F8042FF6E702A9FFF713FE0023CB
:10C22000064601936FF04047019BA342304606D378
:10C23000FFF768FE0028E8D022460B490CE0FFF724
:10C2400061FE38B1019BFA1A2244013345F82200FD
:10C250000193E9E7019A05490548FFF786FB00BF0E
:10C26000AC3E06082C300608DD190608C819060879
:10C270006C2906082DE9FF4183071546CFB2C1F3AB
:10C28000072435D10368394A934202D0384A934291
:10C290002ED10290029803AA01A901F0C7F90198D2
:10C2A0003B1983425CD80399002601EB8003A64228
:10C2B00013D1BC00C01B2144801B04F0B5FE0399C0
:10C2C00045F8260005EB86080B1942468B420AD139
:10C2D0000023029304B0BDE8F08153F8042D45F823
:10C2E00026200136E3E753F8040D42F8040FEDE78A
:10C2F0000021FFF7A7FD002380460193019BBB426D
:10C3000019D30021084604F08FFE06464046FFF789
:10C31000F9FD0146D0B9B168A14221D345F82460A6
:10C3200005EB810205EB8403091BAB4212D13046B9
:10C3300004F095FECEE74046FFF7E4FD80B1019B97
:10C34000FA1A2244013345F82200D6E7304604F0B9
:10C3500019FCDBE7D01AF468205843F8040DE4E731
:10C36000019A04490448FFF700FB00BFAC3E0608F1
:10C370002C300608C81906086C2906082DE9F04F6C
:10C3800085B000AF07F1080204460D46FFF76EFACC
:10C39000FB6823B12A4626492648FFF7E6FAB86823
:10C3A000002840D120460AF09FFA0028F2D007F179
:10C3B000080220461721FFF759FA391DB86806F020
:10C3C00065FF83462846F4F79AFDD7F8048008F104
:10C3D000010400EB040909F10E0323F00703ADEBA0
:10C3E000030D6B464FEAD30A4FEACA064246594646
:10C3F000304613F057FC2E2308F83A302846F4F75D
:10C4000083FD80462846F4F77AFD344402464146CF
:10C41000204613F047FC49463046F4F7CDFC012294
:10C420001E21FFF71FFC1437BD46BDE8F08F00BF8B
:10C43000071906083425060808B50446F3F7FAFE7E
:10C4400018B104490448FFF787FA22460349024815
:10C45000FFF78BFA851806089C260608A11806081F
:10C46000014608B50148FFF777FA00BF6C290608B6
:10C470002DE9F047072886B080468946164603D145
:10C4800091421BD00E2709E0022801D0052809D1CE
:10C4900032464946404601F095F90746384606B00F
:10C4A000BDE8F087082829D1104602F0D9FF38B13D
:10C4B0003146484602F0F1FF0028E3D01E27EDE7A1
:10C4C00016F0030440F03E813268BD4B9A4240F0C2
:10C4D000398106F108077368A342D3D957F8045B82
:10C4E000284602F0BDFF002800F064812946484636
:10C4F00002F0D3FF0028E1D10134ECE711F0010F85
:10C5000000F03E8112F0010A4FEA610500F0098156
:10C510005410232800F21681DFE810F0F300F70032
:10C520001401FB00FF001401140114011401240084
:10C530003000330036007A00820085008800140144
:10C5400094009D00AD00B50024003000330036009B
:10C550007A00820085008800140194009D00AD00DF
:10C56000B500DB0045EA040A4FEA4A0797EA0A0FDA
:10C5700065D55046C11704F0C0F88EE785EA040A75
:10C58000F2E705EA040AEFE7002C02DA8D48FFF72C
:10C5900067FF1F2C09DC6FF040432341AB4204DBF3
:10C5A0004FF040432341AB422FDD2846E91704F00A
:10C5B000A4F88146484600F0BBFE8369002B40F09A
:10C5C000E880A8F116030C2B40F2EC80B8F1240FA0
:10C5D00006D94B46A8F10F08B1465FFA88F81E4607
:10C5E000B8F1240F40F0AE8002A94846FFF72AFCBC
:10C5F00004462046FFF786FC00283FF443AF31464F
:10C6000001F056F90028F4D058E705FA04FAABE730
:10C61000002CBBDB1F2CA8BF1F2445FA04FAA3E79C
:10C6200005EB040AA0E7A5EB040A9DE7214628468E
:10C630000DF030F90028B8D104FB05F77F0047F072
:10C6400001072BE7002C00F0B780214628460DF0AB
:10C6500052F9824688E7002C00F0AE8007EE905A2F
:10C66000B8EEE70A07EE904AF8EEE77A80EE270A7E
:10C6700003F040F811E7002C00F09E802146284688
:10C680000DF02BF9E5E7002C21DA07EE905A114660
:10C69000B8EEE70A03F094F8FFE6E20708D539465A
:10C6A00050460DF0F7F800287FF47FAF07FB0AFA39
:10C6B000012C3FF459AF3946384664100DF0EAF8C2
:10C6C00000287FF472AF7F43002CE6D14CE72F4661
:10C6D000FAE7002C70D00021022008F04FF8214624
:10C6E000074628460DF007F9400040F00100B86009
:10C6F000214628460DF0F1F8400040F00100F860B6
:10C70000CCE6A542FFF6DAAEBCE6A5423FF7D6AED0
:10C71000B8E6A5427FF7D2AEB4E6A542BFF6CEAEEC
:10C72000B0E693072CD11368274A93421BD107EE3A
:10C73000905A3146B8EEE70A03F042F8074600285F
:10C740007FF4ACAE214B484613F8084000F0FCFDE6
:10C750000546304600F0F8FD2B46009022461C4965
:10C760001C48FFF702F91C4A934209D107EE905A80
:10C770003146DFED1A0AB8EEE70A01F04DFFDDE7BA
:10C78000B8F1060F01BF4B464FF02408B1461E46D4
:10C7900010E73246494640469847074600283FF48E
:10C7A00010AF7BE64B4608F10F08B1465FFA88F8F8
:10C7B0001E46FFE62E46C5E709490A48FFF7CCF8B2
:10C7C000AC3E0608C01806086C2A06082E3F06086C
:10C7D000D5180608F42806083420060800000000D2
:10C7E000E8180608E4290608014608B50148FFF7DD
:10C7F000B3F800BFF42806082DE9F04104461746B7
:10C800001E460D4641B1186800F092FD63688342F0
:10C8100002D00548FFF7E8FF33463A462946A068AC
:10C82000BDE8F041FFF77CB97F180608410008B564
:10C8300041F00101024802F06EFDF3F709FC00BF70
:10C8400050270608014608B50148FFF785F800BFE4
:10C850001427060808B540F22A71024802F05BFD71
:10C86000F3F7F6FBC827060830B593B004466846D0
:10C870000D46F3F7D5FB48B920462946FFF7ACF93A
:10C880000446F3F7C5FB204613B030BD01990248BA
:10C8900000F084FD0024F6E7E8080608064B03F1E3
:10C8A0002C02DA64B3F8F42112B20021012A596390
:10C8B00008BFA3F8F41170472C1B0020EFF3108180
:10C8C00072B6084AB2F8F4311B0443BFB2F8F4312F
:10C8D00003F1FF331BB24FF6FF73A2F8F43181F37B
:10C8E000108870472C1B0020EFF3108172B60C4BA0
:10C8F000B3F8F421013212B2A3F8F42118463AB980
:10C90000DA6C12B993F8F6212AB10023A0F8F431B9
:10C9100081F3108870470122A3F8F421F8E700BFE3
:10C920002C1B002070B5124B93F8F6414FF6FF72A6
:10C93000A3F8F421CCB193F8F72102F10A0103EB3B
:10C94000C106013202F00702013C53F83150716810
:10C9500083F8F72183F8F64180F310882846FFF723
:10C9600083FFBDE87040FFF7BFBF80F31088F8E792
:10C970002C1B0020114BB3F8F42112B210B5044661
:10C98000DAB9EFF3108172B6B3F8F42112B292B9AA
:10C99000D86C58B1DA6493F8F62112B90122A3F8E1
:10C9A000F4211CB181F31088F3F752FB0846BDE86F
:10C9B0001040FFF7B7BF81F3108810BD2C1B00207B
:10C9C00070B5EFF3108572B60F4B93F8F621082A75
:10C9D00018D0B3F8F44124B2012C04BF0024A3F80A
:10C9E000F44193F8F741561C224402F00702093241
:10C9F00083F8F66103EBC203C3E90201012085F36A
:10CA0000108870BD0020FAE72C1B002038B1044AC2
:10CA1000D368984202D0D060184670470020704713
:10CA20002C1B002001F00F01012905D003D302299E
:10CA300007D103F072BE7047002814BF1E200E20DD
:10CA4000704703F0EDBE08B500F08AFD10EE100A45
:10CA50002EF048FC41EC100B08BD00F081BD08B57C
:10CA600051EC100B2EF096FCBDE8084000EE100AC9
:10CA700002F040BE02F03EBEF0B593B005466846F7
:10CA80000F4614461668F3F7CBFA78B9002E0CBFA0
:10CA900039460021234632462846FFF73BF9054632
:10CAA000F3F7B6FA012D0BD1284611E0019B236064
:10CAB0001049206802F0F1FC60B92068F3F7C8FA69
:10CAC0002368002DF4D10BB9062323603EB9002062
:10CAD00013B0F0BD206802F0E9FB2060F6E70649DC
:10CAE000304602F0DAFC0028F1D03046FFF79CF81F
:10CAF000E4E700BF40280608F8240608036803B9E5
:10CB00004068FFF7FFB91346C1F30722C9B2FFF728
:10CB100007B81FB501F00F010446032907D8DFE865
:10CB200001F004020D0D00F025FE04B010BD01223D
:10CB300001A900F002FF08B10198F6E7204600F0D5
:10CB4000ABFCF2E708B528B1062803D0FFF76CF874
:10CB5000F3F77EFA08BD10B50C4619B9BDE81040D0
:10CB6000FFF770B9FFF76EF984421CBF0023C4E9D8
:10CB70000030002010BD40F26C4398421CD007D812
:10CB80005E2815D075281FD03E280ED10120704791
:10CB900040F26E43984215D012D340F26F43984250
:10CBA0000CD040F20453984204D04FF0FF3070474D
:10CBB000022070470320704704207047052070470B
:10CBC00006207047072070470020704738B503469D
:10CBD00015460C4609B92C460BE052B111462046C9
:10CBE000984758B1636833B9656044F00103A560A4
:10CBF000EB60204638BDA368DD60F6E76B68E36054
:10CC00006C60002BE7D145F00103AC60E360E2E724
:10CC1000F8B5064631B1002511F0010304D0002318
:10CC2000EB6029460846F8BDCC68CB6014F00103E0
:10CC300007D1E768E36022463046FFF7C7FF3C466E
:10CC400001460A4630462946FFF7C0FF2146054601
:10CC5000E2E78A422DE9F04103460F4606D1002360
:10CC600051685360BDE8F041FFF7D2BFD66896B176
:10CC70001446E468E107FCD524F0010406F001083D
:10CC80006568954218D15168002039B9804518BFB0
:10CC90000E466660D1603846BDE8F0815060D060D5
:10CCA0001846FFF7B5FF05466060EE60B8F1000F6B
:10CCB000F1D0A560EFE70D46E9689142FBD1002075
:10CCC0005168D06050601846FFF7A2FF0028ECD0F2
:10CCD000E8600546E9E70000014B1860704700BFB7
:10CCE0002C1B0020034B82B0186801ABC01A02B0A5
:10CCF000704700BF2C1B0020014B5860704700BFDD
:10CD00002C1B002007B5064A1368526801A95B1A5C
:10CD10009A4201D8FFF79EFD03B05DF804FB00BF07
:10CD20002C1B002010B503461446500CC2F34F02D2
:10CD300021B1E10702D40C48FFF756FD904206D11D
:10CD400098420FD0094902460948FEF70EFE984264
:10CD500004D9C21A07490648FEF707FE9A4201D2D3
:10CD60000549F1E710BD00BF3C1B0608461B06083D
:10CD7000F4280608581B0608601B06082DE9F74F23
:10CD8000DDE90CA5002481468B469046019326469A
:10CD90002746019B9C4204D14F453AD22248FFF7D7
:10CDA00023FD4C450FD2BAF802209205F6D45BF869
:10CDB000240001379AF80220012A23D100F0DAFC7E
:10CDC00005F8240017E0BAF80010C900002241F06D
:10CDD0000201404600F08AF888B9BAF80220D3056B
:10CDE00005D5BAF8002011491148FEF7BEFDDAF862
:10CDF000042045F8242001340AF1080AC9E7013665
:10CE00004068D7E7022A01D100F028FB45F824004A
:10CE1000F1E7D8F80030B6EBD30F01D20548BEE7F2
:10CE200003B0BDE8F08F00BF9A1B0608951B0608EB
:10CE3000F4280608A41B060870B586B004461546FB
:10CE400002EB800203A81E4600F01FF80B9B019323
:10CE50000A9B009303AA334629462046FFF78EFF1C
:10CE600006B070BD08B50148FFF7ECFC6D1B060865
:10CE700010B50446416019B981600123236010BDDB
:10CE8000C800F3F722F9A060F7E70368416061F397
:10CE9000DF030360DBB243F0070303708260704777
:10CEA00003789B0710B5044602D48068F3F71CF999
:10CEB0002368002262F3DF036260236010BD037801
:10CEC0009B0710B5044602D48068F3F70DF9236878
:10CED000002262F3DF032360DBB243F0010362F35D
:10CEE000410362602370A26010BD000003782DE949
:10CEF000F74F13F0010904460E46924610D001F098
:10CF00000702022A0AD011F0030903D109687E4AF8
:10CF1000914205D0BAF1010F40F0F3804FF00109C2
:10CF20005B0762D52768A56827F007072F44BD4235
:10CF300030D3BAF1010F40F0E48021686368C1F397
:10CF4000DC01994211D104316160A068C900F3F796
:10CF5000BEF823686268A060C3F3DC03D21AD20073
:10CF6000002100EBC30012F0E1FE2368A168C3F3C7
:10CF7000DC02501C60F3DF03236041F8326006F0EE
:10CF80000706022E01EBC20521D023786FF30003C0
:10CF900023701CE02868B0421DD1BAF1020F16D1EF
:10CFA00023686E687A1B083B22F0070205F108012E
:10CFB0002360083A284612F0A1FE2368A268C3F352
:10CFC000DC0302EBC305002142F833106E602846F3
:10CFD00003B0BDE8F08FB9F1000F04D1314600F085
:10CFE00067FC0028D9D10835A1E7636833B9BAF1E5
:10CFF000010F40F08680204600F088F806F0070B0D
:10D00000BBF1020F28D1F008F3F774FF0246636802
:10D01000B2FBF3F103FB11231F464FF00008A16898
:10D0200051F8370001EBC705E0B9BAF1010F68D13B
:10D030002368C3F3DC020132B8F1000F18BF454684
:10D0400062F3DF03BBF1020F2360C5E90060BED0CD
:10D05000237860F300039BE731460620FEF7D4FCFB
:10D060004210D4E7042822D1B8F1000F08BFA84627
:10D0700061680137B7FBF1F001FB1077BB42CED1FD
:10D08000BAF1010F3DD1B8F1000F33D0236800226F
:10D090000833BBF1020F2360C8F80060C8F8042011
:10D0A00003D0237862F30003237045468FE7B04234
:10D0B00011D1BAF1020F8AD123686268083B0137A7
:10D0C0002360B7FBF2F302FB1377A36853F8373002
:10D0D00073B92B607BE7B9F1000FC9D13146CDE9B7
:10D0E000002300F0E5FBDDE900230028C0D0E0E7E5
:10D0F0000423EEE72046009200F008F86368009AE7
:10D1000086E7002563E700BF0C3C0608F8B54668D3
:10D1100019490446731C002231F81250AB4206D95B
:10D120000132222AF8D103EB530343F00105E80052
:10D13000A768F2F7CAFF236865606FF3DF03236017
:10D14000DBB243F001032370A0600025B54204D197
:10D150003846BDE8F840F2F7C7BF57F8351049B177
:10D16000042907D001222046FFF7C0FE07EBC503C4
:10D170005B6843600135E9E7AE1B060810B5002384
:10D180000446016043608800F2F79FFFA06010BD75
:10D1900003682DE9F74F04468946924623B912F0F9
:10D1A000010F67D000F068F849460620FEF72CFC16
:10D1B00022684FEA600B0AF00103BBFBF2F7009311
:10D1C00002FB17B73D464FF00008A06850F82560F5
:10D1D000AA0081186EB91AF0010F4BD06368B8F13C
:10D1E000000F18BF414601336360C1F800904E46FE
:10D1F00031E0042E16D1B8F1000F08BF884622682E
:10D200000135B5FBF2F102FB1155AF42DDD1009BB8
:10D2100083B3B8F1000F24D0636801336360C8F8AA
:10D220000090E4E749463046019200F041FB019A44
:10D230000028E4D01AF0020F0DD063682068013B8B
:10D2400001356360B5FBF0F1A36800FB115553F89D
:10D25000251021B99950304603B0BDE8F08F042164
:10D26000F8E7204600F008F82268BBFBF2F702FB63
:10D2700017B7A7E70026EEE7F8B5056886681549F1
:10D2800004466B1C002231F81200834206D9013299
:10D29000222AF8D103EB530343F00100002320605E
:10D2A00063608000F2F711FF3746A06006EB85054A
:10D2B000AF4204D13046BDE8F840F2F715BF57F849
:10D2C000041B0029F4D00429F2D001222046FFF7E4
:10D2D0005FFFEDE7AE1B060870B5016800239942B9
:10D2E00001D1002214E0846854F8232004EB830663
:10D2F0000133002AF3D0042AF1D04568013D45608E
:10D30000B3FBF1F001FB103354F8233013B9336051
:10D31000104670BD0423FAE710B504468068F2F7A2
:10D32000E3FE0023C4E90033A36010BD7047000092
:10D3300083070FBF0068034B00F00F0053F8200075
:10D34000704700BFE41C060808B5FFF7F1FFBDE811
:10D350000840C088F3F7D8BD70B50D4604461646A0
:10D36000FFF7D0FC2846FFF7E3FF83682BB1324676
:10D3700029462046BDE870401847C2880249204629
:10D38000BDE87040D6F7D8BAAC1C06080A4601467C
:10D390000148FFF7E1BF00BFF04F06082DE9F34752
:10D3A000054608460E4602F071F8A8B101AA694682
:10D3B000304602F0C7F8009B73B11A49DFF86C8061
:10D3C000DFF86C90DFF860A02846D5F75BFF009C83
:10D3D000E71EA400002F0BDA022231462846FFF791
:10D3E000BBFF11492846D5F74DFF02B0BDE8F087D5
:10D3F000019A224452E9032341462846D6F79CFA73
:10D40000019B234453F8042C32B951462846D5F7E2
:10D4100039FF033F0C3CDDE749462846D6F78CFA36
:10D42000F7E700BF6A1C0608FED005088E1C060838
:10D43000A31C060808B50246FFF77AFF064B0069F1
:10D44000984204D11046BDE8084008F013B80030F7
:10D4500018BF012008BD00BF995203080E2808B567
:10D46000014613D01E2813D0C20701D5401008BDB5
:10D47000830707D10268074B9A4203D1BDE80840F1
:10D4800003F0F8B90820FEF7BFFAF7E70020EEE74F
:10D490000120ECE7C02E0608C20705D4830705D19A
:10D4A0000268034B9A4201D103F0DCB9FFF7D6BF03
:10D4B000C02E06080E2810B50C4603D100230B60C1
:10D4C000012003E01E2802D10120086010BD10F0E9
:10D4D000010102D042102260F2E710F0030307D1ED
:10D4E0000168054A914205D103F0C4F92060E7E7DD
:10D4F0000846EBE71846E9E7C02E06080E2810B5E7
:10D500000C461DD01E281ED010F0010108D043107B
:10D5100000EE103AB8EEC00A84ED000A012010BDFA
:10D5200010F0030212D103680A498B4202D103F0C2
:10D53000DFFAF1E708498B420AD102F03EF9EBE746
:10D540009FED060AE8E7B7EE000AE5E70846E6E7DA
:10D550001046E4E7C02E06086C2A0608000000000A
:10D5600013B501A90446FFF7C9FF38B92046FFF7F4
:10D57000EBFE044902460448FEF7F7F99DED010A67
:10D5800002B010BD521C0608F42806080E28F8B593
:10D590000E46154604D100230B602B600120F8BD18
:10D5A0001E2804D14FF07E530B600023F5E710F0E6
:10D5B000010707D0431007EE903AF8EEE77AC1ED85
:10D5C000007AF2E710F0030414D103680B4FBB425A
:10D5D00004D103F08DFA86ED000AE6E7084FBB425E
:10D5E00002D102F0EAF8F6E7064DAB4204D101F0B1
:10D5F0000DF8D3E73846D2E72046D0E7C02E06081C
:10D600006C2A06083420060810B50446FFF7BEFF52
:10D6100038B92046FFF798FE024902460248FEF755
:10D62000A4F910BD4B1C0608F428060838B5840779
:10D6300003460ED104680B4DAC4203D1BDE838401F
:10D6400007F0ACB9084DAC4203D1BDE8384003F057
:10D6500001BD1846FFF778FE044902460448FEF76C
:10D6600084F900BFAC3E06082C300608301C0608C2
:10D67000F428060813B50C4601A9FFF7D7FF019B54
:10D68000A34204D0224603490348FEF76EF902B0D4
:10D6900010BD00BF391C06086C290608F7B51F46E7
:10D6A000D30706460D4614460ED554100194019A30
:10D6B000002A1DDA2A440192E7B1002A14DA002375
:10D6C0000193019803B0F0BD01A91046FFF7F2FEE7
:10D6D0000028ECD12046F588FFF736FE2A4603469F
:10D6E00009490A48FEF741F9AA42EAD90195E8E753
:10D6F000002FF9D1019B002B01DBAB42E1D3F28873
:10D7000003490448FEF731F90E1C0608F428060800
:10D710001F1C0608AC250608820701D002F0FDBFD9
:10D72000002801DA03F07CB8400040F001007047A7
:10D73000830710B5014610D102680D4B9A420CD1F7
:10D7400000F00703022B06D1C008F3F7D8FB400016
:10D7500040F0010010BD8068F9E70846FFF7E8FDDA
:10D7600043691BB10520BDE8104018471846F1E792
:10D770005C3906080E2810B5044621D01E2801D1B8
:10D78000012010BD06281BD0C20704D510F1FF30C0
:10D7900018BF0120F5E7FFF7CBFD436943B12146F0
:10D7A0000420984720B1A0F11E0358425841E8E7F1
:10D7B0002046FFF7BDFF0028E2D010F1FF30E7E779
:10D7C0000020DEE705282DE9F84F15BF1E260E269E
:10D7D0000E271E27914280460C46154607D1C807E2
:10D7E00020D40846FFF7A4FD838859071AD504F012
:10D7F0000703022B05D0A20717D122682B4B9A42B0
:10D8000013D105F00703022B05D0AB0712D12A680C
:10D81000264B9A420ED12946204605F0BDFC002831
:10D8200008BF3E463046BDE8F88F14F0010A06D026
:10D83000E80736D423464FF0010A2C461D46204601
:10D84000FFF776FDD0F818B08146BBF1000F11D07C
:10D850008288110704D42846FFF76AFD814509D163
:10D86000B8F1050F0DD0D9F818302A46214602200C
:10D87000984780B9BAF1000FDCD0AC4218BF3E46E1
:10D88000D0E7D306EFD52A4621464046D8470028A0
:10D89000E9D00646C6E7B8F1020F04D0FFF76AFFE9
:10D8A000BDE73E46BEE70646BCE700BF0C3C0608A7
:10D8B00008B50A4601460220FFF784FFBDE808408C
:10D8C000FFF758BF10B50446FFF732FF38B92046BE
:10D8D000FFF73AFD024902460248FEF746F810BD3E
:10D8E0005D1C0608F428060838B504461546FFF7FF
:10D8F0001FFD036A13B120469847A0B9204635B9E9
:10D90000FFF722FD084902460848FEF72EF8042DCD
:10D9100004D1FFF719FD06490246F5E7FFF714FDAC
:10D9200004490246F0E738BDB11C0608F428060891
:10D93000C41C0608D61C0608704710B50446FFF73D
:10D94000F7FCC36A2BB120469847B0FA80F0400933
:10D9500010BD1846FCE7000008B5FFF7EEFF10B950
:10D960000148FEF741FF08BD001C0608062806BF57
:10D97000480040F0010000207047042803D005282B
:10D9800007D0002070478B68002B14BF1E200E208C
:10D9900070478868400040F001007047074B0268FC
:10D9A000C1E900300023C1E90233054B9A4202BFAE
:10D9B0004368C3F317238B6008467047341D06087D
:10D9C000881E0608F8B50D460179044601F07F016E
:10D9D00016464020002208F0DFFAA368E2682768B4
:10D9E0002A6043436B60237903F07F01A9600849F3
:10D9F0008F4209D1190601D4B30707D46368C3F372
:10DA0000172300FB032028600020F8BD0120FCE75D
:10DA1000881E0608F8B5002205460E46014640203D
:10DA200008F0BAFA07461020F2F736FB094A0A4B0B
:10DA30000571012D18BF1346036043686FF31F2360
:10DA40000446C0E9013606FB07F0F2F725FBE0606B
:10DA50002046F8BD101E06084C1E06087FB5044679
:10DA60000122084601A9FFF777FF00222179402013
:10DA700008F092FA6368029DB5FBF0F5C3F3172234
:10DA8000AA42064619D2A16829444143E068F2F748
:10DA90001EFB6368E0606FF31F236360D4E9020339
:10DAA00005FB06F200FB0630019912F0FBF8A368B3
:10DAB00006201D44A56004B070BD521B62F31F23F5
:10DAC000EBE72DE9F041456835F0FF05044688464F
:10DAD0001ED101792A46402008F05EFA6368A168E9
:10DAE000082262F31F231144064641436360E06845
:10DAF000F2F7EDFA6168A268E060C1F3172101391D
:10DB000002FB0667384406FB01F2294612F00EF9C3
:10DB100043462079D4E9022108F06CFCA368013364
:10DB2000A3606368A3F5807363600620BDE8F0819D
:10DB30004268C36891688B4230B40AD21479D168C4
:10DB400082685D1CC5601A4404F07F0030BC08F098
:10DB500089BA002030BC70472DE9F047044686B0F2
:10DB60000D4616460AB90025C5E011F00307806886
:10DB7000DFF814A240F0D5800B687D4A934240F054
:10DB8000D0806A4607F0ABFE10B97A48FEF75AFE1D
:10DB90002179042E01F07F013A464FF0400000F059
:10DBA000938008F0F9F916F00302054658D133685E
:10DBB0007149186A884246D13179402001F07F01CD
:10DBC00008F0EAF9A84202D06C48FEF749FC336835
:10DBD0005345D6E9028904D17368C3F3172305FBC3
:10DBE0000399DDE900062368E768361A5345A8EB78
:10DBF000060637D194F90430002BB4DA002EE3D1B5
:10DC00006368C3F3172305FB037705FB08F2494656
:10DC100005FB007012F072F80199A2680098521A80
:10DC200040446A4305FB017105FB007012F066F881
:10DC3000A06805FB06F230445242002105FB00704B
:10DC400012F074F835E04E4A934209D1012DBBD150
:10DC50002A4603A93046FFF77FFEDDE90398C0E7B7
:10DC6000484893E7002ED0DD6368B6EB132F0BD93D
:10DC7000A168314438466943F2F729FA6368E060E5
:10DC800066F31F23074663600098A2680199404429
:10DC90003244121A6A4301FB057105FB007012F051
:10DCA0002DF8009805FB08F2494600FB057012F0BC
:10DCB00025F86368C6EB132262F31F236360A36831
:10DCC0001E44A660062516E008F066F92368534551
:10DCD000064614D11020F2F7DFF9054694E80F004C
:10DCE00085E80F00009A02EB112363F31F2169609E
:10DCF000019B9B1AAB60284606B0BDE8F087DDE9C2
:10DD000000312079C91AFFF785FEDDE90032E168AC
:10DD1000D21A0546724306FB0311C06811F0C2FF18
:10DD2000E9E700232A4601462068FFF7B7FC23688D
:10DD30005345024611D16368042E00EB13220ED026
:10DD400094F90430002BBFF60EAF2079E16833461A
:10DD500000F07F0008F04EFBB4E7042EF5D12079E7
:10DD6000E16800F07F0008F07DF90546C3E700BFD9
:10DD700058370608B61D060859DB0208DA1D0608E2
:10DD80005C390608F51D0608881E060870B50E28C1
:10DD900088B006460C46154651D003D8022865D0F7
:10DDA000002449E01B281FD02428F9D1012205A90D
:10DDB0002846FFF7C2FD00284AD0A10712D12268E9
:10DDC000364B9A420ED1012202A92046FFF7FAFDF6
:10DDD00001230093DDE90201DDE9052304F02CFCB9
:10DDE000002858D10E2427E0012202A92046FFF77F
:10DDF000E9FD2846012205A9FFF7AEFD00229DF8A6
:10DE00001010402008F0C8F8A168069DB5FBF0F599
:10DE1000064629449DF81000FFF7FCFD0446DDE9A5
:10DE20000212C06811F03EFFE068039B059905FBF4
:10DE300006F2184411F036FF204608B070BD0A689B
:10DE4000174B9A42ACD029462046FFF707FEF3E76E
:10DE5000EA0708D4AB07C5D12B68124A934202D017
:10DE6000114A9342BED10020FEF7ECFC012202A928
:10DE70002046FFF7A7FD012205A92846FFF75DFD13
:10DE80000028AFD0069B0093DDE90212059B3046C7
:10DE900007F064FDA4E71E24CEE700BF4C1E060871
:10DEA000881E0608C02E06086C2A06082DE9F043D5
:10DEB000012885B006460F4608D08B0724D10B6891
:10DEC000254A934202D0254A93421DD1012201A93D
:10DED0003846FFF732FDB8B100223146402008F045
:10DEE0005BF8029CB4FBF0F4074621463046FFF78E
:10DEF00091FD04FB07F205460199C06811F0D2FEBE
:10DF0000284605B0BDE8F0833846FFF711FCB8B1EC
:10DF1000441021463046FFF77DFD00210546384676
:10DF2000FDF790FF002780464046FDF7EBFF0346D4
:10DF30000028E5D034B919462846FFF7C2FDF3E7BB
:10DF40000446E6E73A4607F10109E968304608F079
:10DF500051FA4F46E8E700BF5C3906084C1E060838
:10DF600038B50D461C4611462846094AFEF7DAFE2A
:10DF7000206805F071F9012D007804D10021BDE879
:10DF80003840FFF747BD6168BDE83840FFF78EBFF6
:10DF900004000200F8B50E79012E05460C460ED19C
:10DFA0001A49D5F76FF93346D4E90221284604F01F
:10DFB00069FA28461649BDE8F840D5F763B93246F4
:10DFC0001449D5F7B9FCA368002BF2D01249134FBE
:10DFD0002846D5F757F90026A368B34204D810495C
:10DFE0002846D5F74FF9E4E71EB139462846D5F75C
:10DFF00049F93246E168207908F034F801220146F7
:10E000002846FFF7A9F90136E6E700BF981D060884
:10E010005D1D0708A41D0608AF1D0608B31D0608F0
:10E02000C82C070838B50C462046114606221D4666
:10E03000FEF778FE2CB921460120BDE83840FFF7F5
:10E04000E9BC2968CA070AD48B0703D10A680C4BBC
:10E050009A4204D00120BDE83840FFF727BF0846A8
:10E06000FFF7FCF9054601460120FFF7D3FC2A46DD
:10E0700004460021C06811F059FE204638BD00BF9B
:10E08000C02E060870B50446102015460E46F2F75D
:10E0900003F804714468044A02606FF31F24C0E966
:10E0A0000146C56070BD00BF881E06087FB51D46CD
:10E0B000084611464FF00212FEF734FE012201A974
:10E0C0002868FFF749FC9DF80C40029E214600227B
:10E0D000402007F061FF019AB6FBF0F12046FFF700
:10E0E000D1FF0322044601A92868FFF726FC18B1D6
:10E0F000237963F07F032371204604B070BD0000D4
:10E1000038B5054610200C46F1F7C6FF034A0260F9
:10E110000122C0E90125C46038BD00BF4C1E0608BD
:10E12000136870B56BB94468A51C50F825509C4223
:10E1300007D055F82360B14204D1023350F82330A0
:10E14000136070BD0133F2E72DE9F04788461449AA
:10E15000DFF85490DFF854A016460546D5F792F83C
:10E1600006F1080700247368A34205D828460D4924
:10E17000BDE8F047D5F786B81CB149462846D5F723
:10E1800081F858F8242051462846D5F7D5FB0122BE
:10E1900057F8041B2846FFF7DFF80134E3E700BF18
:10E1A000A13706085D1D0708B31D0608C41E060832
:10E1B0004B6802330A4651F82310FFF7C5BF0E29FA
:10E1C00014BF03210121FEF753B9052805D00E29FC
:10E1D00014BF03210121FDF717BC0020704738B59B
:10E1E0000C462046114602221D46FEF79BFD1CB13F
:10E1F0002868FFF7BFFA08B90E2038BD1E20FCE7DB
:10E20000032A05D10E2914BF04490549D5F73AB8A8
:10E210000E2914BF03490449F8E700BFF0080608B7
:10E22000F508060892F2050840EE0508136813B9D0
:10E230004068FDF71BBB70472DE9F84F994602EB8C
:10E2400043035D1C042B00AF82468B4690464FEA89
:10E2500085051ED805F10E0323F00703ADEB030D72
:10E260006C46002620462A1FB96A40F804BB11F00C
:10E2700019FD23464A4608F101015046FDF750FCBE
:10E28000044616B13046F1F72FFF2046BD46BDE8E3
:10E29000F88F2846F1F70BFF04460028DAD006462F
:10E2A000E0E707B5009313460A46D0E90101FFF7FE
